:100000000C94031B0D949C330D9471330D94463363
:100010000D941B330D94F0320D94C5320D949A3229
:100020000D946F320C94341B0C94341B0C94341BC1
:100030000C94341B0C94341B0C94341B0D94EE4E16
:100040000C94341B0C94341B0C94341B0C94341BF4
:100050000C94341B0C94341B0C94341B0D94FC2E08
:100060000C94341B0D944D360D9423360C94341B94
:100070000C94341B0C94341B0C94341B0C94341BC4
:100080000C94341B0C94341B0C94341B0C94341BB4
:100090000D94B13A0D94273A0D94693A0D94B453E6
:1000A0000C94341B0C94341B0C94341B0C94341B94
:1000B0000C94341B0C94341B0C94341B0C94341B84
:1000C0000C94341B0C94341B0C94341B0D94ED35A0
:1000D0000D94C3350C94341B0C94341B0C94341BBA
:1000E0000C94341B07634236B79BD8A71A3968565D
:1000F00018AEBAAB558C1D3CB7CC5763BD6DEDFD4A
:10010000753EF6177231BF000000803F0800000006
:10011000BE922449123EABAAAA2ABECDCCCC4C3EFC
:1001200000000080BEABAAAAAA3E00000000BF00EB
:100130000000803F0000000000084178D3BB4387E7
:10014000D1133D190E3CC3BD4282AD2B3E68EC82FB
:1001500076BED98FE1A93E4C80EFFFBE01C4FF7F80
:100160003F00000000000D94D5280C944AFC0D942B
:100170003F2B0D9482070C94B7290C94BB5D0D9412
:1001800052060D9477280C94E9F60C943E1E0D94BB
:10019000C8460D94C2420C9479360C946D680C9448
:1001A000C0FD0C945EFC0C9481BD0D9427070D944A
:1001B000AD010C9431FC0C94E0280C94CD310C94DE
:1001C000F1AE0D9437060C94BFB90C94FE400D941B
:1001D000C2480C94E3700C94251C0D946D2C0C9467
:1001E000FB6B0C9449AE0C9493240C94FA1D0C9464
:1001F00073D70D942B060D943B070C9490320D94FD
:1002000078070C94117A0C947F540D945F070C942A
:1002100079630C94D3300C94AD1B0C94D5CA0C9418
:10022000C7B90C9459D00C9490AD0C9406330C942F
:10023000951B0C94991B0C9445240C94BD600D9453
:100240002B2D0C9463D20C94775B0C94C1AE0C9460
:100250008E310C94AEAE0C9437D00C9478540C9430
:100260003ACF0C94961C0D94A34A0D949C4D0C947B
:10027000399F0C94A8AE0C9487B50C943ABC0D949D
:1002800091010C949FE50C94BAEF0D94E90B0D9439
:100290006D2E0C94A7900C944E1D0C94C2B10D942D
:1002A000BB290D943A060D94E2340C94E0900C9422
:1002B00052B80D94D7480C941C680C94E2A20D948B
:1002C0009B2D0C9427FC0D9483010C94AA8F0D9404
:1002D00069070C94EAAE0C946CBC0C943C320D94FF
:1002E0000E480C9427BC0D941A4A0D94C92A0C94FC
:1002F0009B310C9495AE0C945E2F0C94A45B0C94E3
:1003000082CF0C9453200C94BEA10C94881B0C94A7
:10031000CAA20C94A7390D947D2C0C94A5A20D941F
:10032000A1440C94EEAE0D9460060C94B1AD0C9407
:100330003BE20C9426700C9423700C94E3290C94EB
:10034000B9B90C9424700C9472310C94572F0C94FE
:1003500024A20D94A6010C94D7F60C942FE30C94D0
:10036000B85D0C94E8240C94C07A0C9435E70C9496
:1003700053E50C94D7280C94635B0C9428D00C9410
:1003800097900C94BF5D0C9400B70D94312A0C9497
:10039000DA280C94EA900C945FAA0D94F4560C940D
:1003A000B8900C9454FC0D9472430C9456320C94F7
:1003B000C2B90C9451AE0C94557C0C94AE320D9491
:1003C000724A0D94C74D0D9476280C9468FC0C94D9
:1003D000A91C0D9474280C945A350C94717A0C94C1
:1003E00060280C94AD7A0C9474E20C94E51B0D9487
:1003F0005C060C944DAE0C94322F0C9465250C9435
:10040000F2E50D9482440D9431070C9467280C9406
:1004100062BC0C9412AF0C945F1B0D94B3280C9427
:10042000D2FD0D94AA430C94985D0D94CB440D9489
:10043000024E0D944A2A0C940CBC0D94DA3D0C9497
:10044000E6320C9465D20C9449B80C94CE230D94EA
:1004500064290D94582B0D94B23D0C947DD00C94CE
:10046000FB290C948A1B0C94C25C0C94BA5B0C9410
:100470007E1B0C9400E30C9461210C94EB7B0C9498
:100480006BAE0C94665D0C940BFE0D94FE290C94DF
:1004900025740D9465480D94E60B0C945C310C9416
:1004A0004F610C94E87F0D9425060C9463BA0C946C
:1004B00071320C9479D70C94BA440C94BD5D0C94B1
:1004C000C36C0D94D80B0C944B350D94BA2A0D9433
:1004D0001D070C94B0600D94062C0C9430CA0C943B
:1004E00063320C9425700C947D320D94512B0C9436
:1004F0002BAB0C9409FC0D94872B0D9422430D9487
:100500006C2C0C9413320C94155E0D9498010D9480
:1005100017290C94F7C90C9490A20C948FD20C94C8
:10052000C75B0C94482F0C9457FD0C9486A70C9431
:100530001AE30C94B0290C94271C0C94622F0C9491
:1005400040FC0D9496070C945F5E0D9487480C94C4
:10055000821C0D9466060D94E52B0C9477390C944F
:100560006D7C0C949FCA0D94A0070C9422700D947E
:10057000B4010C94A8290C9458560D94772D0D9421
:100580007E560C94D2E50D9444060C9426FD0D94F1
:10059000F32C0C947A680C9455250C94E7900C94E9
:1005A000D6290C94DD290C94FFB00C9482E60C94AF
:1005B000BE1B0D944E060C9446A20C9499290D94E2
:1005C00040060C94D4AE0C942EF70C94C35D0D949D
:1005D000D70B0C94175E0C949CD00C9482320C9424
:1005E000A5280C94D0F60C947E1C0D9455070C9401
:1005F0003BE70C94CF250C94B1320D9458060C9423
:100600001F620C947A1C0C941DE30C941FAB0C9489
:1006100015BC0D944A060C94A0630C9433690D9498
:10062000972C0D94892E0D94902C0C9481240C946D
:100630005E220C9429E50C94EB310C94C5B80C9413
:1006400032230D945B470C94BEB80C94ED7C0C9453
:10065000B9A20C94FDE20C944CB80C942FE70D94C5
:10066000B8290C9408CB0C9418530C94DD900C947E
:1006700060E20C947A1B0C94D6300C94761B0C948C
:10068000925B0C94467D0D942F060D94152B0D94C2
:100690006E2C0C9487E20C9409D00D948A010C9472
:1006A00040AF0C94F8ED0C94BD310C94775D0D9433
:1006B00033060C9463E70C9477BC0C949D1B0C944C
:1006C0009C390C9417F70C94AC5C0D94992D0C94F8
:1006D0006BA20C940CE30D94E2460C9430910C94B4
:1006E0000FE30D9443070D94E62A0C9440FD0C94FF
:1006F0000BE60C943D2F0C94C15D0C94BF5C0C94E4
:1007000079BC0C948D1B0D94C42C0C94ACAE0D9440
:1007100044470C948BAE0C94575D0D94072B0C94AE
:10072000573A0C94D07A0C94B7670C94B9300C9467
:100730001A7D0C9455AE0C94F5E40C942F5C0C943B
:10074000F7640C9449E60C9454630C94EC290D94D2
:10075000C7280C941B5C0C9441AE0C94A0790C94AB
:10076000195E0C9427630C94E2790D94FB2B0D9485
:10077000CF2B0C9434280C9413680C9426B10C9451
:100780006AD70C94F9BB0C949D310C949F560C9431
:1007900090290C94BCB90C945DE70C9445AE0C9474
:1007A0005E5A0D9403470D942D4E0D94AA070C9498
:1007B00002BC0C94EB250C94F5300C94C95C0C94A1
:1007C00006A30D9410070C94D4B50C9469240C94D2
:1007D000407C0C9469E60C94FBE10C94B4250C94D9
:1007E00037FD0D946C4D0C949E300C9432320D9468
:1007F000B1290C9474AA0C946AA00C946D1B0C94EF
:1008000081D00D9465060C94024D0C94FECE0D948F
:1008100063430C94EB300C944EBC0D94132D0C944C
:10082000CBCF0D94C1290C947B1E0C94DD5B0D94F1
:10083000A4280C94291C0C945B5B0C9498BB0C941E
:100840008F700C94B6B90C941AAB0D948C070C9461
:1008500066710C9419FC0C942A780D944B070D9436
:1008600028350D949C2A0C94FE310D94384A0C9432
:10087000ED600D946A060D9475280C94745D0C94CB
:10088000F2E20C94621B0C9454900C94611D0D9434
:1008900018070C94F8F60C9407B10C9459AE4E411D
:1008A0004E494E495459494E46CDCCCC3D0AD723EA
:1008B0003C17B7D13877CC2B329595E6241FB14F32
:1008C0000A000020410000C84200401C4620BCBE77
:1008D0004CCA1B0E5AAEC59D746364696E6F70730B
:1008E0007578585B0020002D3E00436F6E76657270
:1008F00074696E6720002D3E0057726F6E6720414D
:10090000737369676E6D656E742000524742783A62
:10091000200020764C6576656C3A0020436F6E7639
:10092000563A0020436F6E76533A0020486F743A6F
:1009300000436F6C643A0020436F6E766572746595
:100940006420563A00436F6E766572746564205376
:100950003A002D3E0057726F6E67204173736967CE
:100960006E6D656E7420002D3E0057726F6E6720AD
:1009700041737369676E6D656E7420004D41503A26
:100980002076616C206D617070656420746F20202A
:10099000004D41503A2076616C75652061626F763A
:1009A0006520726967687420626F756E642000202C
:1009B00069732062656C6F77206C65667420626F66
:1009C000756E6420004D41503A2076616C7565204B
:1009D000004D41503A20636D64206D617070656414
:1009E00020746F2000000000000000000000004F95
:1009F0004E00000000000000004F464600000000CE
:100A000000000052455354000000000000544F47BE
:100A1000474C450000000048414C540000000000D5
:100A200000584F4E00000000000000584F4646009E
:100A30000000000000494E43524541534500004428
:100A4000454352454153450000454E41424C450007
:100A500000000044495341424C45000000554E46B9
:100A60005245455A450000465245455A450000004A
:100A7000004155544F00000000000046414E5F4FBA
:100A80004E4C590000484947480000000000004D06
:100A9000454449554D000000004C4F5700000000F0
:100AA000000000484541545F434F4F4C00484541CA
:100AB00054000000000000434F4F4C0000000000B5
:100AC000004452590000000000000052474200005C
:100AD00000000000004853560000000000000052D3
:100AE00045534554000000000020537566663A00E7
:100AF0002041543A0053746F7070696E6720496EDC
:100B00007075747300206973200044656C657469A6
:100B10006E6720636F6E662E2052414D20776173A1
:100B20003A0053746F70706564006E6F7468696E1C
:100B30006720746F2073746F700053746F707069E6
:100B40006E67206368616E6E656C73202E2E2E00BA
:100B500043616E206E6F7420636C65616E202D2082
:100B60006C6F636B656400436F6E666967206368D2
:100B7000616E676564206C6F63616C6C792C2070AA
:100B80006F7274616C2064697361626C6564002FBC
:100B9000636F6E6669672E6A736F6E007265626F4F
:100BA0006F742000436D643A20002F636F6D6D6198
:100BB0006E642F002F72616D2F002F6974656D2F89
:100BC000002F6974656D2F0022687474703A2F2F9E
:100BD0006C617A79686F6D652E72752F70776122FE
:100BE000004C6F636174696F6E3A20687474703A78
:100BF0002F2F003F6D61633D002669703D00267018
:100C00006F72743D00266E616D653D002F002000FF
:100C10004D5154543A20436F6D706C6574652E20AD
:100C200052656D6F766520746F7069632000246370
:100C30006F6D6D616E64004D5154543A20436C6584
:100C4000616E55702072657461696E656420746FA1
:100C50007069632000220022004F75744F664D6555
:100C60006D6F727921005D20003A5B004D51545444
:100C70003A005D00456D7074793A205B000A003AD5
:100C8000004D41433A00554450205379736C6F67CF
:100C900020696E697469616C697A65642E0A005313
:100CA00079736C6F6720706172616D733A002E6C9E
:100CB0006F63616C0053657276696365207265636A
:100CC0006F72643A20006D444E5320726573706FEA
:100CD0006E64657220737461727465642E0045726F
:100CE000726F722073657474696E67207570204D21
:100CF000444E5320726573706F6E646572210047B5
:100D00006F7420495020616464726573733A0027E0
:100D10006970205B69705B2C646E735B2C67775B1A
:100D20002C7375626E65745D5D5D5D27202D20738B
:100D30006574207374617469632049500A004661C8
:100D4000696C656420746F20636F6E666967757285
:100D5000652045746865726E6574207573696E6789
:100D600020444843502E20596F752063616E2073D4
:100D70006574206970206D616E75616C6C792100FD
:100D8000204D41534B3A002047573A0020444E53E0
:100D90003A004C6F616465642066726F6D20666C0A
:100DA0006173682049503A000A757365732044489E
:100DB00043500A005374617274696E67206C616EEF
:100DC000004142434445464748494A4B4C4D4E4FEB
:100DD000505152535455565758595A61626364657D
:100DE000666768696A6B6C6D6E6F7071727374752B
:100DF000767778797A303132333435363738392B63
:100E00002F3D00426173696320003A004F54412036
:100E1000696E697469616C697A65640A0044454663
:100E200041554C542070617373776F726420666F04
:100E300072204F5441204150492E20557365206F38
:100E4000746170776420636F6D6D616E6420746F80
:100E5000207365740070617373776F7264004D5115
:100E600054543A2074727969796E67206E656E7891
:100E7000742062726F6B6572004D5154543A205465
:100E80006F6F206D616E7920636F6E6E656374693C
:100E90006F6E206572726F72732E2052657374616B
:100EA0007274204C414E0020747279206167616930
:100EB0006E20696E2035207365636F6E6473004D1C
:100EC0005154543A206661696C65642C2072633D0C
:100ED000004D5154543A204177616974696E67201E
:100EE000666F722072657461696E656420746F70DC
:100EF00069637300636F6E6E65637465642061730C
:100F00002000202E2E2E0020757365723A003A00C4
:100F10000A4D5154543A20417474656D7074696E71
:100F20006720636F6E6E656374696F6E20746F20E7
:100F300000646973636F6E6E6563746564005573F6
:100F4000696E67204D5154542070617373776F72CE
:100F5000642066726F6D20636F6E666967002E6C29
:100F60006F63616C006D444E53206E616D6520753A
:100F70007064617465643A20004465766963652035
:100F80004E616D653A004D5154543A204174206CC5
:100F90006561737420646576696365206E616D6553
:100FA00020616E642062726F6B6572204950206D03
:100FB00075737420626520636F6E6669677572650C
:100FC0006400757074696D652C667265656865612D
:100FD0007000353635313935645F323032362D3078
:100FE000352D3235004C69676874487562200024DD
:100FF0006E616D6500526562696E6420737563632E
:101000006573732E20495020616464726573733A6E
:10101000004572726F723A20726562696E64206672
:1010200061696C0052656E657765642073756363F2
:101030006573732E20495020616464726573733A3E
:10104000004572726F723A2072656E657765642032
:101050006661696C000A4E6F206C696E6B00436FAD
:101060006E74696E75652077697468207072657634
:10107000696F75736C79206C6F6164656420636F50
:101080006E6669670033307320454550524F4D20DE
:101090006973206E6F742072656C6F616465642E75
:1010A000205265626F6F74004D5154543A20416371
:1010B00063657074696E6720636F6D6D616E6473D4
:1010C0002E2E2E0A004E6F204D51545420636F6E09
:1010D00066696775726564004C6F6164696E67204C
:1010E000636F6E6669672066726F6D20706F7274D1
:1010F000616C2064697361626C65642E2075736530
:1011000020676574204F4E20746F20656E61626C9D
:101110006500436F6E6669672069732076616C694C
:101120006400436F6E74696E75652077697468201A
:1011300070726576696F75736C79206C6F61646528
:101140006420636F6E666967005365747570204F25
:101150005441004D5154543A2073657420666972AD
:1011600073742062726F6B65720043757272656E84
:1011700074204C414E20636F6E6669672869702C3D
:10118000646E732C67772C7375626E6574293A00F0
:101190000A55736520746865736520636F6D6D61B2
:1011A0006E64733A202768656C7027202D20746860
:1011B000697320746578740A276D61632064653AE9
:1011C00061643A62653A65663A66653A303027206E
:1011D00073657420616E642073746F7265204D4175
:1011E000432D6164647265737320696E20454550B8
:1011F000524F4D0A276970205B69705B2C646E73D7
:101200005B2C67775B2C7375626E65745D5D5D5DED
:1012100027202D20736574207374617469632049DD
:10122000500A277361766527202D2073617665202B
:1012300063757272656E7420636F6E66696720698C
:101240006E204E5652414D3B204F4E7C4F4646201D
:101250002D20656E61626C652F64697361626C65D7
:10126000206175746F736176650A2767657427203E
:101270005B636F6E66696720616464725D27202D11
:101280002067657420636F6E6669672066726F6D94
:10129000207072652D636F6E666967757265642074
:1012A00055524C20616E642073746F7265206164C6
:1012B00064722C204F4E7C4F4646202D20656E6177
:1012C000626C652F64697361626C6520646F776E10
:1012D0006C6F6164206F6E20737461727475700A34
:1012E000276C6F616427202D206C6F616420636F11
:1012F0006E6669672066726F6D204E5652414D0AC8
:101300002770776427202D20646566696E652061EB
:101310006E642073746F7265204D51545420706157
:101320007373776F72640A276F7461707764272014
:101330002D20646566696E6520616E642073746F2C
:101340007265204854545020415049207061737395
:10135000776F72640A276C6F67205B7365726961CF
:101360006C5F6C6F676C6576656C5D205B75647037
:101370005F6C6F676C6576656C5D27202D206465FA
:1013800066696E65206C6F67206C6576656C2028D9
:10139000302E2E37290A276B696C6C27202D20747C
:1013A000657374207761746368646F670A27636C80
:1013B00065617227202D20636C6561722045455060
:1013C000524F4D0A2773656172636827202D207381
:1013D000656172636820312D776972652064657676
:1013E0000A277265626F6F7427202D207265626F05
:1013F0006F7420636F6E74726F6C6C657200536FE4
:101400006674207265626F6F74696E672E2E2E008F
:10141000206E65770020697320003157543A0031FF
:1014200057543A20536561726368696E672064653A
:10143000760052414D3D000A5379736C6F6720006E
:101440000A312D7769726520000A6D71747420006D
:101450000A6D6F64627573207632000A6D6F646284
:10146000757320763120282B29000A696E707574F7
:101470007320000A6974656D7320000A436F6E66FD
:101480006967757265643A002F00496E3A20004919
:101490006E697469616C697A696E6720496E7075EE
:1014A0007473003157543A207365747570207265F7
:1014B000736F6C7574696F6E20003157543A204415
:1014C00053323438322D313030206E6F74207072C8
:1014D0006573656E74003157543A20445332343882
:1014E000322D3130302049324320726573746F726F
:1014F0006564003157543A204275732072657365F4
:1015000074206572726F72003157543A20427573BD
:1015100020526573657420646F6E65003157543ACC
:10152000204453323438322D31303020707265739C
:10153000656E742C207265736574004572726F72EB
:1015400020312D7720696E6974003157543A204458
:1015500053323438325F3130305F4932435F544F59
:101560005F31575F42524944474520696E697400B4
:10157000444D584F75742E20467265653A00444DAF
:1015800058696E2042756666657220616C6C6F6387
:101590002065727200496E697420696E2063683A32
:1015A000003B003D0050696E3A003B003D4C4F57F8
:1015B00000546865726D6F3A004F6E6520776972EE
:1015C000652052656164790A00467265653A004497
:1015D0004D58206F757420737461727465642E2089
:1015E0004368616E6E656C733A2000444D58206903
:1015F0006E20737461727465642E204368616E6E30
:10160000656C733A0042726F6B65727320636F6E24
:10161000666967757265643A004170706C79696ECD
:101620006720636F6E666967004C6F616465642054
:10163000455441473A004E6F2073746F72656420C1
:10164000636F6E666967004C6F61646564206672E3
:101650006F6D20454550524F4D006C6F61642066A0
:1016600061696C6564004A534F4E2064657465631C
:10167000746564004C6F6164696E6720436F6E66C9
:1016800069672066726F6D20454550524F4D00438B
:101690006F6E666967206175746F736176653A0075
:1016A0000A5379736C6F67206465627567206C6597
:1016B00076656C3A0053657269616C206465627589
:1016C00067206C6576656C3A0053617665640A0044
:1016D0005365742064796E616D69632049500A0016
:1016E0004F54412050617373776F7264207570643A
:1016F000617465640A004E6F204950206164726510
:10170000737300205361766564004C6F6164696E89
:1017100067204854545020636F6E666967206F6E6F
:1017200020737461727475703A000000000000004C
:10173000000000004F4E00000000000000004F4677
:101740004600000000000000524553540000000015
:101750000000544F47474C450000000048414C549E
:10176000000000000000584F4E0000000000000084
:10177000584F4646000000000000494E4352454184
:101780005345000044454352454153450000454EF2
:1017900041424C450000000044495341424C450041
:1017A0000000554E465245455A45000046524545B3
:1017B0005A45000000004155544F00000000000051
:1017C00046414E5F4F4E4C59000048494748000083
:1017D000000000004D454449554D000000004C4FAD
:1017E0005700000000000000484541545F434F4F40
:1017F0004C0048454154000000000000434F4F4C4E
:1018000000000000000044525900000000000000E9
:1018100052474200000000000000485356000000FC
:101820000000000052455345540000000000636F63
:10183000756C64206E6F742070617273653A20005D
:10184000557064617465640A00454550524F4D20DF
:10185000636C65617265640A004D51545420506197
:101860007373776F726420757064617465640A00C5
:101870002B002D00455461673A20004765742045D0
:101880005441473A2000485454502F312E310025FE
:10189000733A2025730D0A0020485454502F312EDE
:1018A000310D0A486F73743A2025730D0A41636342
:1018B0006570743A202A2F2A0D0A436F6E6E656395
:1018C00074696F6E3A20636C6F73650D0A0025733F
:1018D0000020000D0A00474554006661696C65648C
:1018E00020746F20636F6E6E6563740A00455252F8
:1018F0004F523A2053657276657220726574757224
:101900006E65642000436F6E666967206E6F742099
:101910006368616E6765640A00446F6E652E0A0035
:10192000436F6E6669672070617273696E672066C7
:1019300061696C65640A004765742061626F727446
:10194000656400676F7420436F6E6669670A00689C
:1019500074747020726574636F64652000667265CC
:10196000652000436F6E666967205552493A2068CA
:101970007474703A2F2F002044656661756C742072
:10198000636F6E6669672073657276657220757322
:1019900065643A20006C617A79686F6D652E7275A6
:1019A000000A282D294352595054000A282D295045
:1019B000554C5345206F6E2050494E3132000A2855
:1019C0002D2943414E000A282D29535052494E4B90
:1019D0004C4552000A282D294D4552435552590075
:1019E0000A282B294D554C544956454E54000A2877
:1019F0002B2950574D5F52454C4159000A282B293D
:101A00004D444E53000A282D295541525442524903
:101A1000444745000A282B295359534C4F47000A85
:101A2000282B29504944000A282D294D4350323390
:101A3000303137000A282D294152544E4554000AAE
:101A4000282B294F5441000A282D29535049204C56
:101A50004544000A282B294D4F544F5220435452DD
:101A6000000A282D294143204841494552000A28AF
:101A70002D29434353383131202620484443313007
:101A80003830000A282B29524553544152545F4C98
:101A9000414E5F4F4E5F4D5154545F4552524F522D
:101AA00053000A282D294841524452455345542C8D
:101AB000207573696E6720736F6674000A282B297E
:101AC000434F554E544552000A282B294448540090
:101AD0000A282B294453323438322D313030000A51
:101AE000282B294F57495245000A282D2949504D86
:101AF0004F44425553000A282B294D4F4442555319
:101B000020307830362061742053657269616C3200
:101B10002073706565643A39363030000A282B2905
:101B20004144414652554954204C4544000A282B13
:101B300029444D58000A282B2957697A6E65743557
:101B4000783030000A282B294672656552616D2075
:101B50007072696E74696E67000A282B29574154A8
:101B60004348444F47006C617A79686F6D652E7207
:101B700075000A436F6E66696720736572766572D9
:101B80003A003230313130334C0020432B2B207659
:101B9000657273696F6E3A00353635313935645F79
:101BA000323032362D30352D3235000A4C617A799B
:101BB000686F6D652E7275204C6967687448756230
:101BC00020636F6E74726F6C6C65722000204F46DC
:101BD0004600204F4E00204259504153530053615C
:101BE00076656420746F20454550524F4D00536117
:101BF00076696E6720636F6E66696720746F204533
:101C00004550524F4D2E2E00556E6B6E6F776E20E5
:101C10007375666669782000556E6B6E6F776E20FF
:101C2000636D642000436F756E7465723A200044E2
:101C30004D582D4F757420496E69743A2000444DFB
:101C4000582D4F75742073746F703A200041737370
:101C500069676E65643A00444D58206374726C3A4B
:101C600020006931360001693332000275313600D7
:101C7000037533320004693868000569386C000662
:101C8000753868000775386C000878313000093104
:101C90003030000A44656661756C74207365726942
:101CA000616C206D6F6465204E38312075736564FA
:101CB00000384531002600384E31000600384532E4
:101CC000002E00384E32000E00384F3100360038FA
:101CD0004F32003E00374531002400374532002C9A
:101CE00000374F31003400374F32003C00374E315F
:101CF000000400374E32000C0020616464656420EB
:101D00006279206E756D20004D4255533A20004196
:101D10006464696E672072656773207769746820F0
:101D2000616374696F6E733A004D4255533A0041D6
:101D30006464696E6720726566657272656420729C
:101D40006567733A004D4255533A00416464696EC9
:101D50006720707265666574636820726567733AA0
:101D6000004D4255533A004D4255533A204D6F6451
:101D70006275732074656D706C617465206E6F742C
:101D800020666F756E643A20004D4255533A2049E3
:101D90006E76616C69642074656D706C6174652E1B
:101DA000002C002C002C002C004D4255533A20638F
:101DB0006F6E666967206661696C65643A004D42C2
:101DC00055533A20636F6E666967206572726F7251
:101DD000004D4255533A20636F6E666967206C6F01
:101DE0006164656420004D4255533A204F7574205C
:101DF0006F66206D656D6F7279004D4255533A20C4
:101E0000506F6C6C696E67206572726F7220004D46
:101E10004255533A204E6F7420737570706F727410
:101E200065642072656720747970650A004D4255BB
:101E300053443A2049676E6F726564202D206571A6
:101E400075616C20776974682073657474656420AB
:101E500076616C004D425553443A204D6170706577
:101E6000643A004D425553443A204E65737465649C
:101E70004D61707065643A004C6173744B6E6F779E
:101E80006E2076616C75653A2000536561726368F7
:101E9000696E67207265673A2000206F7574206F45
:101EA000662072616E6765206275666665722C20B9
:101EB0006665746368696E6700646566207265674D
:101EC0002320004D425553443A20536561726368A4
:101ED000696E672072656723003A002066726F6D35
:101EE000207479706520004D425553443A20676F45
:101EF0007420002076616C3A0020004D425553203A
:101F00007265733A20002076616C206E6F742063D6
:101F100068616E6765642E20436F6E74696E7565C7
:101F2000004D4255533A003A20657175616C20743A
:101F30006172676572742E003D004D4255533A0040
:101F40002076616C206368616E6765642E004D4287
:101F500055533A00204E6F773A00204C6173743A23
:101F6000002023002070726566657463682000207D
:101F70005265672F636F696C206D7573742062659D
:101F800020696E740020696E7465726E616C2073D6
:101F9000656E64206572726F72202D206E6F2072E4
:101FA00065672F636F696C0020696E7465726E617E
:101FB0006C2073656E64206572726F72202D206EC6
:101FC0006F2074656D706C6174650020696E746556
:101FD000726E616C2073656E64206572726F722020
:101FE0002D206E6F2073746F7265004D42555344FF
:101FF0003A20656E64506F6C6C20004D425553441E
:102000003A20506F6C6C2000206E6F7420666F75E4
:102010006E64004D4255533A2020706172616D200C
:10202000002073656E64696E672063616E63656C22
:102030006C6564004D4255533A2020706172616DA9
:1020400020004D4255533A2020002073656E6420D5
:102050006572726F722E20004D4255533A20200057
:102060004164642040563A20002056616C3A2000BA
:102070004D425553443A207375666669783A00209C
:102080006F722073756666697820004D4255533A29
:10209000204E6F2074656D706C61746520666F7280
:1020A00020004D6F746F723A2074696D656F75749E
:1020B00000556E6B6E6F776E20636D64004D6F74AC
:1020C0006F723A20466F7263656420657865637548
:1020D00074696F6E0056454E543A20636F6E6669A0
:1020E00067206661696C65640056454E543A206904
:1020F0006E69740056454E543A2050494420503D74
:102100000056454E543A2044652D496E6974005678
:10211000454E543A2070617373697665206D6F6423
:10212000653A20006E6F74204F4B004F4B005645B0
:102130004E543A204354524C20726573756C743A75
:10214000200056454E543A204354524C2066616E4E
:10215000206C6576656C3A2000204F75743A00203B
:102160005265713A0056454E543A2000206D3300B6
:102170002066726F6D2000204D6178207265713A83
:10218000002066616E253A002061637469766520DF
:10219000563A0056454E543A20546F74616C20569E
:1021A0003A002075706461746564206279207465FA
:1021B0006D703A200056454E543A205049442069EB
:1021C0006E7075743A200056454E543A207A6F6E00
:1021D000652066726F7A656E0056454E543A207AD5
:1021E0006F6E652066726F7A656E0056454E543A82
:1021F0002046414E20636F6E74726F6C2064697369
:1022000061626C6564206279205049440056454EF5
:10221000543A207A6F6E652066726F7A656E00415F
:1022200043206D6F64653A200056454E543A2000B5
:1022300056454E543A20626F6F7374206D6F64651B
:10224000206465746563746564004143207365743C
:102250003A200056454E543A200041432066616EB4
:102260003A200056454E543A20004143206169729D
:102270002074656D703A200056454E543A20005641
:10228000454E543A2053746F7020616C6C207A6F05
:102290006E65732E200056454E543A205265737475
:1022A0006F726520616C6C207A6F6E65732E2000F2
:1022B0002074726573686F6C643A0056454E543AE8
:1022C000204368616E2062616C616E63653D002031
:1022D0006F75743A0056454E543A20434F4F4C2088
:1022E00050415353205049443A2000206F75743AAE
:1022F0000056454E543A20484541542050415353CE
:10230000205049443A2000203C414C4D3E00206F73
:1023100075743A00207365743A0020696E3A00566D
:10232000454E543A200056454E543A2050494420D8
:1023300073657420746F204D414E55414C20647577
:1023400065206E6F20484541542F434F4F4C2E203F
:102350007A6F6E653A005049443A20616C7265614B
:10236000647920696E697469616C697A656400508A
:1023700049443A20496E76616C69642070617261EB
:102380006D2061727261792E002C002C002C002CC3
:10239000005049443A20636F6E6669672066616940
:1023A0006C65643A005049443A20636F6E66696711
:1023B000206572726F72005049443A20636F6E66F6
:1023C0006967206C6F6164656420005049443A205D
:1023D0004F7574206F66206D656D6F72790050497E
:1023E000443A2044652D496E69742000203C414CDC
:1023F0004D3E0020443A0020493A0020503A002047
:10240000696E3A00207365743A005049443A2000DE
:102410005049443A20496E76616C6964207061725B
:10242000616D2061727261792E00536574206F7541
:102430007420746F20002050494420616C61726DDB
:102440002E20002050494420616C61726D3A206357
:102450006C6F736564005049443A20556E6B6E6F23
:10246000776E2073756666697820005049443A207B
:10247000556E6B6E6F776E20636D6420005049441B
:102480003A2072657365740020536574706F696ECD
:10249000743A005049443A200020496E7075742007
:1024A00076616C75653A005049443A200020696EA7
:1024B000697400200050574D2D4F75742023002063
:1024C00073746F7000200050574D2D4F757420238A
:1024D000003D0050696E3A0020696E6974007069B1
:1024E0006E230072656C61794374723A2000207328
:1024F000746F700052656C61792D4F7574202300E4
:1025000072656C61794374723A200069646C65008D
:102510006F66660068656174696E670066616E006B
:10252000647279696E6700636F6F6C696E670061D2
:102530006374696F6E0020697320004F757420000A
:1025400072656C61794374723A2000556E6B6E6FE0
:10255000776E20737566666978200072656C6179A4
:102560004374723A2000556E6B6E6F776E20636D08
:1025700064200072656C61794374723A2000616373
:1025800074696F6E0072656C61794374723A2000F1
:102590005B305D3A2000202D202D202D20EFBBBF89
:1025A000003E003E31202D20005B305D3A200020AF
:1025B0002D202D202D20EFBBBF003E003E31202DD1
:1025C00020005379736C6F6720726573756D656455
:1025D000005379736C6F6720726573756D65640065
:1025E0005379736C6F672073757370656E6465647F
:1025F000000000000000636D64000073657400005B
:1026000076616C000064656C00004853560000520F
:102610004742000066616E00006D6F646500637480
:10262000726C006875650000736174000074656DFC
:102630007000726177000020002E00696E00735FE9
:102640006F7574006D79686F6D65004354524C2F3F
:10265000657865633A204F75744F664D656D6F728E
:10266000793A2000202D3E20004D5154543A20004C
:10267000202D3E2000456D69743A203C00202D3EFF
:1026800020004974656D436D643A2000202D3E2082
:10269000004974656D3A2000556E6B6E6F776E2041
:1026A0007375666669782000556E6B6E6F776E2065
:1026B000636D642000636C724374723A2000444D71
:1026C00058494E3A00454F46003D00494E3A0025D4
:1026D00000C2B04320483D002044485432322074A8
:1026E0007970652E20543D00494E3A00204E6F20EF
:1026F000656D69742064617461210020436F756E9B
:1027000074657220747970652E2076616C3D004985
:102710004E3A0020436F756E74657220747970654F
:102720002E20494E434F525245435420496E746502
:102730007272757074206E756D6265722121210050
:102740004952513A00416374697661746520696E3B
:102750002000416374697661746520696E20002DE4
:102760003E00200023002D3E00200050656E646571
:10277000643A2023002D3E00456D69743A002D3ED9
:1027800000456D69743A002D3E00456D69743A004C
:102790002D3E00456D69743A003D004C454741436C
:1027A0005920494E3A0020666F7220286D73293AED
:1027B000004354524C3A205363686564756C65203D
:1027C000636D642000206D730020666F72200043EB
:1027D00054524C3A2041726D656420002044697364
:1027E00061726D6564004354524C3A200020746954
:1027F0006D653A004354524C3A205265733A004397
:1028000054524C3A206D6F6D656E7461727920651B
:1028100076656E74002054533A0020543A005448B0
:1028200045524D3A00436C65616E696E6720616C7C
:1028300061726D20003D0050696E3A004354524C65
:102840003A20436F6D6D616E6420626C6F636B65DF
:102850006420627920647269766572004354524C38
:102860003A204F4E3A416C7265616479204163743D
:102870006976650A004354524C3A2048414C543A18
:10288000416C726561647920496E61637469766533
:102890000A004354524C3A20584F4E3A2044697330
:1028A00061626C65640A004354524C3A20584F4EA2
:1028B0003A416C7265616479204163746976650A96
:1028C000004354524C3A20584F464620736B69706F
:1028D0007065642E205072657620636D643A004303
:1028E00054524C3A205475726E6564206F666620AF
:1028F00066726F6D3A004354524C3A2052657374BD
:102900006F7265642066726F6D3A004354524C3AA0
:102910002049676E6F7265642C206368616E6E6516
:102920006C20636D643D0020457865633A00435434
:10293000524C3A204163746976653A004354524CD4
:102940003A2048414C543A416C726561647920499F
:102950006E6163746976650A004354524C3A20589C
:102960004F4E3A2044697361626C65640A004354B7
:10297000524C3A20584F4E3A416C7265616479204E
:102980004163746976650A004354524C3A20584FAB
:10299000464620736B69707065642E2050726576B0
:1029A00020636D643A004354524C3A205475726E61
:1029B0006564206F66662066726F6D3A00435452FC
:1029C0004C3A20526573746F7265642066726F6D45
:1029D0003A0044697361726D696E67206E6F74208E
:1029E000617574686F72697A6564004354524C3A39
:1029F00020636F6D6D616E64206A75737420666FFD
:102A00007220004354524C3A204E6F7420656E6F12
:102A1000756768206D656D6F727920666F722067CB
:102A2000726F7570206F7065726174696F6E0049A6
:102A30006E76616C69642061726700496E76616CC4
:102A400069642061726700496E76616C6964206117
:102A50007267004354524C3A20556E6B6E6F776E1E
:102A60002073756666697800536B697070696E676C
:102A7000207363686564756C65642067726F757038
:102A80002065786563004354524C3A206368616E58
:102A90006E656C2066726F7A656E004354524C3AD4
:102AA000206368616E6E656C2066726F7A656E0079
:102AB000536B697070656420686F6D69652073740D
:102AC000756666002000205375623D0020497465DC
:102AD0006D3D004354524C3A2052414D3D00435409
:102AE000524C3A204F75744F664D656D6F72793A4E
:102AF0002000282D292000282B2920002076616C19
:102B00007565206973200020756E6B6E6F776E0A95
:102B1000005D3D005B0020696E76616C6964002099
:102B2000004143544956453A00206F6B003A00205B
:102B30006661696C6564003A005265747279696E09
:102B40006720564354454D5020434D440A0052657A
:102B5000747279696E6720564320434D440A0052CF
:102B600065747279696E67206D6F64627573204356
:102B70004D440A005265747279696E6720434D4472
:102B80000A00206572726F723D004D423A20706FEC
:102B90006C6C696E6720002056616C3A20004D42D3
:102BA0003A20004D423A204E6F7420737570706F5A
:102BB000727465642072656720747970650A004DCF
:102BC000423A20706F6C6C696E672064696D6D6548
:102BD0007220004D423A20496C6C6567616C20613F
:102BE0007267756D656E74730A00206572726F721C
:102BF0003D004D423A20706F6C6C696E6720504901
:102C000020002D004D423A2050492056616C203A58
:102C1000004D423A20706F6C6C696E6720504920FD
:102C2000004D423A20706F6C6C696E6720464D20F3
:102C30006661756C742000206572726F723D004D84
:102C4000423A20706F6C6C696E6720002D004D4217
:102C50003A20464D2056616C203A004D423A207091
:102C60006F6C6C696E6720464D20004354524C2FA8
:102C7000706F6C6C3A204F75744F664D656D6F7256
:102C8000793A2000207365632072656D61696E6911
:102C90006E6700537461747573206465666665724F
:102CA00065640A002D3E005075623A20002D3E00FA
:102CB0005075623A20002D3E005075623A200000A7
:102CC00000000000636D64000073657400007661AD
:102CD0006C000064656C0000485356000052474287
:102CE000000066616E00006D6F6465006374726C55
:102CF000006875650000736174000074656D700094
:102D000072617700002D3E005075623A20002D3E22
:102D1000005075623A200053454E44535441545577
:102D2000533A20556E6B6E6F776E20636D64200A88
:102D300000000000000000000000004F4E000000F6
:102D400000000000004F4646000000000000005256
:102D5000455354000000000000544F47474C4500C5
:102D600000000048414C54000000000000584F4E45
:102D700000000000000000584F4646000000000020
:102D800000494E4352454153450000444543524596
:102D90004153450000454E41424C4500000000446F
:102DA000495341424C45000000554E465245455A54
:102DB000450000465245455A450000000041555423
:102DC0004F00000000000046414E5F4F4E4C59003E
:102DD00000484947480000000000004D454449555F
:102DE0004D000000004C4F5700000000000000485C
:102DF0004541545F434F4F4C00484541540000004B
:102E0000000000434F4F4C000000000000445259A6
:102E100000000000000000524742000000000000D7
:102E2000004853560000000000000052455345542E
:102E30000000000000206661696C65643A004D6F17
:102E400064627573206F7020004D423A206F6B00F2
:102E50003D004D423A205643230020636D643D00FF
:102E60003D004D423A2056435F6865617423004D32
:102E7000423A204E6F7420737570706F727465647F
:102E80002072656720747970650A002056616C3A7B
:102E900030780020543A00205265673A3078004D6F
:102EA000423A20416464723A00444D5800000000E8
:102EB0000000444D58524742570000444D58524775
:102EC0004200000050574D0000000000004D4255E8
:102ED0005344494D0000544845524D4F00000052A4
:102EE000454C41590000000047524F55500000002A
:102EF00000564354454D500000004D425553564333
:102F00000000004143484149455200005350494C9C
:102F100045440000004D4F544F52000000005049FE
:102F2000440000000000004D425553000000000026
:102F300055415254425244470052454C4159505712
:102F40004D00444D5852474257570056454E545332
:102F500000000000454C455641544F5200434F5528
:102F60004E544552000048554D0000000000004DF1
:102F70004552435552590000535052494E4B4C5202
:102F80000000002100240027002A002D003000331B
:102F90000001010000040107010A010000220025D0
:102FA0000028002B002E0031003400020100000533
:102FB0000108010B010505050507050808080802B9
:102FC0000202020A0A0808040404040101010101C2
:102FD0000101010303030303030303040707070CB1
:102FE0000C0C0C0C0C0C0C02020202060606060667
:102FF0000606060B0B0B0B0B0B0B0B010210202014
:10300000080810204010204080020102010804023C
:1030100001010204081020408080402010080402B2
:10302000018004020180402010080402010804020B
:103030000101020408102040800102040810204011
:103040008000000A0B02090C0D0E080703040100A2
:103050000000000000000000000000000000000070
:10306000000000000000000000000000001211102D
:103070000000000000000000000000000000000050
:10308000000000000000004D4255533A20416464A6
:103090002040533A20002F64617461002F736B65E8
:1030A000746368004163636573732D436F6E74725C
:1030B0006F6C2D526571756573742D5072697661F0
:1030C00074652D4E6574776F726B3A2074727565F6
:1030D000004163636573732D436F6E74726F6C2D63
:1030E000416C6C6F772D486561646572733A202A74
:1030F000004163636573732D436F6E74726F6C2D43
:10310000416C6C6F772D4D6574686F64733A205015
:103110004F53542C4745542C4F5054494F4E530055
:103120004163636573732D436F6E74726F6C2D41D1
:103130006C6C6F772D43726564656E7469616C7336
:103140003A2074727565004F5054494F4E530044F5
:10315000454C455445005055540047455400504F88
:10316000535400617574686F72697A6174696F6E27
:103170003A2000417574686F72697A6174696F6E84
:103180003A2000436F6E74656E742D4C656E6774E3
:10319000683A20006F637465742F73747265616D93
:1031A00000696D6167652F6A70656700696D6167A9
:1031B000652F67696600746578742F68746D6C009C
:1031C0006170706C69636174696F6E2F6A736F6E82
:1031D00000746578742F706C61696E00436F6E7453
:1031E000656E742D547970653A2000436F6E6E657C
:1031F0006374696F6E3A20636C6F7365004163633B
:103200006573732D436F6E74726F6C2D416C6C6FB0
:10321000772D4F726967696E3A202A00556E6B6E82
:103220006F776E004E6F74204D6F646966696564D8
:10323000004F4B004D6F766564207065726D616E56
:10324000656E746C7900496E7465726E616C2053A2
:103250006572766572204572726F72005061796C8A
:103260006F616420546F6F204C61726765004E6F10
:103270007420666F756E64005757572D41757468DA
:10328000656E7469636174653A2042617369632095
:103290007265616C6D3D2241636365737320726575
:1032A00073747269637465642200556E6175746825
:1032B0006F72697A6564005061796C6F6164207324
:1032C000697A652077726F6E67004261642072656B
:1032D000717565737400485454502F312E3120009D
:1032E000200057726F6E67207061796C6164004DC9
:1032F0005154543A204354524C2F7478743A204F0E
:1033000075744F664D656D6F72793A2000202D3EC1
:103310002041543A004368616E20747970653A0028
:103320004E6F2073746F7265642076616C7565737F
:10333000202D2064656661756C743A2000536176B7
:10334000656420455441473A005365742045544113
:10335000473A20003157543A204275732072657302
:103360006574206572726F72003157543A2042754D
:103370007320526573657420646F6E650031575415
:103380003A204453323438322070726573656E745B
:103390002C20726573657400493243205265736551
:1033A0007400005EBCE2613FDD83C29C7E20A3FD11
:1033B0001F419DC3217FFCA2401E5F01E3BD3E6013
:1033C00082DC237D9FC1421CFEA0E1BF5D0380DE45
:1033D0003C62BEE0025CDF81633D7C22C09E1D43F7
:1033E000A1FF4618FAA427799BC584DA3866E5BBA5
:1033F0005907DB856739BAE406581947A5FB7826D3
:10340000C49A653BD987045AB8E6A7F91B45C69804
:103410007A24F8A6441A99C7257B3A6486D85B05B6
:10342000E7B98CD2306EEDB3510F4E10F2AC2F7164
:1034300093CD114FADF3702ECC92D38D6F31B2EC92
:103440000E50AFF1134DCE90722C6D33D18F0C52C4
:10345000B0EE326C8ED0530DEFB1F0AE4C1291CF76
:103460002D73CA947628ABF517490856B4EA693724
:10347000D58B5709EBB536688AD495CB2977F4AA52
:103480004816E9B7550B88D6346A2B7597C94A1484
:10349000F6A8742AC896154BA9F7B6E80A54D78936
:1034A0006B353E3E2000496E76616C696420636F27
:1034B0006D6D616E6400000020002300260029006D
:1034C0002C002F0032000001000003010601090159
:1034D0003E3E3E004E6F204D414320636F6E666955
:1034E00067757265643A20736574206669726D77DA
:1034F0006172652773204D41430A00454550524F84
:103500004D207369676E6174757265206F6B004939
:103510006E697469616C697A696E672045455052BD
:103520004F4D2E002072656164206572726F7220AB
:10353000666F7220003E2000203C003157543A0054
:103540003157543A206E6F7420696E697400315798
:10355000543A20425553592074696D656F75740053
:103560003157543A204453323438325F4552524F27
:10357000525F434F4E464947003157543A20312D50
:10358000776972652073686F727465640072656133
:1035900064790024737461746500757074696D6575
:1035A0000066726565686561700024737461747388
:1035B0000020457870697265640A00202D7461727C
:1035C000676574207A6F6E652D0020416C61726DA5
:1035D00020457870697265640A0020636D643A0062
:1035E000204375723A00205365743A002054696D87
:1035F00065723A00204C6F636B733A0052414D3D47
:103600000000CD01BF0211241FBECFEFD1E2DEBF0B
:10361000CDBF00E00CBF1CE0A0E0B2E0ECE8F7EEAC
:1036200002E00BBF02C007900D92AC34B107D9F78E
:1036300024E1ACE4BCE001C01D92A336B207E1F77F
:103640001BE1C2E0DBE100E006C021970109802F09
:10365000FE010F94966BC130D10780E00807A9F7EF
:103660000F947F5A0D94B4730C940000CF93DF93A2
:10367000FC01C681D78180858F70853079F08630D6
:10368000E1F42097D1F0E881F981309719F0808139
:103690008F7B79F40A80DB81C02DF3CF209769F00E
:1036A000CE010E94361B811105C00A80DB81C02D2E
:1036B000F5CF81E0DF91CF91089580E0FBCF84E1E9
:1036C00090E00895DC01ED91FC910484F585E02DF6
:1036D00060E0199581E090E008958FE090E090938C
:1036E000401380933F1388EC90E00895FC0184819F
:1036F00095810895FC01768765870895DC01ED9139
:10370000FC9102A0F3A1E02D199591E0892708957D
:10371000862F089581E08627089521E0FC018485A5
:10372000883008F020E0822F0895FC01848595857B
:103730000895FC0184899589089521E135E0FC0113
:1037400031832083FB014089518962897389FC019F
:1037500042835383648375830895DC01ED91FC916A
:10376000048CF58DE02D199460E778E1811102C099
:1037700062E778E18DE091E10D9477356EEF73E1CA
:103780008DE091E10F947735F0E0E0E0199584EF5A
:1037900091E008958091C90C8823B1F0E091CA0CA2
:1037A000F091CB0C309731F0868197819093C80CC3
:1037B0008093C70C63E571E18DE091E10F9477355B
:1037C0008DE091E10D9478340895CF93DF93EC016F
:1037D0006EE37CE18EEB91E10F947735EA81FB811A
:1037E0000280F381E02D608171818EEB91E10F9475
:1037F00020358EEB91E10F947834E881F9810484CF
:10380000F585E02D60E0CE01199581E090E0DF9133
:10381000CF910895CF93DF936115710589F0EB0186
:10382000DC011296ED91FC9162E0848195810E9409
:1038300062F6BE010E94EAF5DF91CF910D948A04F1
:1038400090E080E0DF91CF9108950D942F620D9468
:103850002F620D942F62CF93DF9300D000D01F9280
:103860001F92CDB7DEB7E7EFF0E1128A118A80E050
:1038700090E19587848784E890E0948B838B81E046
:10388000868780E090E2908B878787E7858B1C8214
:103890001B8285EC92E09A838983FE83ED838FEF10
:1038A0009FEF98878F836EEE7BE18DE091E10F941F
:1038B00077356091520C7091530CCE0101960E94A5
:1038C000FDFC87EF90E10E9440AF6EED7BE18DE063
:1038D00091E10F9477358DE091E10F9478340F9456
:1038E000C31328960FB6F894DEBF0FBECDBFDF918D
:1038F000CF91089560E08DE00D946E0661E08DE05B
:103900000D946E06CF93C1E068EE73E080E090E026
:103910000F94E4086C2F8DE091E10E9474F6CF5F64
:10392000C43191F784EF91E0CF910895892B71F024
:10393000FB01828193810E9412F869E578E18DE0B4
:1039400091E10F94773588EC90E0089590E080E065
:10395000F2CF0F931F93CF93DF93EB0102970CF4F9
:1039600083C00A811B8164E377E1C8010F94AE63D1
:10397000892B51F481E00E94A0FA88EC90E0DF915D
:10398000CF911F910F9108956EE377E1C8010F94D5
:10399000AE63892B11F480E0EECF6AE077E18DE031
:1039A00091E10F9477350E9402FA672F609561705C
:1039B00070E08DE091E10E947BF68DE091E10F9443
:1039C00078348091E9109091EA10892BE9F10A810D
:1039D0001B810E94A3F78823B9F1F8010190002010
:1039E000E9F73197E01BF10BB09770F582E70E9481
:1039F0008EF78091E9109091EA10DC01ED91FC9135
:103A00000088F189E02D60E270E01995B80180919D
:103A1000E9109091EA100F9420358091E91090916F
:103A2000EA10DC01ED91FC910190F081E02D60E065
:103A300019958091E9109091EA10DC01ED91FC91CB
:103A40000488F589E02D19956A817B818DE091E1EB
:103A50000F94203563E077E18DE091E10F947735A5
:103A60008DE091E10F94783480913F139091401351
:103A700002973CF080EF9FEF9093401380933F13A9
:103A80007CCF66EF76E187E191E10F94773587E1AE
:103A900091E10F94783484EF91E071CF892B71F02C
:103AA000FB01828193810E9460F860EE76E18DE0F7
:103AB00091E10F94773588EC90E0089590E080E0F4
:103AC000F2CFEF92FF920F931F93CF93DF93CDB777
:103AD000DEB72C970FB6F894DEBF0FBECDBF8C01BA
:103AE0007B0181E195E09A8389831B821C821D8280
:103AF0001E8298878F8319861A861B861C8605303E
:103B00001105ECF0BE01695F7F4FF701808591855B
:103B10000E94F66D892B99F0CE0107960E9403F959
:103B2000BE01695F7F4FF701868197810E94F66D24
:103B3000892B61F0CE0107960E94ADF90EC0CE012F
:103B400001960E9403F90430110554F7CE01019645
:103B50000E94ADF903301105A4F1BE01695F7F4FEA
:103B6000F701848195810E94F66D892B51F1CE0178
:103B700007960E9458F9BE01695F7F4FF701828165
:103B800093810E94F66D892B19F1CE0107960E9450
:103B9000AEF869EC76E18DE091E10F94773580E045
:103BA0000E9497FA88EC90E02C960FB6F894DEBF4E
:103BB0000FBECDBFDF91CF911F910F91FF90EF907E
:103BC0000895CE0101960E9458F9023011059CF625
:103BD000CE0101960E94AEF801301105D1F6CE015A
:103BE00001960E94AEF860ED76E18DE091E10F94D0
:103BF0007735CFCF0F931F93CF93DF938C01EB01DA
:103C00000297C4F08A819B810F94606380931E02A7
:103C100099270E94AAFA0230110549F08C819D81F2
:103C20000F94606380931D0299270E94B4FAC8EC38
:103C3000D0E002C0C0E9D1E065EB76E18DE091E132
:103C40000F94773560911E028DE091E10E9474F629
:103C500060EA76E18DE091E10F94773560911D0285
:103C60008DE091E10E9474F68DE091E10F9478343B
:103C7000CE01DF91CF911F910F910895CF93DF93E4
:103C8000EB010297ACF164E377E18A819B810F94A9
:103C9000AE63892B29F40E9402FA7D7F0E9447FAC5
:103CA0006EE377E18A819B810F94AE63892B29F4BF
:103CB0000E9402FA72600E9447FA6FE876E18DE096
:103CC00091E10F9477350E9402FA71FB662760F943
:103CD00071E0672770E08DE091E10E947BF68DE056
:103CE00091E10F94783488EC90E0DF91CF910895C2
:103CF0000E942B1CF8CF0F931F93CF93DF93CDB768
:103D0000DEB769970FB6F894DEBF0FBECDBFE09166
:103D10003613F0913713309709F460C08091431344
:103D200090914413892B09F459C08FEF838714862F
:103D300013821482158216821782108611861286CB
:103D40006FE174E18DE091E10F9477358DE091E1C1
:103D50000F947834BE016E5E7F4F80913613909140
:103D600037130F94DA521816CCF5A895AE014F5FB1
:103D70005F4F68E0CE0142960F94D854198ABE0175
:103D80006F5F7F4F80914313909144130E94EAF537
:103D90008C016AE174E18DE091E10F947735BE0109
:103DA0006F5F7F4F8DE091E10F9420350115110574
:103DB00091F0C8010E9403708C01892B59F265E1D2
:103DC00074E18DE091E10F947735B8018DE091E1D8
:103DD0000F942035BBCF60E174E1B4CF88EC90E064
:103DE00069960FB6F894DEBF0FBECDBFDF91CF91BD
:103DF0001F910F910895CF92DF92EF92FF920F9350
:103E00001F93CF93DF9300D000D0CDB7DEB7809162
:103E1000D90C81119AC080913F1390914013029761
:103E20000CF493C08091520C9091530C009709F4BC
:103E30008CC062E375E00E94EAF58C01009709F4FA
:103E400084C00E9434F7E82EF12CE114F10409F447
:103E50007CC070E060E0C8010F94C6556C01EA9424
:103E6000EF2809F481C061E0C8010E9462F6FC01FC
:103E700001851285CE0101960F94AB4ECE010196BD
:103E80000F946E026FE97CE08DE091E10F9477353D
:103E9000B6018DE091E10F94203565E27AE08DE086
:103EA00091E10F942035B8018DE091E10E947BF6FD
:103EB00065E27AE08DE091E10F9420356AE27EE0E0
:103EC0008DE091E10F9420358DE091E10F947834ED
:103ED00062E072E08CED91E10F941A4AD092D21117
:103EE000C092D1111093D4110093D3118AE29EE0B5
:103EF000892BE9F580E395E09093D6118093D51155
:103F00008091C70C9091C80C009741F070E060E080
:103F10000F94C6559093DB0C8093DA0C8091DA0CE9
:103F20009091DB0C009731F19093D8118093D711C9
:103F30001092DA111092D91181E08093D90C66E8C1
:103F40007CE08DE091E10F94773526960FB6F894DA
:103F5000DEBF0FBECDBFDF91CF911F910F91FF90BC
:103F6000EF90DF90CF90089502E012E083CF8AE2D5
:103F70009EE0C2CF80E792E0D7CFCF92DF92EF9260
:103F8000FF920F931F93CF93DF93CDB7DEB7C1544A
:103F9000D1090FB6F894DEBF0FBECDBF6C01AB01E7
:103FA00030E020E060E4CE0101967C010E94916A3D
:103FB000F70101900020E9F731978F010E191F09D1
:103FC000A801B701C6010F941770892B11F010E0FA
:103FD00000E0C801CF5BDF4F0FB6F894DEBF0FBE25
:103FE000CDBFDF91CF911F910F91FF90EF90DF90A8
:103FF000CF900895EF92FF920F931F93CF93DF938B
:10400000EC01892B51F188858F70843009F5E984A2
:10401000FA84C7010E9403B38C0118161906ECF448
:10402000C7010F94F63BC801012E000CAA0BBB0B75
:1040300089879A87AB87BC878885807F82608887DD
:10404000C801DF91CF911F910F91FF90EF900895DC
:10405000823019F409851A85F3CF10E000E0F0CF23
:104060000F931F93CF93DF938C01D0E0C0E0011535
:104070001105B1F0BE016E59734EC8010F94CC63A7
:10408000892B51F4FE01EA59F34E849190E0DF91BF
:10409000CF911F910F9108952596C233D10539F71D
:1040A00081E090E0F4CF0895EF92FF921F93CF93B9
:1040B000DF93192F7B01C82FD92FD7FF03C0D195CC
:1040C000C195D10961E08C2F0F949C0682E0E8161F
:1040D000F10499F460E08C2F0F946E0666ED7BE19D
:1040E0008EEB91E10F9477358EEB91E1DF91CF91DB
:1040F0001F91FF90EF900D947834612FEF2851F4C9
:104100006095661F6627661F8C2F0F946E0662ED02
:104110007BE1E6CF661F6627661F8C2F0F946E0625
:104120006DEC7BE1DDCFBF92CF92DF92EF92FF92F9
:104130000F931F93CF93DF93CDB7DEB72E970FB6B4
:10414000F894DEBF0FBECDBF20913D1330913E13DA
:10415000232B09F4A6C020913C132111A2C07C019D
:1041600080913C138F5F80933C1380913B138F5F52
:1041700080933B130F9417090091D10C1091D20C2E
:104180002091D30C3091D40C601B710B820B930BDC
:104190006B3071058105910508F479C083E0E8165C
:1041A000F104A9F00F9417090091CD0C1091CE0CD9
:1041B0002091CF0C3091D00C601B710B820B930BB4
:1041C000BB24B394643671058105910508F4B12CC4
:1041D000E0913D13F0913E13068117810115110501
:1041E000C1F1F80180858F70863079F519870887CD
:1041F00070E060E0CE0108960E94A7E0B701CE0112
:1042000008960E94D8E369E375E0C8010E94EAF5C8
:10421000FC01892BD1F090859F7095509230A8F4C5
:10422000C680D780C114D10481F0DA82C982B80176
:10423000CE0101960E94A7E0B701CE0101960E942F
:10424000D8E3F601C280D380EDCFF801028113815B
:10425000C5CFF3E0EF16F10451F00F941709609306
:10426000D10C7093D20C8093D30C9093D40CBB20C0
:1042700051F00F9417096093CD0C7093CE0C80937E
:10428000CF0C9093D00C10922D1210922E12809180
:104290003B13815080933B1380913C13815080935A
:1042A0003C132E960FB6F894DEBF0FBECDBFDF9144
:1042B000CF911F910F91FF90EF90DF90CF90BF9023
:1042C0000895A89582E090E00C94932080913A1391
:1042D0008F5F80933A13A89583E090E00E9493202B
:1042E0000F94B03B80913A13815080933A13089514
:1042F0006BEA7BE18DE091E10F94773568E97BE132
:104300008DE091E10F9477356AE87BE18DE091E1F2
:104310000F94773562E87BE18DE091E10F9477357A
:104320008DE091E10F94783462E77BE18DE091E1DB
:104330000F94773566E67BE18DE091E10F94773558
:1043400069E57BE18DE091E10F94773564E47BE1F1
:104350008DE091E10F94773565E37BE18DE091E1AC
:104360000F9477356DE27BE18DE091E10F94773525
:104370006CE17BE18DE091E10F94773566EF7AE1B6
:104380008DE091E10F94773569EE7AE18DE091E16E
:104390000F9477356FED7AE18DE091E10F947735E9
:1043A00060ED7AE18DE091E10F94773568EC7AE188
:1043B0008DE091E10F9477356CEB7AE18DE091E13E
:1043C0000F94773562EA7AE18DE091E10F947735C9
:1043D00063E87AE18DE091E10F9477356EE67AE15A
:1043E0008DE091E10F94773561E67AE18DE091E11E
:1043F0000F94773563E57AE18DE091E10F9477359D
:1044000067E47AE18DE091E10F9477356FE37AE12B
:104410008DE091E10F94773564E37AE18DE091E1ED
:104420000F94773567E27AE18DE091E10F9477356B
:104430006FE17AE18DE091E10F94773564E17AE103
:104440008DE091E10F94773565E07AE18DE091E1BF
:104450000F9477356CEF79E18DE091E10F9477352A
:104460006EEE79E18DE091E10F94773560EE79E1C0
:104470008DE091E10F94773564ED79E18DE091E184
:104480000F94773566EC79E18DE091E10F94773503
:104490006EEB79E18DE091E10F9477356BEA79E18C
:1044A0008DE091E10F94773561EA79E18DE091E15A
:1044B0000F9477358DE091E10D9478340F931F932D
:1044C000CF93DF9300D000D0CDB7DEB70E94782124
:1044D0006AE671E18DE091E10F947735CE010196A6
:1044E0000F94AB4ECE0101960E94A06D01E115E044
:1044F0001A8309838091000F9091010FA091020F00
:10450000B091030F8B839C83AD83BE83CE01019654
:104510000E94A06D1A8309831B821C821D821E8249
:1045200080E591E00F946B0244E050E0BE016D5FC6
:104530007F4F81E090E00F94903E0F949E41CE011A
:1045400001960E94A06D1A8309831B821C821D8222
:104550001E8280E591E00F946B0244E050E0BE01C2
:104560006D5F7F4F85E090E00F94903E0F949E41E9
:10457000CE0101960E94A06D60E971E18DE091E1AC
:104580000F94773588EC90E026960FB6F894DEBF4E
:104590000FBECDBFDF91CF911F910F910895CF92A4
:1045A000DF92EF92FF921F93CF93DF9300D000D062
:1045B000CDB7DEB761E87CE08DE091E10F9477350F
:1045C00081EFE82E80E1F82E10E090E1C92ED12C89
:1045D000F70181917F01803130F46DE375E08DE06A
:1045E00091E10F942035153041F1F7013197808129
:1045F00090E0B0E0A0E089839A83AB83BC83DE8245
:10460000CD82BE016F5F7F4F8DE091E10E94AFBE12
:104610006FE77CE00F9477351F5F1630C9F626965A
:104620000FB6F894DEBF0FBECDBFDF91CF911F91C3
:10463000FF90EF90DF90CF9008958091F61090E07A
:10464000B0E0A0E089839A83AB83BC83DE82CD8215
:10465000BE016F5F7F4F8DE091E10E94AFBE0F946E
:104660007834DACFEF92FF920F931F93CF93DF93BB
:1046700000D000D01F92CDB7DEB77B01CE010796E8
:104680009F938F9301979F938F9301979F938F93FE
:1046900001979F938F9301979F938F9301979F9378
:1046A0008F938E010F5F1F4F1F930F938FE395E042
:1046B0009F938F93DB0113968C9113978F93129690
:1046C0008C918F930F94AC700FB6F894DEBF0FBE31
:1046D000CDBF0697ECF46EE278E187E191E10F94AB
:1046E0007735D70112966D917C9187E191E10F9416
:1046F000203580E991E027960FB6F894DEBF0FBE13
:10470000CDBFDF91CF911F910F91FF90EF90089552
:104710008091E9109091EA10892BA9F10E94A3F7EA
:10472000882389F182E70E948EF78091E9109091A9
:10473000EA10DC01ED91FC910088F189E02D64E044
:1047400070E019958091E9109091EA10DC01ED91EB
:10475000FC910280F381E02D46E050E0B80119950C
:1047600086E0F801A1EFB0E101900D928A95E1F7A2
:104770008091E9109091EA10DC01ED91FC910488A0
:10478000F589E02D19950E94CF2260E478E18DE053
:1047900091E10F94773588EC90E0ADCF08952F929A
:1047A0003F924F925F926F927F928F929F92AF92C1
:1047B000BF92CF92DF92EF92FF920F93CF93DF934E
:1047C00000D01F92CDB7DEB77C017A8369835C830A
:1047D0004B836901DB011C92FC0160818FEF860F26
:1047E000893108F04FC034FF4DC0FAE06F9FB0012F
:1047F00011246B51764FCD010F940364D7011196AC
:104800008C918F7051F0D5FE08C04B815C8160EABD
:1048100075E089819A810F940770E981FA8101908E
:104820000020E9F7319729813A81E21BF30B190146
:104830002E0E3F1E4B815C814E1B5F0B4150510978
:104840005C834B83D7011196EC911197EF7009F4BB
:10485000F7C0D5FEF5C0E150EC3008F0F1C0F0E053
:104860008827EA5CFB4D8F4F0D94966B4524E82416
:104870005525B425CF2593246525652565258124F7
:104880006924EB2529803A80DDCFF7018481282F28
:1048900030E050E040E0002359F030E0A4E6B0E022
:1048A0000F945F6B2FEF30E040E050E00F942D6BE2
:1048B0005F934F933F932F9383E595E09F938F935F
:1048C000FC81FF932B812F933F922F920F943F7087
:1048D000B2C017968C9117978F9316968C91169756
:1048E0008F9315968C9115978F9314968C918F9327
:1048F00086E595E09F938F93BC81BF93EB81EF9307
:10490000E3CF17968C9117978F9316968C911697E5
:104910008F9315968C9115978F9314968C918F93F6
:104920008AE595E0E7CF1496CD90DD90ED90FC9070
:104930001797F7FE34C084E6882E912CA12CB12C59
:10494000C701B601A50194010F942D6B9B01AC0129
:1049500088279927DC01821B930BA40BB50BBF930F
:10496000AF939F938F9366277727CB016C197D09AF
:104970008E099F09A50194010F942D6B5F934F93AE
:104980003F932F938EE595E09F938F933C813F93C8
:104990004B814F933F922F920F943F704CC0C701B1
:1049A000B60124E630E040E050E00F942D6B9F9379
:1049B0008F937F936F935F934F933F932F938FE5E5
:1049C00095E09F938F939C819F93AB81AF93E2CFB0
:1049D000C7010E948AB2BC01D7011696CC901697E7
:1049E0001796DC901797D0FADD24D0F814969C9196
:1049F00014971596FC90EB80BC80292F30E050E096
:104A000040E077FD35C0011135C07F936F931F9251
:104A10001F921F929F931F92FF92DF92CF9288E680
:104A200095E09F938F93FC81FF932B812F933F926F
:104A30002F920F943F700FB6F894DEBF0FBECDBF1C
:104A400089819A810F900F900F900F90DF91CF91F5
:104A50000F91FF90EF90DF90CF90BF90AF909F901D
:104A60008F907F906F905F904F903F902F90089520
:104A7000002361F0292F30E0A4E6B0E00F945F6BD3
:104A80002FEF30E040E050E00F942D6B5F934F9399
:104A90003F932F931F92FF92DF92CF928BE695E088
:104AA0009F938F93BF92EF9275CF15968C91159728
:104AB0001F928F9316969C91169717968C918170E2
:104AC0008F939F938EE695E015CF14968D909D90D1
:104AD000AD90BC90179720E030E0A901C501B4016A
:104AE0000F94C1692401350187FF04C077FA7094DF
:104AF00077F87094C301B2010F94936C6B01072E89
:104B0000000C880B990B0F94C8699B01AC01C30181
:104B1000B2010F94B46B20E030E04AE754E40F9404
:104B2000276A0F941E6D0F94936C062F772E20E04A
:104B300030E0A901C501B4010F94C16987FF07C026
:104B40007F920F93DF92CF9284E795E0D3CE7F924E
:104B50000F93DF92CF9285E795E09F938F933C81EF
:104B60003F934B814F93B0CE14968C9114971F9224
:104B70008F9315968C9115971F928F9316968C9103
:104B80001F928F938BE695E09F938F93BC81BF9389
:104B9000EB81EF933F922F920F943F704CCF17967B
:104BA0008C9117971F928F9314968C9114971F9244
:104BB0008F9315968C9115971F928F9316968C91C3
:104BC0001F928F9388E695E09F938F93BC81BF934C
:104BD000EB81EF93DFCE14966D917C914B815C81DC
:104BE000C1010F9425702CCFEF92FF920F93CF93BA
:104BF000DF93CDB7DEB7A0970FB6F894DEBF0FBE38
:104C0000CDBF7C0100E020E030E340E250E0BE0197
:104C10006F5F7F4F0E94CF23BE016F5F7F4F8EEB90
:104C200091E10F94203560EF7AE08EEB91E10F94E3
:104C30007735F70161816F708EEB91E10E9474F618
:104C400069EE7AE08EEB91E10F947735F70162819E
:104C50008EEB91E10E9474F68EEB91E10F94783423
:104C6000A0960FB6F894DEBF0FBECDBFDF91CF91F7
:104C70000F91FF90EF900895CF92DF92FF920F93E4
:104C80001F93CF93DF93F12C6115710509F48FC049
:104C90006A01EB018C01CB010E9469B3F82E8823D5
:104CA00009F485C0D6FE0EC0D8018C918B3009F472
:104CB00052C008F043C040E051E060E070E08A304C
:104CC00009F452C0D4FE0BC0F80160816A3020F0B4
:104CD0006E3028F0693119F0CE010E947CBCD5FEFF
:104CE00066C0D80114964D915D916D917C91179796
:104CF00011968C918F70873030F08930C8F18A50CE
:104D0000823008F45DC0CE010E94ECB4EE81FF81D8
:104D1000309709F44CC080858F709EEF980F9230C9
:104D200010F0811144C0D80111968C91982F929562
:104D3000907F80858F70892B808739C08C3081F07F
:104D400040E056E060E070E08D3009F0BBCFCE016E
:104D50000E942FB6B7CF40E051E060E070E0F7CF9F
:104D600040E056E060E070E0CE010E9406B6AACFB7
:104D7000EE81FF813097D9F080858F709EEF980F7C
:104D8000923010F0811113C0418752876387748776
:104D9000EE81FF818085807F83608087EE81FF8147
:104DA0008085982F907F8F708067903629F28F2DA5
:104DB000DF91CF911F910F91FF90DF90CF900895D9
:104DC000CE010E94ECB4F3CFCF93DF9300D000D09C
:104DD0001F921F92CDB7DEB7FC01628398E0DE011F
:104DE000119601900D929A95E1F729813A814B81B4
:104DF0005C816D817E818F81988528960FB6F894AD
:104E0000DEBF0FBECDBFDF91CF910895CF93DF936B
:104E100000D000D01F921F92CDB7DEB7FC01608397
:104E200098E0DE01119601900D929A95E1F72981A3
:104E30003A814B815C816D817E818F819885289636
:104E40000FB6F894DEBF0FBECDBFDF91CF910895AE
:104E5000CF93DF9300D000D01F921F92CDB7DEB763
:104E6000FC019181907F9A6091834483558366838E
:104E7000778388E0DE01119601900D928A95E1F723
:104E800029813A814B815C816D817E818F819885FA
:104E900028960FB6F894DEBF0FBECDBFDF91CF913D
:104EA0000895AF92BF92CF92DF92EF92FF920F934D
:104EB0001F93CF93DF9300D000D01F921F92CDB7E6
:104EC000DEB76115710509F45FC05A016B017C0101
:104ED000CB010E9469B3082F882369F1D601169689
:104EE0008D919C91009709F443C0FC011085212FFE
:104EF0002F703EEF320F323010F021112EC012957C
:104F00001F70B4FE59C0C6010E949BBCF70180838C
:104F1000112381F18181807F182B1183D601169690
:104F2000ED91FC9181859285A385B485F7018483F9
:104F30009583A683B783802F28960FB6F894DEBF9B
:104F40000FBECDBFDF91CF911F910F91FF90EF90DA
:104F5000DF90CF90BF90AF900895253049F460E086
:104F60000E9462F6009721F0DC0118961C91C7CFD1
:104F700010E0C7CFD6011696ED91FC9180858F7019
:104F8000823021F0833051F000E0D5CF4185528549
:104F900063857485C7010E942827CDCF418552853E
:104FA00063857485F7018181807F87608183448375
:104FB000558366837783BFCF1123E1F2F701AACF30
:104FC000CF93DF9300D000D01F921F92CDB7DEB7F2
:104FD000FC016F3F710519F014F06FEF70E077FD81
:104FE00060E09181892F8F7081508230C8F4648392
:104FF00088E0DE01119601900D928A95E1F72981F2
:105000003A814B815C816D817E818F819885289664
:105010000FB6F894DEBF0FBECDBFDF91CF910895DC
:10502000907F91609183E3CFCF92DF92EF92FF92D6
:10503000DC01362F1196EC911197EF70EC3008F0EF
:10504000B6C0F0E08827E85DF74D8F4F0D94966B62
:10505000DA2860286028D728D728D728A5286728E5
:10506000D728D7283428342814968D919D910D90F7
:10507000BC91A02D662399F0B7FD9FC08F3F91058D
:10508000A105B10529F024F08FEF90E0A0E0B0E099
:105090002FEF30E0A901481B590BCA010CC0B7FD26
:1050A00089C08F3F9105A105B10529F024F08FEF4C
:1050B00090E0A0E0B0E0FF90EF90DF90CF900895F7
:1050C00014962C91822F90E06623A9F3E1CF1496D9
:1050D000CD90DD90ED90FC901797662301F120E0D4
:1050E00030E0A901C701B6010F94C16987FD65C011
:1050F00020E030E04FE753E4C701B6010F94C96CDC
:1051000018160CF457C0A701960160E070E08FE715
:1051100093E40F94B46B0F94936CCB01CCCF20E04D
:1051200030E0A901C701B6010F94C16987FD42C0F3
:1051300020E030E04FE753E4C701B6010F94C96C9B
:105140001816DCF1C701B601E6CF14966D917D917A
:105150008D919C9117973323B1F06D395FEF7507EF
:105160008507950754F1611524E6720781059105BD
:105170000CF52CE93FEF4FEF5FEF0F942D6BC9015A
:1051800081509F4F98CF6D394FEF74078407940774
:105190008CF0611554E675078105910574F424E6D9
:1051A00030E040E050E00F942D6BC90184CF8FEFC9
:1051B0009FEF81CF90E080E07ECF8FEF90E07BCFBC
:1051C000CF92EF92FF920F931F93CF93DF9300D074
:1051D00000D01F921F92CDB7DEB77C0109831A83DE
:1051E0002B833C834D835E836F83788765E27CE10C
:1051F0008EEB91E10F947735CE0101960E94F42554
:10520000898181112CC00B81013089F128F010E0D7
:105210000230F1F5CC2001F160E0CE0101960E9450
:105220001428F70102811381892B81F0C8010E94A3
:10523000D0B4672B682B692B79F44FEF5FEFBA017D
:1052400080E00F945256AB01BC0103C040E050E037
:10525000BA01C8010E948FB481E090E02AC0803179
:10526000B0F58E30B8F58130A9F18230B9F168E13E
:105270007CE18EEB91E10F94773569818EEB91E1C2
:105280000E9474F68EEB91E10F94783401E010E007
:1052900068E07CE18EEB91E10F947735B8018EEBFD
:1052A00091E10E947BF68EEB91E10F94783490E0CF
:1052B00080E028960FB6F894DEBF0FBECDBFDF9119
:1052C000CF911F910F91FF90EF90CF900895835150
:1052D000843068F6F70102811381A8CF40E050E0E6
:1052E000BA01F70182819381B5CFDC011196EC916F
:1052F0001197EF70E150EB3008F039C0F0E08827EB
:10530000EB57F64D8F4F0D94966BA829A829B72916
:10531000902990299929B029B029B029902990295C
:1053200014966D917D918D919C9117970F94C869FA
:10533000089514966D917D918D919C91179724E617
:1053400030E040E050E00F942D6BCA01B901EECF80
:1053500014966C9170E090E080E00F94C669089517
:1053600014966D917D918D919C911797089560E0B1
:1053700070E0CB010895DC011196EC911197EF706C
:10538000E150EB3008F037C0F0E08827E553F64DE8
:105390008F4F0D94966BDD29DD29FB29D629D6295F
:1053A000EC29E329E329E329D629D62914966D911E
:1053B0007D918D919C911797089514966C9170E052
:1053C00090E080E0089514966D917D918D919C916F
:1053D00017970F94936C089514966D917D918D910C
:1053E0009C91179724E630E040E050E00F942D6B3D
:1053F000CA01B901089560E070E0CB0108952F92D1
:105400003F924F925F926F927F928F929F92AF9254
:10541000BF92CF92DF92EF92FF920F931F93CF93A1
:10542000DF93CDB7DEB7A2970FB6F894DEBF0FBEFD
:10543000CDBF6115710549F528E0FC01DE0111962B
:1054400001900D922A95E1F729813A814B815C8187
:105450006D817E818F819885A2960FB6F894DEBF0C
:105460000FBECDBFDF91CF911F910F91FF90EF90B5
:10547000DF90CF90BF90AF909F908F907F906F9074
:105480005F904F903F902F9008956B018C016BEDD2
:1054900077E0C6010E94EAF5FC01892B09F413C1EB
:1054A00080858F70843009F457C0853009F00BC1B6
:1054B000E680F780E114F10409F405C1D7011896DC
:1054C0008C9118978F70823019F41296ED90FC90A1
:1054D000E114F10409F4F7C0F70180858F7085307D
:1054E00011F0D701F2CFC7010E9434F78230C9F71B
:1054F00060E0C7010E9462F65C010E94FA1F61E051
:10550000C7010E9462F64C01FC0180858F708230D9
:1055100041F7C8010E94BB29D40119964D905D90B6
:105520006D907C901C976415750586059705C9F6E6
:10553000A114B10409F4C7C019821A821B821C820B
:105540001D821E821F8218868A81807F8A83F501D0
:105550006185CE0101964EC063E979E0818592852F
:105560000F94F76F892B09F0AEC0C8010E94BB29C8
:10557000611571058105910509F48BC0660F771FD0
:10558000881F991F2FEF30E040E050E00F942D6B03
:1055900057FD15C023303105410551050CF05FC0A2
:1055A000DA01C9010196A11DB11D82309105A10545
:1055B000B105D9F10397A105B10509F450C01982CD
:1055C0001A821B821C821D821E821F8218868A817B
:1055D000807F8A8367E0CE0101960E94E4262987B6
:1055E0003A874B875C876D877E878F87988B62E1D0
:1055F000CE0109960E940627298B3A8B4B8B5C8B38
:105600006D8B7E8B8F8B988F49895A896B897C89AA
:105610008D899E89AF89B88D49835A836B837C833A
:105620008D839E83AF83B8870FCF19821A821B8226
:105630001C821D821E821F8218868A81807F8A8337
:1056400067E0CE0101960E94E42629873A874B87BE
:105650005C876D877E878F87988B61E1C9CF1982C0
:105660001A821B821C821D821E821F8218868A81DA
:10567000807F8A8367E0CE0101960E94E426298715
:105680003A874B875C876D877E878F87988B60E131
:10569000AFCF19821A821B821C821D821E821F823A
:1056A00018868A81807F8A8367E0CE0101960E94F6
:1056B000E42629873A874B875C876D877E878F87AB
:1056C000988B62E095CF6DE775E0C6010E94EAF520
:1056D0007C01009709F4F6C0DC0118968C918F705C
:1056E000853009F0ECC0C7010E9434F7843008F41B
:1056F000E9C060E0C7010E9462F65C0161E0C70199
:105700000E9462F63C0162E0C7010E9462F6DC0181
:1057100019962D913D914D915C911C97298F3A8F4F
:105720004B8F5C8F63E0C7010E9462F64C0165E01D
:10573000C7010E9462F66C0167E0C7010E9462F631
:105740007C01C8010E94BB29298D3A8D4B8D5C8D4F
:10575000621773078407950794F4D601CD28E9F4FE
:1057600019821A821B821C828A81807F8A834981E6
:105770005A816B817C8180E090E0DC014DCFF401A7
:1057800021843284438454842616370648065906F9
:1057900004F5E114F10421F3D70118968C911897C0
:1057A0008F708230E9F619821A821B821C821D8258
:1057B0001E821F8218868A81807F8A8319964D9166
:1057C0005D916D917C911C97CE0101960E942827D6
:1057D00013CFF5010184F285E02DFE8FED8FD3010B
:1057E00019966D907C9019821A821B821C821D82F0
:1057F0001E821F8218868A81807F8A839301072CEC
:10580000000C440B550B2F8F38A349A35AA36F01EB
:10581000FF0FEE08FF08498D5A8D4A01550FAA085F
:10582000BB08C8010E94BB299B01AC01281939099A
:105830004A095B096F8D78A189A19AA16C197D092C
:105840008E099F090F94FB6A9101032C000C440BF5
:10585000550B281939094A095B090F942D6BC20EA3
:10586000D31EE41EF51EC301AD8DBE8D8A1B9B0B9E
:10587000B101E98DFA8D6E1B7F0B0F94826B77FF60
:1058800002C06F5F7F4F75956795CB01770FAA0BAD
:10589000BB0B8C0D9D1DAE1DBF1D40E050E0BA013D
:1058A000B7FD92CF4F8D58A169A17AA184179507B2
:1058B000A607B7070CF088CFAC01BD0185CF8823C0
:1058C00009F44ECFD8014D915D916D917C91139764
:1058D00014968D919D910D90BC91A02D9DCE2F92EF
:1058E0003F924F925F926F927F928F929F92AF9270
:1058F000BF92CF92DF92EF92FF920F931F93CF93BD
:10590000DF93CDB7DEB765970FB6F894DEBF0FBE55
:10591000CDBF6115710549F528E0FC01DE01119646
:1059200001900D922A95E1F729813A814B815C81A2
:105930006D817E818F81988565960FB6F894DEBF64
:105940000FBECDBFDF91CF911F910F91FF90EF90D0
:10595000DF90CF90BF90AF909F908F907F906F908F
:105960005F904F903F902F9008953B018C016BED1D
:1059700077E0C3010E94EAF56C01D801FC90FF209A
:1059800009F45AC0009709F457C0FC0180858F7054
:10599000843009F4DEC0853009F04EC080911E02CB
:1059A000893020F480911D02893050F061E875E063
:1059B0008EEB91E10F9420358EEB91E10F947834CA
:1059C000D6011696ED90FC90E114F104A9F1F701CF
:1059D00080858F705701823069F0B12CA12CE114C1
:1059E000F10409F436C1D70118968C918F70853077
:1059F00021F0F701E280F380F2CFC7010E9434F773
:105A00008230B9F760E0C7010E9462F60E94FA1F77
:105A10004C0161E0C7010E9462F66C01D8018C91D3
:105A20008815190431F7F60180858F70823009F7E7
:105A3000C114D10409F017C16DE775E0C3010E94DC
:105A4000EAF57C01D80111968C918F7009F43BC165
:105A5000E114F10409F43BC1F70180858F708530B2
:105A600009F0D0C1C7010E9434F7843008F4CAC1DC
:105A700064E0C7010E9462F66C0166E0C7010E9403
:105A800062F61C01C8010E94BB294B015C0160E069
:105A9000C7010E9462F6DC0119964D905D906D90F1
:105AA0007C901C97B0911E02B98B84149504A604B7
:105AB000B7040CF016C1B93020F480911D02893072
:105AC00050F165EC79E08EEB91E10F947735C801E8
:105AD0000E94BB29AB01BC012AE030E08EEB91E1D2
:105AE0000F949A346FEA79E08EEB91E10F94773559
:105AF00060E0C7010E9462F6FC0141855285638522
:105B000074852AE030E08EEB91E10F949A348EEBAD
:105B100091E10F947834C114D10409F479C1D6010C
:105B200018968C9118978F70823009F071C1198284
:105B30001A821B821C821D821E821F8218868A8105
:105B4000807F8A8319964D915D916D917C911C9710
:105B500043C063E979E0818592850F94F76F892BC3
:105B600009F06ACFB0E1FB1609F463C0BF1580F0FD
:105B7000E2E0FE1619F1D8014D915D916D917C9195
:105B8000139714968D919D910D90BC91A02D38C0C6
:105B9000F1E1FF16F1F122E1F212EDCF19821A8242
:105BA0001B821C821D821E821F8218868A81807F32
:105BB0008A8344E150E060E070E00EC019821A82EE
:105BC0001B821C821D821E821F8218868A81807F12
:105BD0008A8340E050E0BA01CE0101960E94282756
:105BE00029873A874B875C876D877E878F87988B5D
:105BF00049855A856B857C858D859E85AF85B8895D
:105C000049835A836B837C838D839E83AF83B8875C
:105C10008BCE19821A821B821C821D821E821F82D9
:105C200018868A81807F8A8340E850E060E070E0D7
:105C3000D3CF19821A821B821C821D821E821F8270
:105C400018868A81807F8A834FEF50E060E070E0A1
:105C5000C3CFA114B10409F4EFCEF50180858F7094
:105C600009F4EACE650180911E02893020F480910A
:105C70001D028930B8F061ED79E08EEB91E10F946F
:105C80007735D60119964D915D916D917C911C9758
:105C90002AE030E08EEB91E10F949A348EEB91E1A3
:105CA0000F94783419821A821B821C821D821E82F4
:105CB0001F8218868A81807F8A83F60141855285FA
:105CC0006385748589CFE114F10409F09BC0F80164
:105CD000408151816281738184819581A681B781E0
:105CE0008FCF61E0C7010E9462F6DC0119962D9109
:105CF0003D914D915C911C972A8B3B8B4C8B5D8B1E
:105D0000281539054A055B053CF5B989B93020F4F9
:105D100080911D02893050F061E979E08EEB91E1CC
:105D20000F9477358EEB91E10F9478342114310480
:105D300009F46EC0F10180858F70823009F068C06F
:105D400019821A821B821C821D821E821F82188663
:105D50008A81807F8A83B2CF63E0C7010E9462F6A6
:105D60008C0162E0C7010E9462F6DC011996CD90B9
:105D7000DD90ED90FC901C97F801218532854385DC
:105D800054852C193D094E095F09C501B4016419F8
:105D90007509860997090F94FB6A2A893B894C8902
:105DA0005D8924193509460957090F942D6BC20ED8
:105DB000D31EE41EF51EF989F93020F480911D02EE
:105DC000893090F06CE779E08EEB91E10F947735B4
:105DD0002AE030E0B701A6018EEB91E10F949A34EE
:105DE0008EEB91E10F94783419821A821B821C8207
:105DF0001D821E821F8218868A81807F8A83B70156
:105E0000A601EACED70118968C918F7009F05FCF6A
:105E100019821A821B821C828A81807F8A8349812F
:105E20005A816B817C8180E090E0DC01E9CEDC016D
:105E30001196EC911197EF70E150EB3008F03EC0F5
:105E4000F0E08827E95DF04D8F4F0D94966B3D2F64
:105E50003D2F5E2F322F322F572F482F482F482F9C
:105E6000322F322F14962D913D914D915C911797C1
:105E7000A4E6B0E00F944C6B089514966C9184E600
:105E8000689FB0011124072E000C880B990B089510
:105E900020E030E048EC52E414966D917D918D91B4
:105EA0009C9117970F94276A0F94936C08951496FA
:105EB0006D917D918D919C911797089560E070E0B0
:105EC000CB0108958F929F92AF92BF92CF92DF92B3
:105ED000EF92FF920F931F93CF93DF9300D000D0E8
:105EE0001F921F92CDB7DEB76D7F6130710509F447
:105EF000B7C0FC01E280F380E114F10409F4B0C002
:105F00008C01C7010E94D0B44B015C0161E070E0DC
:105F1000C7010E9416B581149104A104B10409F4CB
:105F20009FC020E030E04AE754E40F94276A0F94C2
:105F30009A6C6B017C01C114D104E104F10409F4F1
:105F40008FC00F941709681979098A099B096C1584
:105F50007D058E059F0508F483C0F801A280B380FB
:105F600070E060E0C5010E9416B520E030E048EC2A
:105F700052E40F94276A0F949A6C6B017C014FEFE7
:105F80005FEFBA0180E00F945256AB01BC01C5012E
:105F90000E948FB419821A821B821C821D821E826B
:105FA0001F8218868A81807F8A83F80162817381CB
:105FB00040E050E3CE0101960E945127CE010196A8
:105FC0000E94172F4B015C016FE875E08EEB91E1A9
:105FD0000F942035B501A4018EEB91E10E9471F67A
:105FE0006EE975E08EEB91E10F942035B701A601C3
:105FF0008EEB91E10E9471F68EEB91E10F94783473
:10600000C80CD91CEA1CFB1C8A81807F86608A83AD
:10601000CD82DE82EF82F886F8016281738140E0F2
:1060200050E2CE0101960E943C2662EA75E08EEBBA
:1060300091E10F942035B701A6018EEB91E10E940A
:1060400071F68EEB91E10F94783430E020E040E07F
:1060500050E260E070E0F801828193810E94E8B92B
:1060600090E080E028960FB6F894DEBF0FBECDBF5B
:10607000DF91CF911F910F91FF90EF90DF90CF9024
:10608000BF90AF909F908F9008952F923F924F9224
:106090005F926F927F928F929F92AF92BF92CF92B8
:1060A000DF92EF92FF920F931F93CF93DF93CDB7C1
:1060B000DEB768970FB6F894DEBF0FBECDBF6C0198
:1060C00009871A872B873C874D875E876F87788B78
:1060D00022E1E216F10480F5F701EC5EFC4F30811D
:1060E000398BCE0109960E948AB297FD04C0BC018B
:1060F000C6010E94ABB28B85D60112968C93129783
:1061000089858C931196EC911197EF70EC3008F023
:106110006CC0F0E08827E057FF4C8F4F0D94966BD2
:10612000EB31B930B93032329E30AE32FE313C32D2
:106130003C323C32FE31FE31198AD3CFF12C9A85A4
:106140009F709D3008F0A7C4E92FF0E08827E45540
:10615000FF4C8F4F0D94966BF530E6320633E632E6
:10616000B132B132E632E6324B354B35E632E63209
:10617000BD319A859F709D3008F00FC1E92FF0E086
:106180008827EA53FF4C8F4F0D94966BF5309B3167
:106190008E31EB30D630D33072319D31CD31CD31AF
:1061A0005C315C31BD318889F60187838F85D601EA
:1061B00016968C9316978E8515968C9315978D85CC
:1061C00014968C93149711968C911197807F892B3C
:1061D00011968C930AC08F859889F60186838781F2
:1061E00090FB80F987838E858583B989BB2309F469
:1061F00060C0F60181818F702B2F30E0821713066B
:1062000009F457C06AEE78E08EEB91E10F94773590
:10621000D60111966C916F708EEB91E10E9474F62D
:1062200067EE78E08EEB91E10F94773569898EEB1C
:1062300091E10E9474F665EE78E08EEB91E10F94A7
:106240007735F601008119821A821B821C821D8219
:106250001E821F82188689898F709A81907F892B70
:106260008A830983EE24EA94FE2C118122813381F2
:106270004481558166817781CE0101960E94453027
:10628000D6012C9311963C93119712964C9312972A
:1062900013965C93139714966C93149715967C93AE
:1062A000159716968C93169717969C93C6010E9485
:1062B000F42588E0F60163C18D859E85AF85B88998
:1062C000B7FD0EC08F3F9105A105B10529F024F05F
:1062D0008FEF90E0A0E0B0E0D60114968C9385CFCC
:1062E00080E0FACF6D857E858F85988920E06D39B5
:1062F000BFEF7B078B079B076CF02FEF6115E4E680
:106300007E078105910534F424E630E040E050E05A
:106310000F942D6BD60114962C9367CF8F85988997
:10632000F6018683878190FB80F987838E8585833C
:106330008D8584835ACF8D85CFCF8D849E84AF8405
:10634000B88820E030E0A901C501B4010F94C1690B
:1063500060E087FD0FC020E030E04FE753E4C50167
:10636000B4010F94C96C6FEF181624F0C501B40185
:106370000F949A6CF601648338CFD60111968C91F4
:106380001197807F8C6011968C9311978D859E85D7
:1063900015969C938E93149728CF6AE679E08EEB3E
:1063A00091E10F9477356A856F708EEB91E10E94D1
:1063B00074F667E679E08EEB91E10F947735F6019C
:1063C00061816F708EEB91E10E9474F68EEB91E12A
:1063D0000F9478340ACF9A859F7011968C911197FB
:1063E000807F892B11968C938D859E85AF85B8898A
:1063F000F60184839583A683B783F7CE9A859F7031
:10640000933089F09C3009F4B8CF4D855E856F8557
:106410007889F60144835583668377838181807F01
:10642000892B8183E2CE60E0C6010E941428D60148
:1064300014968C9314978F85988916968C9316973B
:1064400017968C91179790FB80F917968C93179756
:106450008E8515968C93159711968C911197807F48
:106460008260B6CE60E0CE0109960E941428D60163
:1064700014968C931497F0CF9A859F709D3008F0F6
:1064800057C0E92FF0E08827E75BFD4C8F4F0D9454
:10649000966BF5306332903213329032903256322E
:1064A00082328232823271327D32BD318D859E855B
:1064B000AF85B889F60184839583A683B7838181EC
:1064C000807F8660AECF6D8570E090E080E00F94B5
:1064D000C669D60114966D937D938D939C931797FF
:1064E00084CE6D857E858F8598890F94C869F60165
:1064F000648375838683978378CE6D857E858F854B
:106500009889E5CFF6018181807F982B91838D85D5
:106510009E85AF85B88984839583A683B78365CE2E
:1065200011968C911197807F982B11969C935CCF3C
:1065300065E579E08EEB91E10F9477356A856F70B0
:106540008EEB91E10E9474F662E579E08EEB91E1C9
:106550000F947735D60111966C9133CFFF24F394C5
:10656000EECD4D855E856F857889F6014483558330
:10657000668377838181807F982B918388E0DE0119
:10658000119601900D928A95E1F729813A814B810C
:106590005C816D817E818F81988568960FB6F894B5
:1065A000DEBF0FBECDBFDF91CF911F910F91FF9046
:1065B000EF90DF90CF90BF90AF909F908F907F90A3
:1065C0006F905F904F903F902F900895963009F410
:1065D00037C148F46D85913071F06FEF70E0933002
:1065E00051F060E008C0973009F436C19A506D85CB
:1065F0007E859230B0F784E68F8788898E7F888B7E
:106600001E868A85807F82608A876D872E8530E02E
:10661000AFEFB0E00F945F6B812C912C54018A9402
:106620006115F4E67F078105910544F424E630E026
:1066300040E050E00F942D6B49015A0114012D8563
:106640002A8B022F10E0FF2009F470C088898695FC
:10665000A82FA150BB0B7D01BFEFEB16FB0609F085
:106660001BC1E0E88E1691040CF0FDC08FE790E0AE
:1066700088199909809FD001819FB00D909FB00D1E
:1066800011242FEF30E00F94AD6B21E83EE740E09E
:1066900050E00F942D6BD60117962C93ABE9B0E028
:1066A000A50194010F944C6B3FE7432E512C612CB4
:1066B000712CA30192010F942D6B2C593F4F4F4F1A
:1066C0005F4F1901AEEFB1E0A50194010F944C6B3F
:1066D000A30192010F942D6BD8010F944C6B2FEFF7
:1066E00030E040E050E00F942D6B89012F3F3105E1
:1066F00019F014F00FEF10E065E479E08EEB91E112
:106700000F947735B1018EEB91E10E947BF667E340
:1067100079E08EEB91E10F947735B8018EEB91E142
:106720000E947BF68EEB91E10F947834E5EBFFE26B
:10673000E491F0E0EE0FFF1FE556F04D8591949146
:10674000EBEFFFE2E4912F8538893170AFEFBFEFB7
:106750000F945F6B2DE631E040E050E00F942D6B1D
:1067600044275527AAEFB5E00F944C6BDC01CB0111
:106770009058AF4FBF4FCD01BB2797FDB095AB2FC2
:106780008E3FE1E09E0708F05FC1382F8F3F9105F3
:1067900008F47CC14EEF481B50E03FEF0F5F1F4FE6
:1067A000F101FF2731962094312C3E9FC0013F9F7D
:1067B000900D1124292F3327220D331DD8010F945A
:1067C000AD6B4B015C018824AA24BB245E9F900121
:1067D0005F9F300D1124232F3327220D331D0F947B
:1067E000AD6BBB27A92F982F872F882A992AAA2A11
:1067F0004E9F90014F9F300D1124232F3327220DE0
:10680000331DD8010F94AD6BB82FA72F962F882773
:1068100088279927BB2788299929AA29F601A683C1
:10682000958384836BE079E08EEB91E10F9477356B
:10683000C6010E94F42560E080E00F949C06D5CC50
:106840006D857E858F85988924E630E040E050E0B4
:106850000F942D6BB901CFCE6D857E858F8598897C
:106860000F94936CC8CEA5019401205831094109B9
:106870005109ABE9B0E00F944C6B2FE730E040E0FA
:1068800050E00F942D6B2C593F4F4F4F5F4F190124
:10689000D60117961C9230CF9701AAEBBFEF0F9449
:1068A000A56B24E630E040E050E00F942D6B290109
:1068B0003A01B4E64B0E511C611C711C26E430E019
:1068C000D7010F94AD6B24E630E040E050E00F9428
:1068D0002D6BDA01C9014E96A11DB11D8D8B9E8BCA
:1068E000AF8BB88F90E8891691040CF092C08FE7B7
:1068F00090E088199909809FD001819FB00D909FE9
:10690000B00D11242D893E894F89588D0F94576BF6
:106910009B01AC01AFEFB0E00F944C6B24E63AE67C
:1069200040E050E00F942D6BD60117962C93A501F3
:106930009401240D351D461D571DAEEFB1E00F9497
:106940004C6B23EE30E040E050E00F942D6B79016A
:106950008A013C8B2B8BAFEFB0E0A50194010F9423
:106960004C6B2FE730E040E050E00F942D6B1901A5
:10697000EA89AE2FB0E0A80197010F944C6B2FEF7E
:1069800030E040E050E00F942D6B89012F3F31053E
:1069900019F014F00FEF10E061E379E08EEB91E174
:1069A0000F9477352AE030E0B301A2018EEB91E13C
:1069B0000F949A346BE279E08EEB91E10F94773586
:1069C0002AE030E04D895E896F89788D8EEB91E108
:1069D0000F949A3463E279E08EEB91E10F9477356E
:1069E000B1018EEB91E10E947BF66BE179E08EEBD9
:1069F00091E10F947735B8018EEB91E10E947BF61F
:106A000062E179E08EEB91E10F9477356B897C89B7
:106A100085CEA50194012058310941095109ABE9FE
:106A2000B0E00F944C6B2FE730E040E050E00F9463
:106A30002D6B2C593F4F4F4F5F4F1901D6011796C1
:106A40001C921C8A1B8AA8CF8C3FF3E09F0768F436
:106A50008D3F22E0920728F452E0580F3FEF40E0CC
:106A60009DCE3CEF381B5FEFFACF8A3F35E09307AE
:106A700081F08B3FE4E09E0728F444E0480F5FEF8D
:106A800030E08CCE5AEF581B30E001C050E04FEFA1
:106A900085CE50E0F9CF69EF78E08EEB91E10F946D
:106AA00077356A856F708EEB91E10E9474F666EF20
:106AB00078E04CCD4F925F926F927F928F929F922F
:106AC000AF92BF92CF92DF92EF92FF920F931F93FC
:106AD000CF93DF93CDB7DEB768970FB6F894DEBFDC
:106AE0000FBECDBF098B1A8B2B8B3C8B4D8B5E8BD6
:106AF0006F8B788FDC0112962D913C911397232B8D
:106B000009F4DEC0CC2009F4DBC06C01ED91FC91EE
:106B1000008CF18DE02D19955C0167E57CE18EEB31
:106B200091E10F947735CE0141960E94F425A1148E
:106B3000B10471F460E0CE0141960E941428682FE0
:106B4000F601848195810F94D74F81E090E0BAC01F
:106B5000CE0141960E948AB24C0194E0F2E0AF1659
:106B6000B10459F081E1A816B10409F445C091E0DF
:106B7000A1E0AA16B10409F495E019861A861B86CD
:106B80001C861D861E861F86188A8A85807F892B13
:106B90008A87EE24EA94FE2C09891A892B893C897C
:106BA0004D895E896F89788DCE0109960E944530A6
:106BB0006DE47CE18EEB91E10F947735CE0109967F
:106BC0000E94F425B2E0AB16B10489F0E1E1AE1603
:106BD000B104B1F0AA94AB2809F0B7CF188963E0EB
:106BE00070E0C6010E94A2EF612F0F94D74F6F850E
:106BF000F6018481958151C0888D8170888FBCCFCA
:106C00000FE710E08FEF88169806A9F0092C000C0A
:106C1000AA08BB08A5019401295931094109510964
:106C2000AFEFB0E00F944C6B2BE531E040E050E06B
:106C30000F942D6B890163E070E0C6010E94A2EF02
:106C40005C01288930E0D8010F94AD6B412C512CA8
:106C500032014A94A30192010F942D6B622FC5015A
:106C60000F94D74F64E070E0C6010E94A2EF5C0170
:106C7000AFEFB0E0A01BB10B288930E00F94AD6BF3
:106C8000A30192010F942D6B622FC5010F94D74F72
:106C90006F85D60114968D919C910F94D74F1E85C8
:106CA00061E070E0C6010E94A2EF612F0F94D74F00
:106CB0001D8562E070E0C6010E94A2EF612F43CF04
:106CC00090E080E068960FB6F894DEBF0FBECDBFAF
:106CD000DF91CF911F910F91FF90EF90DF90CF90B8
:106CE000BF90AF909F908F907F906F905F904F90EC
:106CF00008956F927F928F929F92AF92BF92CF92A0
:106D0000DF92EF92FF920F931F93CF93DF933C019B
:106D1000DC0114968D919C911597892B71F4129634
:106D2000CD91DC9184E190E00F949361BC01CE01A0
:106D30000E944CB4E3019D838C83F301C481D5810F
:106D4000209769F466EE7DE187E191E10F94773554
:106D500087E191E10F94783490E080E0B9C24FEF81
:106D60005FEFBA0180E00F9452566E837F8388876D
:106D70009987D3011496ED90FC901597E114F104D6
:106D8000D1F01296ED91FC913097A9F0C481D58194
:106D9000209789F088858F70853069F4CE010E9434
:106DA00034F7823040F00091D50C1091D60C0115CB
:106DB000110509F08CC069EA7DE187E191E10F944A
:106DC000773561E070E0E3018C819D81892B11F4BE
:106DD00070E060E087E191E10E947BF667EA7DE187
:106DE00087E191E10F94773561E070E0F3018281F2
:106DF0009381892B11F470E060E087E191E10E94BA
:106E00007BF665EA7DE187E191E10F947735D30167
:106E10001296ED91FC9161E070E084819581892B5F
:106E200011F470E060E087E191E10E947BF663EA93
:106E30007DE187E191E10F947735E301EA81FB8100
:106E40000480F581E02D80858F7061E070E08530F1
:106E500011F470E060E087E191E10E947BF661EA65
:106E60007DE187E191E10F947735D3011296ED91A1
:106E7000FC91848195810E9434F761E070E082305A
:106E800010F070E060E087E191E10E947BF687E11D
:106E900091E10F9478346EEB7DE187E191E10F94FD
:106EA000773587E191E10F947834D301ED91FC912E
:106EB0000484F585E02D61E0C3011995E301E881C3
:106EC000F9810084F185E02DC301199545CF61E07A
:106ED000CE010E9462F6EC0188858F70843029F41F
:106EE00069857A856115710539F469E87DE187E185
:106EF00091E10F947735CBCFC8010E94EAF58C0160
:106F0000009769F467E67DE187E191E10F947735B9
:106F100069857A8587E191E10F942035B8CF67EBD9
:106F200075E00E94EAF5009709F4D8C0EC012885C5
:106F30002F70243009F0D2C0C984DA84D0E0C0E0D8
:106F4000C114D10409F4BDC0BE016F54734EC60113
:106F50000F94CC63892B09F0AFC0FE01EB54F34EC4
:106F600025913491922F832FF701928383836EEBC7
:106F700075E0C8010E94EAF5E301EC81FD8100970C
:106F800009F4B4C0DC0118962C9118972F702230A8
:106F900009F0ACC019968D919D910D90BC91A02DDA
:106FA0000097A105B10509F4A1C0918380834081B8
:106FB0005181052E000C660B770B22818CE39EE03D
:106FC0000F94833663EC75E0C8010E94EAF57C01FA
:106FD000F301C481D581009709F48EC0DC011896B5
:106FE0008C918F70863009F087C068EC75E0C7011E
:106FF0000E94EAF59B878A876DEC75E0C7010E94C5
:10700000EAF59D878C8761ED75E0C7010E94EAF57E
:107010009F878E8767ED75E0C7010E94EAF5998B1F
:10702000888B6CED75E0C7010E94EAF5009709F4C2
:1070300060C0FC01818592859D838C8362EE75E042
:10704000C8010E94EAF59B8B8A8B892B09F41EC12B
:1070500061E67DE18EEB91E10F9477356BE47DE1A4
:107060008EEB91E10F9477358EEB91E10F947834AC
:10707000D3011496ED91FC910288F389E02DC6812D
:10708000D781209709F441C066EE75E0CE010E94D9
:10709000EAF5009769F0FC0120852F70213041F45A
:1070A0008185882329F068817981C3010E940A1CA7
:1070B0000A80DB81C02DE5CF2696C834D10509F0C2
:1070C0003FCF64E97CE18EEB91E10F9477358EEB55
:1070D00091E10F94783496E080E046CF86E090E02E
:1070E000D70113969C938E93129741CF80E895E237
:1070F0005CCF88EE93E0A0CF1B861A8688EE93E0E3
:107100009D838C831D861C8699CF65E47DE18EEB83
:1071100091E10F9477356FE27DE18EEB91E10F9471
:1071200077358EEB91E10F947834D3011496ED917D
:10713000FC910288F389E02DE680F780E114F104E8
:1071400009F478C06FEE75E0C7010E94EAF5009778
:1071500009F465C063EF75E00E94EAF58C010097C1
:1071600009F45DC0EC0188858F70823009F04BC056
:10717000C984DA84D3011496ED91FC910288F389D5
:10718000E02D309709F453C0C681D78146010D2CFC
:10719000000CAA08BB08209709F449C067EF75E006
:1071A000CE010E94EAF50097F1F1FC0120852F70D5
:1071B0002230C9F581859285A385B4858815990506
:1071C000AA05BB0581F568E07DE18EEB91E10F94A6
:1071D0007735688179818EEB91E10F94203569EFE5
:1071E0007CE18EEB91E10F947735B6018EEB91E166
:1071F0000E947BF68EEB91E10F947834688179815F
:10720000C3010E940A1CF80180858F70843039F414
:10721000D80119966D917C91C3010E940A1CE70167
:10722000EA80FB808BCF0A80DB81C02DB4CF70E079
:1072300060E0E6CF69E27DE18EEB91E10F94773576
:107240006FE07DE18EEB91E10F9477358EEB91E16C
:107250000F947834D3011296ED91FC9162E0848111
:1072600095810E9462F6009789F0FC01C681D78162
:10727000209761F0CE010E94361B882319F0CE01C1
:107280000F948A040A80DB81C02DF2CF61ED7DE18D
:107290008DE091E10F947735D3011296ED91FC9139
:1072A0000280F381E02D608171818DE091E10F9486
:1072B00020358DE091E10F947834E301E881F98184
:1072C0000484F585E02D62E0C301199581E090E02A
:1072D000DF91CF911F910F91FF90EF90DF90CF90B2
:1072E000BF90AF909F908F907F906F900895CF93B5
:1072F000DF93EC016FE27CE18EEB91E10F94773547
:10730000EA81FB810280F381E02D608171818EEB47
:1073100091E10F9420358EEB91E10F947834E88160
:10732000F9810484F585E02D62E0CE01199581E0B4
:1073300090E0DF91CF910895DC01ED91FC91048400
:10734000F585E02D62E0199581E090E00895EF92D7
:10735000FF920F931F93CF93DF9300D000D0CDB750
:10736000DEB78091E9109091EA10892B09F46CC086
:1073700087E70E948EF78091E9109091EA10DC0176
:10738000ED91FC910088F189E02D70E060E01995A5
:1073900010E000E08091E9109091EA10DC01ED919D
:1073A000FC9111971C962D913C910217130740F404
:1073B0000190F081E02D60E019950F5F1F4FEACF3B
:1073C0000088F189E02D70E060E019950AE114E091
:1073D0008EE1E82E84E0F82E8091E9109091EA1079
:1073E000F80161918F01DC01ED91FC910190F08138
:1073F000E02D1995E016F10679F78091E91090914A
:10740000EA10DC01ED91FC910488F589E02D1995D5
:1074100062EF7BE0CE0101960F941832CE01019607
:107420000F945413CE0101960F94D93187E090E068
:107430000E94AAFA87E090E00E94B4FA69E478E139
:107440008DE091E10F947735109209111092081197
:1074500080E090E1909304118093031184E890E020
:1074600090930B1180930A1181E08093051180E0C5
:1074700090E2909307118093061182E780930C119C
:1074800087EF90E10E9495AE87EF90E10E9440AFB8
:1074900088EC90E026960FB6F894DEBF0FBECDBF05
:1074A000DF91CF911F910F91FF90EF900895FF9280
:1074B0000F931F93CF93DF9300D000D0CDB7DEB7EB
:1074C0008C01BC01CE0101960F940F32BE016F5F9B
:1074D0007F4F8EEB91E10F9469358EEB91E10F9424
:1074E0007834CE0101960F94D93164E778E1CE016A
:1074F00001960F94E131BE016F5F7F4FC8010F9479
:107500001730F82ECE0101960F94D931FF2069F083
:10751000B801CE0101960F940F32CE0101960F945F
:107520005413CE0101960F94D93126960FB6F894D4
:10753000DEBF0FBECDBFDF91CF911F910F91FF90A6
:1075400008958F929F92BF92CF92DF92EF92FF9217
:107550000F931F93CF93DF93CDB7DEB7AE970FB6E0
:10756000F894DEBF0FBECDBF8091520C9091530CAA
:10757000892B09F43CC680913B13811138C6809158
:107580003B138F5F80933B1369E176E18DE091E1DE
:107590000F9477358DE091E10F9478340091520C7F
:1075A0001091530C6BEF75E0C8010E94EAF59093BF
:1075B00042138093411361E076E0C8010E94EAF52E
:1075C0009093DD0C8093DC0C6AE379E0C8010E94A3
:1075D000EAF590933E1380933D1368E076E0C8018E
:1075E0000E94EAF59093CB0C8093CA0C009739F176
:1075F000DC011696ED91FC91309709F120852F70F2
:107600002530E9F465E076E18DE091E10F9477357E
:107610008091CA0C9091CB0C0E9434F78093C90CD6
:10762000682F8DE091E10E9474F68DE091E10F9456
:107630007834E091CA0CF091CB0C868197819093BD
:10764000C80C8093C70C0E94FB1E6DE076E0809111
:10765000520C9091530C0E94EAF59093510C809338
:10766000500C009709F4B0C00E9434F7082F10E0C6
:107670000115110509F4A8C0000F111F000F111FFB
:1076800080914E0C90914F0C892B09F08EC078019F
:10769000013811051CF020E8E22EF12CC7010F94EF
:1076A000936190934F0C80934E0CE0924D0C10928E
:1076B0002F1310922E131092C60C1092C50C10921C
:1076C0002D131092311310923013C70101960F94AD
:1076D0009361909333138093321390932C13809380
:1076E0002B138E0D9F1D90932613809325130F94BB
:1076F000170960932713709328138093291390938D
:107700002A1390E080E0E0913213F0913313E80FF8
:10771000F91F10820196E816F906ACF782E090E0B6
:1077200090932F1380932E138091C50C9091C60CCB
:10773000009741F061E00F949C0660E08091C50CD9
:107740000F946E0680E98093C9001092C8001092D1
:10775000CD0083E08093CC008EE08093CA00F0924D
:107760001C02E0921B02209132133091331380915E
:107770001B0290911C02820F931F909326138093FB
:107780002513232B09F45DC065E975E18EEB91E1CA
:107790000F947735B7018EEB91E10E94BFFA82EC2E
:1077A00091EB90932413809323136BEE75E18DE09E
:1077B00091E10F947735B8018DE091E10E947BF65D
:1077C0008DE091E10F94783463E176E08091520C82
:1077D0009091530C0E94EAF58C01009709F46BC05C
:1077E0000E9434F7882309F466C06FEF680FC80160
:1077F0000E9462F6FC01E184F284909122139923A5
:1078000059F0809170008E7F809370001092221347
:10781000109219021092180282E1809317029111BE
:107820000F947B4FC7010F94A34F01E010E0E016C7
:10783000F10674F060E0C8010F94D74F0F5F1F4F3F
:10784000F6CF6EE775E18EEB91E10F949B35A7CFF4
:1078500060E775E18EEB91E10F9477350E94346E0D
:10786000AB01BC018EEB91E10E9471F68EEB91E1D0
:107870000F9478346FEC75E18DE091E10F947735DA
:10788000B7018DE091E10E947BF68DE091E10F94CC
:10789000783469EC75E18EEB91E10F9477350E94B5
:1078A000346EAB01BC018EEB91E10E9471F68EEB60
:1078B00091E10F9478340091520C1091530C67E1D0
:1078C00076E0C8010E94EAF59093D60C8093D50C1F
:1078D0006EE176E0C8010E94EAF59093441380932C
:1078E0004313892B09F448C080914513811144C08A
:1078F0008091361390913713892B09F0D8C16AE42F
:1079000075E18EEB91E10F9477358EEB91E10F9459
:1079100078348FE090E00F9493618C0188E1D80176
:1079200011968C93119712961C9212971C921E9688
:107930001C921E921D970F94AC0210933713009364
:107940003613012B09F08CC06BE375E187E191E1FF
:107950000F94773587E191E10F94783480E081705E
:107960008093451380914513882331F069EB75E1CD
:107970008DE091E10F9477351092391310923813FE
:10798000E0914113F0914213309709F4BFC2C680D1
:10799000D78000914113109142130115110509F48C
:1079A000AEC2C114D10409F4AAC2F60180858F7059
:1079B000853099F7C6010E9434F7823070F3A80130
:1079C000B601CE0101960E9497BECE0101960E949B
:1079D00069B38823E1F18C859D85009709F406C27F
:1079E000DC01ED91FC910284F385E02D1995892B42
:1079F00049F08C859D85DC01ED91FC910084F18539
:107A0000E02D19958C859D85DC01ED91FC9106801A
:107A1000F781E02D1995892BD1F0CE0101960E94B6
:107A20009BBC882341F040E050E160E070E0CE0173
:107A300001960E942FB68F819885892B41F040E0F6
:107A400050E260E070E0CE0101960E942FB6D601B0
:107A50001296CD90DC90CE0101960E9464BE99CF23
:107A60000F94AC0280913613909137130F942250EB
:107A7000882309F489C06CE175E18DE091E10F94F0
:107A80009B3580913613909137130F94F251E0910A
:107A90003613F091371381E08083809136139091F3
:107AA00037130F94005268E075E1811102C063EF53
:107AB00074E18EEB91E10F949B358091431390918B
:107AC0004413892B09F44ACF8091341390913513D4
:107AD000892B09F0DEC083E190E00F9493618C0163
:107AE000809136139091371329EE31E0F801328BF3
:107AF000218B968385831482108289E0818381E0C3
:107B00008283838310933513009334130F941709E2
:107B10006B017C01F0E1CF0EF7E2DF1EE11CF11CEE
:107B2000D8011596ED91FC9116978FEF83871486F7
:107B3000138214821582168217821086118612868D
:107B400014961C92BB24B394BE01605E7F4FF80173
:107B5000858196810F94DA5218160CF095C00F9417
:107B600017096C157D058E059F0508F08DC0DE0197
:107B7000909698E080E0915019F1ED91E827F0E0BF
:107B8000EE55FC4C8491F7CF0F94DC558091361361
:107B9000909137130F942250882359F066ED74E1C9
:107BA0008DE091E10F9477358DE091E10F94783479
:107BB00084CF6AEB74E187E191E10F949B35CECEDF
:107BC0009FA19813C1CFD8018C91811138C015960F
:107BD0008D919C910F940052BE01605E7F4FF80121
:107BE000858196810F94D35140E064EBD8011596BE
:107BF0008D919C910F94AD51F80185809680C401C0
:107C00000F943151C4010F94055067E884E09FE060
:107C10000F94C42C60E884E09FE00F94C42C0F9470
:107C2000E108C4010F943151982ED80115968D9119
:107C30009C910F94005295FC02C0F801B082AE01F5
:107C40004F5F5F4FBE01605E7F4FC8010F9441528E
:107C5000D80111969C9088A1803109F4CAC2BE0156
:107C6000605E7F4FC8010F94B052891510F5F8017E
:107C70008181D80111968C93119714968C91149749
:107C80008F5F14968C9360CFE0913413F09135138D
:107C90001282E0914313F0914413E680F7809FE74E
:107CA000D92E8091431390914413892B71F481E074
:107CB00056CE88A1803111F48CE0DBCFBE01605E2E
:107CC0007F4FC8010F94B052D4CFE114F10479F37F
:107CD000BE01605E7F4FF701808191810E94C96F74
:107CE000882329F363EA74E18EEB91E10F947735F1
:107CF000D7016D917C918EEB91E10F9420358EEB45
:107D000091E10F9478340091341310913513AE0142
:107D10004F5F5F4FBE01605E7F4FC8010F94965268
:107D2000882309F45EC088A1803109F45AC0DD823D
:107D3000F801858196810F940052BE01605E7F4FED
:107D4000D80115968D919C910F94D35140E06EE42B
:107D5000F801858196810F94AD5140E06B81D80187
:107D600015968D919C910F94AD5140E06C81F80176
:107D7000858196810F94AD5188A1803141F040E01A
:107D80006D81D80115968D919C910F94AD51F8019C
:107D9000858196810F940052BE01605E7F4FD801AD
:107DA00015968D919C910F94D351F801408168E410
:107DB000858196810F94AD5164E170E080E090E0A0
:107DC0000F94E408D8018C91882331F06AE070E0C8
:107DD00080E090E00F94E408F801858196810F948B
:107DE0000052D7011296ED90FC905BCF70E060E0FE
:107DF000CE0101960E945CB58C01912C812C97FFDD
:107E000006C011950195110988248394912CCE0107
:107E100001960E949BBCE82EF12C8B85853091F059
:107E2000863009F014CEB02E61E0802F0F949C06AE
:107E300061E0892809F441C0EA94EF2809F041C0C3
:107E400060E03FC0EF2829F462E0CE0101960E9475
:107E50007CBC40E050E160E070E0CE0101960E9401
:107E60002FB68F819885892B41F040E050E260E089
:107E700070E0CE0101960E942FB661E0802F0F9432
:107E80009C0660E0802F0F946E0661EB75E18EEB2F
:107E900091E10F947735B8018EEB91E10E947BF66A
:107EA0006CEA75E18EEB91E10F9477356AEA75E142
:107EB0008EEB91E10F947735CACDEA94EF2809F063
:107EC000BFCFE62EF12C8B2D0F946E0665EA75E17F
:107ED0008EEB91E10F947735B8018EEB91E10E9422
:107EE0007BF663EA75E18EEB91E10F947735B7018C
:107EF0008EEB91E10E947BF661EA75E1D9CFF80142
:107F00008681978190933913809338138EEB91E19A
:107F10000F9478346FE874E18DE091E10F94773538
:107F20008DE091E10F947834E0913D13F0913E1390
:107F3000309709F4A8C080913B138F5F80933B1367
:107F4000E680F780E114F10409F498C0D70118968F
:107F50008C918F70863009F07EC0F9A6E8A670E09B
:107F600060E0CE0188960E94A7E08DA59EA5892B92
:107F700009F471C08091520C9091530C892B09F433
:107F80006AC0C8A4D9A4C114D104B9F1F60180858E
:107F90008F70863091F5D9A2C8A270E060E0CE0162
:107FA00080960E94A7E0EDA1FEA1108211821282AC
:107FB000138269E375E0C6010E94EAF5FC01892B92
:107FC000E1F090859F7095509230B8F4068117814A
:107FD0000115110591F01A830983B601CE010196AE
:107FE0000E94A7E0EE81FF8110821182128213822B
:107FF000D80112960D911C91EBCF6AE874E18EEBDB
:1080000091E10F9477356BA58EEB91E10E9474F6A8
:1080100068E874E18EEB91E10F9477356AA58EEBF9
:1080200091E10E9474F68EEB91E10F947834EDA506
:10803000FEA510821182128213828AA5843078F400
:10804000823098F060E08BA50F949C06EDA5FEA50C
:108050008181807F8183F701E280F38073CF803458
:1080600059F0823421F08032B1F762E0ECCF60E069
:108070008BA50F949C06EFCF62E0FACF80913B1363
:10808000815080933B136BE774E18DE091E10F9495
:10809000773563E774E18DE091E10F94773581E006
:1080A0002091411330914213232B09F480E00E9468
:1080B000B41B6AE674E18DE091E10F94773581E0BD
:1080C00020913D1330913E13232B09F480E00E9450
:1080D000B41B6BE574E18DE091E10F94773560E5B9
:1080E00074E18DE091E10F94773581E02091D50C1A
:1080F0003091D60C232B09F480E00E94B41B69E474
:1081000074E18DE091E10F94773581E02091C70C07
:108110003091C80C232B09F480E00E94B41B60E46A
:1081200074E18DE091E10F94773581E02091431364
:1081300030914413232B09F480E00E94B41B67E3C1
:1081400074E18DE091E10F9477358091D90C0E9414
:10815000B41B8DE091E10F94783462E374E18DE01B
:1081600091E10F9477350E94346EAB01BC018DE034
:1081700091E10E9471F68DE091E10F94783481E0F5
:108180008093CC0C8AED90E10F946548882351F0E0
:108190008AED90E10F94874884E090E0909340133B
:1081A00080933F1380913F1390914013079731F4D0
:1081B00084E090E09093401380933F1380913B13B1
:1081C000815080933B138091CC0CAE960FB6F894FF
:1081D000DEBF0FBECDBFDF91CF911F910F91FF90FA
:1081E000EF90DF90CF90BF909F908F90089580E0A8
:1081F000ECCFFCE0F91508F43ACD5ECD5F926F92BA
:108200007F928F929F92AF92BF92CF92DF92EF9226
:10821000FF920F931F93CF93DF93CDB7DEB7C15774
:10822000D1090FB6F894DEBF0FBECDBF4C018B0154
:10823000F42E642F8EEB91E10E9474F66EE07CE0E8
:108240008EEB91E10F947735B801CE0101965C0178
:108250000F940F32B5018EEB91E10F9469358EEBDF
:1082600091E10F947834C5010F94D93192E0F9125D
:10827000A4C26CE07CE0C5010F94E131B501C801F6
:108280000F944730F82EC5010F94D931FF2009F41F
:108290000DC320E04DE251E0B40188EB90E10F9472
:1082A000BF39E090DA0CF090DB0C65E07CE0CE01A9
:1082B00084599F4F0F94E1316EEF7BE0CE018A59D4
:1082C0009F4F0F94E131CE01865A9F4F0F94AB4ED2
:1082D000A0961FADA0976F960FAD6F976E96DFAC0F
:1082E0006E976D96CFAC6D9762EF7BE0CE01819675
:1082F0000F941832BE016F5D7F4FC5010F940F328E
:108300006C2DC5010F942A3161E276E00F945B3148
:108310006D2D0F942A3161E276E00F945B31602F6E
:108320000F942A3161E276E00F945B31612F0F9454
:108330002A31BC01CE01805A9F4F0F940F32C501E4
:108340000F94D931CE0181960F94D93169EF7BE03A
:10835000CE018C5A9F4F0F94E13162EF7BE0CE014A
:10836000825B9F4F0F94183209EE10E1D8011896E6
:108370006C9170E084E0759567958A95E1F7C50189
:108380000E9462F74D815E8169817A81CE01825BB4
:108390009F4F0F94D830C5010F94D931F8016085F3
:1083A0006F7070E0C5010E9462F74D815E81698146
:1083B0007A81CE01825B9F4F0F94D830C5010F9414
:1083C000D9310F5F1F4FF0E10F3E1F0779F663EFC2
:1083D0007BE0CE01885B9F4F0F94E13161EE7BE043
:1083E000CE0181960F94E131BE016F5D7F4FCE01CA
:1083F000805C9F4F0F940F3226960EAD1FAD2697CF
:10840000085E1F4FB801CE01805C9F4F0F94B030C3
:10841000811184C0CE01805C9F4F0F941831BE0142
:10842000685B7F4FCE01805C9F4F0F947531BE011A
:10843000625B7F4F0F947531BE016C5A7F4F0F9472
:108440007531BE01605A7F4F0F947531BE016A5974
:108450007F4F0F9475318C014AE0B50180E590E0C3
:108460000F944864F50101900020E9F73197AF01BE
:108470004A195B09B501C8010F94D830811103C0B6
:10848000C8010F941831BE0164597F4FC8010F9481
:108490007531B7010F945B31BC01C4010F9469358C
:1084A000C4010F947834CE01805C9F4F0F94D93172
:1084B000CE0181960F94D931CE01885B9F4F0F94E6
:1084C000D931CE01825B9F4F0F94D931CE018C5AA6
:1084D0009F4F0F94D931CE01805A9F4F0F94D931BD
:1084E000CE018A599F4F0F94D931CE0184599F4FA5
:1084F0000F94D931C4010F94783464E670E080E0C1
:1085000090E00F94E408D401ED91FC910488F58982
:10851000E02DC401199501E010E0ABC022962EAD0C
:108520003FAD229726968EAD9FAD269768EC7BE0F7
:10853000820F931F0F94D56326961FAF0EAF269719
:108540006ECF2A966EAD7FAD2A97CE0181960E949E
:108550007DFE892B09F464C124961CAE1DAE1EAEAF
:108560001FAE249728961CAE1DAE1EAE1FAE2897D8
:1085700022968FAD2297807F22968FAF229740E080
:1085800050E3BE016F5D7F4FCE01805C9F4F0E9424
:10859000512700E020E030E340E250E0B501CE0199
:1085A000805C9F4F0E94CF23BC01C6010F94B33162
:1085B00008EC10E137C1EE2009F4FDC046E050E0C0
:1085C00070E060E0C8010F94A32F409141135091D7
:1085D0004213D8016D917C91CE0181960E94C7BD56
:1085E000CE0181960E9469B300E911E08823E9F188
:1085F0008BA5873061F4CE0181960E94D7D661E0C9
:10860000892B09F462E0CE0181960E947CBC2496FD
:108610001CAE1DAE1EAE1FAE249728961CAE1DAE1E
:108620001EAE1FAE289722968FAD2297807F22968E
:108630008FAF229740E050E3BE016F5D7F4FCE01C8
:10864000805C9F4F0E94512700E020E030E340E231
:1086500050E0B501CE01805C9F4F0E94CF23BC014A
:10866000C6010F94B33108EC10E1CE0181960E944F
:1086700064BEC801CF58DF4F0FB6F894DEBF0FBEFF
:10868000CDBFDF91CF911F910F91FF90EF90DF90C1
:10869000CF90BF90AF909F908F907F906F905F90A2
:1086A0000895F801608171810E94EAF57C01892BAF
:1086B00009F044C104E911E0DCCFEE2009F47BC0ED
:1086C00049E050E070E060E0C8010F94A32F4AE059
:1086D000B401C5010F94F53341E050E060EA75E064
:1086E000C8010F94D8304D815E8169817A81C801BB
:1086F0000F94D83064EA7BE08EEB91E10F947735EC
:10870000B801CE0181960F940F32BE016F5D7F4F8D
:108710008EEB91E10F9469358EEB91E10F947834F3
:10872000CE0181960F94D9316CE97BE0CE01819620
:108730000F94E131F801848195812DA13EA182172A
:108740009307E1F4892BA1F1E080F18069A07AA080
:10875000D7018D917D01882359F1082E000C990BCA
:108760000F947C6F6C01F30181913F01082E000C86
:10877000990B0F947C6FC816D90651F3CE018196E0
:108780000F94D931552041F021E048EC50E0B4017C
:1087900088EB90E10F94BF39D8018D919C910F9493
:1087A0003F3B009711F484E991E08C01C50141C081
:1087B00055245394E3CF01E97ECFB1E0FB1274C09E
:1087C00061EC7BE0C5010F94E131B501C8010F9464
:1087D0001730582EC5010F94D931552069F1EE207C
:1087E00051F346E050E070E060E0C8010F94A32F21
:1087F0004AE0B401CE01885B9F4F0F94F53340915E
:10880000411350914213F80160817181CE0181962C
:108810000E94C7BDCE0181960E9469B3811191CE9D
:1088200000E911E0CE0181960E9464BECE01885B12
:108830009F4F0F94D9311DCF6AEA7BE0C5010F9499
:10884000E131B501C8010F941730F82EC5010F941E
:10885000D931F11032CF6FE87BE0C5010F94E131DF
:10886000B501C8010F941730182FC5010F94D931E5
:1088700000E0112309F4FDCE80E00E94A0FA67E633
:108880007BE08DE091E10F9477358DE091E10F94DD
:10889000783462EF7BE0C5010F941832C5010F9464
:1088A0005413C5010F94D93100E036CE6AEB7BE05A
:1088B000C5010F94E131B501C8010F941730F82EAE
:1088C000C5010F94D931F11076CE64EB7BE0C50180
:1088D0000F94E131B501C8010F941730F82EC5018E
:1088E0000F94D931FF2001F3EE2009F464CF45E065
:1088F00050E070E060E0C8010F94A32F61E276E0E1
:10890000C8010F943230882339F0E0904113F09081
:108910004213E114F10491F462EF7BE0C8010F947B
:108920003230811107C0809141139091421300971A
:1089300009F0B7CEE090520CF090530C20E048ECD8
:1089400050E2B40188EB90E10F94BF39C4010F9459
:1089500078341C821B8285EC92E09A8389839E8204
:108960008D828FEF9FEF98878F83B701C5010E949B
:10897000FDFCC3CD8F929F92AF92BF92CF92DF92B8
:10898000EF92FF920F931F93CF93DF93CDB7DEB794
:10899000CF55D1090FB6F894DEBF0FBECDBF8C0105
:1089A0006B016115710519F04115510579F56DE7F8
:1089B0007CE08EEB91E10F94773564E77CE08EEB01
:1089C00091E10F947735B8018EEB91E10F9420354A
:1089D00062E77CE08EEB91E10F9477358EEB91E1CD
:1089E0000F947834C15ADF4F0FB6F894DEBF0FBE34
:1089F000CDBFDF91CF911F910F91FF90EF90DF904E
:108A0000CF90BF90AF909F908F900895460F571FC3
:108A1000DA011C920E94346E4B016CE67CE08EEB16
:108A200091E10F947735B4018EEB91E10E947BF6D2
:108A300069E67CE08EEB91E10F947735B8018EEB1F
:108A400091E10F94203566E67CE08EEB91E10F9486
:108A50007735BAE38B16B1E09B064CF469E57CE010
:108A600087E191E10F94773587E191E1B9CF67E52F
:108A70007CE08EEB91E10F947735B6018EEB91E1BE
:108A80000F94203565E57CE08EEB91E10F9477350E
:108A90008EEB91E10F9478341A821982FE0133969D
:108AA0008EE3DF011D928A95E9F780913F13909143
:108AB0004013059791F563E070E0C8010E94BD1F67
:108AC0007C01892BD1F5E091160FF091170F808171
:108AD00080FF88CF61E070E0C8010E94BD1F892B34
:108AE00009F480CF64E270E0C8010F943470892BE0
:108AF00009F078CF67E37CE08EEB91E10F94773556
:108B0000B8018EEB91E10F9420358EEB91E10F943B
:108B10007834C8010F94410465CF61E070E0C8016A
:108B20000E94BD1F7C01892B09F465C04FE350E012
:108B3000B801CE0101960F942570A12CBB24B394EB
:108B4000E00EF11E6EE27CE0C7010F94CC63892B2E
:108B500009F45EC064E270E0C8010F943470892BA0
:108B600009F040CFB11003C0AA2009F43BCF4091D7
:108B7000411350914213B701CE018F5B9F4F0E946A
:108B8000C7BDCE018F5B9F4F0E9469B3182F88230A
:108B900059F0B601CE018F5B9F4F0E947DFE11E020
:108BA000181619060CF010E0CE018F5B9F4F0E9443
:108BB00064BE112309F416CF8981882309F412CFEA
:108BC00080913F1390914013059709F40BCF60E11A
:108BD0007CE08EEB91E10F947735BE016F5F7F4FA4
:108BE0008EEB91E10F9420358EEB91E10F94783468
:108BF000CE0101968FCF62E070E0C8010E94BD1FD8
:108C00007C01892B09F4EECEAA24A394B12C98CF31
:108C1000F60101900020E9F73197EC19FD09329730
:108C200008F498CFC8010F944104B11003C0AA20E2
:108C300009F4D8CEC6010F943F3BD4CE0F931F93B7
:108C4000CF93DF93CDB7DEB76F970FB6F894DEBF43
:108C50000FBECDBF2091520C3091530C232B09F441
:108C600013C120913B13022E000C330B8217930784
:108C7000B4F460E57BE087E191E10F94773587E11B
:108C800091E10F94783480E06F960FB6F894DEBFD0
:108C90000FBECDBFDF91CF911F910F9108956AE371
:108CA0007BE08EEB91E10F9477358EEB91E10F94A1
:108CB00078348091550C8F5F8093550C65EF7AE086
:108CC0008DE091E10F9477358DE091E10F94783448
:108CD000E0913D13F0913E13309709F180913B13E1
:108CE0008F5F80933B13068117810115110591F069
:108CF000D80118968C918F70863041F41A830983BD
:108D000070E060E0CE0101960E94A7E0F8010281C8
:108D10001381EBCF80913B13815080933B13E09103
:108D20004113F09142133097A1F10681178101158B
:108D30001105C9F1D80118968C918F70853029F5ED
:108D4000C8010E9434F7882301F1409141135091EA
:108D50004213F80160817181CE0101960E94C7BD66
:108D6000CE0101960E9469B3882359F08C859D85B8
:108D7000009739F0DC01ED91FC910084F185E02D44
:108D80001995CE0101960E9464BEF80102811381FB
:108D9000CECF6AE27BE08EEB91E10F9477358EEBDC
:108DA00091E10F947834109239131092381362E2E3
:108DB0007BE08EEB91E10F9477358EEB91E10F9490
:108DC000783464E670E080E090E00F94E40810925C
:108DD000D90C1092CC0C6AE07BE08EEB91E10F9401
:108DE00077350E94346EAB01BC018EEB91E10E949D
:108DF00071F68091520C9091530C009711F00F94E2
:108E0000CF011092530C1092520C10923E131092FC
:108E10003D1310924213109241131092DD0C1092E8
:108E2000DC0C1092CB0C1092CA0C1092C80C109251
:108E3000C70C1092DB0C1092DA0C1092C90C109235
:108E4000510C1092500C1092441310924313109234
:108E5000D60C1092D50C65E07BE08EEB91E10F947F
:108E600077350E94346EAB01BC018EEB91E10E941C
:108E700071F68EEB91E10F9478341092C40C8091CE
:108E8000550C81508093550C81E0FECE4F925F923D
:108E90006F927F928F929F92AF92BF92CF92DF920A
:108EA000EF92FF920F931F93CF93DF93CDB7DEB76F
:108EB000C859D1090FB6F894DEBF0FBECDBF8E01E1
:108EC0000F5B1F4FD8011D921C92FE01ED5BFF4FFF
:108ED0008EE1DF011D928A95E9F78091E91090916A
:108EE000EA10892B09F4CEC10E94A3F7882309F464
:108EF000C9C182E70E948EF78091E9109091EA1033
:108F0000DC01ED91FC910088F189E02D60E270E0D8
:108F100019954FE150E0B8018091E9109091EA1065
:108F20000E94E8F77C018091E9109091EA10DC0141
:108F3000ED91FC910488F589E02D1995E114F10477
:108F400009F4A0C1F801EE0DFF1D10828091F6100A
:108F50001F928F938091F5101F928F938091F41040
:108F60001F928F938091F3101F928F938091F21034
:108F70001F928F938091F1101F928F9383E296E05E
:108F80009F938F931F9280E48F93FE0131966F0120
:108F9000FF93EF930F943F7063E679E18DE091E1E9
:108FA0000F947735B8018DE091E10F942035B6012B
:108FB0008DE091E10F9420358DE091E10F947834AC
:108FC0007E01F1E6EF0EF11CD70113961C921E9262
:108FD000129788EE93E0A0E0B0E0F70184839583D8
:108FE000A683B78388E0848788EE93E09687858799
:108FF0008DE792E091838083108A1786128B018B14
:10900000148A138A80E590E0968B858B118E6BE72E
:1090100078E18EEB91E10F9477356BEE70E1CE0144
:1090200085589F4F0F940F32BE0165587F4F8EEBCE
:1090300091E10F9469358EEB91E10F947834CE0174
:1090400085589F4F0F94D93162E576E0CE01835762
:109050009F4F0F94183262E576E0CE0185589F4FFE
:109060000F941832BE0165587F4FCE018B579F4F2A
:109070000F940F326BEE70E1CE018B579F4F0F9420
:109080007531BE0163577F4F0F947531BC01CE011E
:109090008D569F4F0F940F32CE018B579F4F0F94D9
:1090A000D931CE0185589F4F0F94D931CE018357C6
:1090B0009F4F0F94D93184E596E0CB57DF4F9983CA
:1090C0008883C558D040C757DF4F19821882C958C6
:1090D000D040C557DF4F19821882CB58D040CD56AB
:1090E000DF4F88819981C359D040C957DF4F998399
:1090F0008883C758D0406DE579E18EEB91E10F94FC
:1091000077350E94346EAB01BC018EEB91E10E9479
:1091100071F68EEB91E10F94783464E670E080E0B4
:1091200090E00F94E40887E59AE3D70150969C936A
:109130008E931F976FE571E08DE192E00F94D664F6
:109140008C010FB6F894DEBF0FBECDBF892B09F49A
:10915000F4C083E090E00F949361D8011D969C9336
:109160008E931C97FC01F182E0821282C7010F945A
:109170006548882319F0C7010F948748D701539693
:109180006D917C9154975596AD90BC906115710589
:1091900009F48FC0CE0185589F4F0F94B735A501B4
:1091A000BE0165587F4FC7010F942D4E1816190642
:1091B0000CF0C0C0D7015196BC9051975296AC901C
:1091C000DF92CF9286ED98E19F938F931F930F9339
:1091D0000F945D65DF92CF9281ED98E19F938F931D
:1091E0001F930F930F945D65D8011C96ED91FC9130
:1091F00081E08283DF92CF928EEC98E19F938F93F0
:109200001F930F930F945D65D8011C96ED91FC910F
:109210001282AF92BF9288E998E19F938F931F9338
:109220000F930F945D650FB6F894DEBF0FBECDBFF0
:10923000B12C8FE8C82E88E1D82E8B2D94E08902BE
:10924000F0011124A5E8B0E0AC0FBD1FEA0FFB1F31
:10925000808191810097A9F1228133812115310507
:10926000C9F33F932F939F938F93DF92CF921F93D6
:109270000F930F945D65B3940FB6F894DEBF0FBEE5
:10928000CDBFDBCF40E250E065E979E1C8010F9442
:10929000036467E779E18DE091E10F947735B801D8
:1092A0008DE091E10F9420358DE091E10F947834B9
:1092B0004DCEF70161897289A501C7010F94D74886
:1092C00075CF83ED98E19F938F931F930F930F9426
:1092D0005D65D70158961C921E925797D8011C962F
:1092E000ED91FC91C080D1800F900F900F900F9066
:1092F00043E3A42EB12CD601ED91FC910084F185BD
:10930000E02DC601199541975CF4B1E0AB1AB108A4
:1093100039F064E170E080E090E00F94E408EBCF76
:10932000D601ED91FC910084F185E02DC6011995DF
:10933000419734F4C8010F94B33D10E000E05AC0E7
:1093400062EF7BE0CE0183579F4F0F941832912C30
:10935000A12CD601ED91FC910688F789E02DC6017C
:1093600019958823E1F1BDE0AB1201C0A92CD6010B
:10937000ED91FC910688F789E02DC60119958111C0
:10938000BBC0D601ED91FC910084F185E02DC601B2
:109390001995892B09F4C2C0D601ED91FC91028484
:1093A000F385E02DC6011995B82EBAE08B1709F4A4
:1093B000B7C0EDE08E1709F4B3C0FFEF8F1709F4C3
:1093C000ADC0682FCE0183579F4F0F9404319A2C64
:1093D000AB2CBFCFBAE0BB12FACFAB12F8CFCC2484
:1093E000C394D12CCE0183579F4F0F94D931CD28F0
:1093F00009F4A3CFD7015796ED90FC906FE479E183
:109400008EEB91E10F947735B7018EEB91E10E94DD
:109410007BF68EEB91E10F94783464E670E080E0A7
:1094200090E00F94E4080115110509F461C1B8EC4E
:10943000EB16F10409F03AC163E479E18DE091E1C2
:109440000F94773564EF71E080E090E00F94E408CA
:10945000EF961FAE1EAEEF97C158DF4F19821882EC
:10946000CF57D0408FEF9FEFCF57DF4F998388833F
:10947000C158D0408FEA92E0ED969FAF8EAFED9746
:10948000CD57DF4F19830883C358D040F89490E03C
:1094900080E00E941E468111CAC067E379E187E13E
:1094A00091E10F94773587E191E10F947834C80109
:1094B0000F94B33D24EFE22EFF24F394CE018D569A
:1094C0009F4F0F94D931C701C856DF4F0FB6F8949C
:1094D000DEBF0FBECDBFDF91CF911F910F91FF90E7
:1094E000EF90DF90CF90BF90AF909F908F907F9044
:1094F0006F905F904F900895D601ED91FC9100849C
:10950000F185E02DC6011995892B09F03ACF64E663
:1095100070E080E090E00F94E40829CFBB24BA9477
:1095200062E676E081E291E10F942035BE01635757
:109530007F4F81E291E10F94693581E291E10F94CF
:10954000783466E878E1CE0185589F4F0F94E13179
:10955000BE0165587F4FCE0183579F4F0F94173040
:10956000982ECE0185589F4F0F94D931992079F1CB
:10957000CF56DF4F28813981C159D04049E050E0B2
:10958000BE0163577F4FCE0185589F4F0F942932FC
:10959000ED968EAD9FADED97412C512C3201009789
:1095A00019F00F947E632B014201CE0185589F4F25
:1095B0000F94D9314114510429F0D70158965C9287
:1095C0004E925797B40181E291E10E94BFFAF701F0
:1095D0008784908881149104D1F0CF56DF4F888121
:1095E0009981C159D040892B91F0BE0163577F4FBB
:1095F000CE0185589F4F0F940F32CE0185589F4F53
:10960000F4011995CE0185589F4F0F94D93162EF1F
:109610007BE0CE0183579F4F0F94A931FFEFBF121C
:10962000D9CEC8010F94B33DD12CC12CDBCECE01D5
:1096300085589F4F0F94C3029093530C8093520C04
:109640007894C8010F94B33D8091520C9091530CC3
:10965000892BD1F462EF7BE0CE0183579F4F0F94AB
:109660001832CE0183579F4F0F945413CE01835766
:109670009F4F0F94D93160E279E187E191E10F9436
:109680007735F12CE12C1ACF0E94A13A8091CC0CB5
:10969000882329F00E9402FA71FF0E942B1C69E1C5
:1096A00079E18DE091E10F94773508CFE0E3EE1694
:1096B000E1E0FE0651F465E079E18DE091E10F947F
:1096C0007735C8010F94B33DF9CE6DEE78E187E1AF
:1096D00091E10F947735C8010F94B33DB70187E14D
:1096E00091E10E947BF687E191E10F947834E6CE18
:1096F0006AED78E18EEB91E10F947735EE24EA94F0
:10970000FE2CDCCECF93DF93CDB7DEB72E970FB60E
:10971000F894DEBF0FBECDBF80913B13811121C1F4
:1097200080913B138F5F80933B1364E776E18DE07C
:1097300091E10F9477358DE091E10F947834109298
:1097400009111092081180E090E190930411809328
:10975000031184E890E090930B1180930A1181E04B
:109760008093051180E090E2909307118093061199
:1097700082E780930C1187EF90E10E9426B18B372E
:10978000910509F0C5C066E676E18EEB91E10F9494
:1097900077358EEB91E10F9478348091520C909153
:1097A000530C892B21F081E090E00E941E461C8220
:1097B0001B8285EC92E09A83898387EF90E19E83F8
:1097C0008D838FEF9FEF98878F83CE0101960F9443
:1097D000C3029093530C8093520C87EF90E10E9448
:1097E00040AF8091520C9091530C892B01F56AE5A2
:1097F00076E187E191E10F94773587E191E10F946C
:10980000783462EF7BE0CE0109960F941832CE01D6
:1098100009960F945413CE0109960F94D931809173
:109820003B13815080933B1390E080E019C067E4C4
:1098300076E18DE091E10F9477358DE091E10F9421
:10984000783480913B13815080933B130E94A13A5E
:109850008091E9109091EA10892B59F481E090E011
:109860002E960FB6F894DEBF0FBECDBFDF91CF911D
:1098700008950E94A3F7882389F382E70E948EF758
:109880008091E9109091EA10DC01ED91FC91008843
:10989000F189E02D60E670E019956091E910709112
:1098A000EA1040E0CE0109960F94F533BE01675FE0
:1098B0007F4F8BEE90E10F947730CE0109960F9495
:1098C000D9318091E9109091EA10DC01ED91FC9181
:1098D0000488F589E02D199569E276E18EEB91E136
:1098E0000F9477356BEE70E1CE0109960F940F322D
:1098F000BE01675F7F4F8EEB91E10F9469358EEB70
:1099000091E10F947834CE0109960F94D931A6CF06
:1099100087EF90E10E946BAE892BA1F087EF90E179
:109920000E9495AE62EF7BE0CE0101960F94183253
:10993000CE0101960F945413CE0101960F94D931A4
:109940000F94C31387EF90E10E9440AF66E376E186
:109950008DE091E10F9477358DE091E10F947834AB
:109960005ECF8FEF9FEF7CCF4F925F926F927F928F
:109970008F929F92AF92BF92CF92DF92EF92FF921F
:109980000F931F93CF93DF93CDB7DEB7CF52D14064
:109990000FB6F894DEBF0FBECDBF20913F133091BC
:1099A0004013F9017196E532F10508F041C68827A8
:1099B000E352F34B8F4F0D94966B2F5C1B5C185347
:1099C000185318531853775B635B18531853185385
:1099D000185318531853185318531853024D7854EA
:1099E0007F5458569F565E5A5B5B18531853185352
:1099F00018531853925BA45BDD5BBA5B1853185382
:109A00001853C75B8091CC0C0F94C74E029709F492
:109A10000FC681E195E0CC5DDE4F99838883C45207
:109A2000D140CA5DDE4F188219821A821B82C6524B
:109A3000D140C25EDE4F99838883CE51D140C05E53
:109A4000DE4F188219821A821B82C052D140C85E32
:109A5000DE4F99838883C851D140C65EDE4F18829D
:109A600019821A821B82CA51D140CE5EDE4F998381
:109A70008883C251D140CC5EDE4F188219821A828F
:109A80001B82C451D14064EB7DE08DE091E10F94E5
:109A900077358DE091E10F9478348091E9109091C1
:109AA000EA108E010F571F4F892B09F45CC00E94EA
:109AB000A3F7882309F457C082E70E948EF78091AC
:109AC000E9109091EA10DC01ED91FC910088F18998
:109AD000E02D60E170E01995BE016F5F7F4F8091CE
:109AE000E9109091EA100E9444F789819A81AB8134
:109AF000BC81CA5DDE4F88839983AA83BB83C6522B
:109B0000D1408091E9109091EA10DC01ED91FC9137
:109B10000488F589E02D1995CA5DDE4F8881C6520B
:109B2000D140882301F18F3FA9F4C95DDE4F8881C0
:109B3000C752D1408F3F71F4C85DDE4F8881C85253
:109B4000D1408F3F39F4C75DDE4F8881C952D14083
:109B50008F3F49F00E9402FA72FFA1C18091BF0CB1
:109B6000833008F09CC168EA7DE08DE091E10F94BC
:109B700077350FB6F894A89580916000886180933E
:109B80006000109260000FBE8091B40C81112AC059
:109B900010929C0C10929B0C88EE93E0A0E0B0E039
:109BA00080939D0C90939E0CA0939F0CB093A00C5F
:109BB00087EE94E090939A0C8093990C81E195E064
:109BC0009093A80C8093A70C1092A90C1092AA0C49
:109BD0001092AB0C1092AC0C88E08093B10C81E039
:109BE0008093B40C86E59CE09093BE0C8093BD0CF2
:109BF0000F949F41F12CE12C882309F4AEC080E53D
:109C000091E00F946B0246E050E061EF70E189E073
:109C100090E00F94543F81E195E09A8389831B8201
:109C20001C821D821E82CE0103960F9489410F94DF
:109C30009E418091BD0C9091BE0CFC0112A213A21A
:109C400014A215A2DC0116A217A210A611A612A634
:109C500013A614A615A640EE5EE260E070E046ABE7
:109C600057AB60AF71AF40EA5FE060E070E042AFD9
:109C700053AF64AF75AF189626E0FD01322F1192F5
:109C80003A95E9F7AC01425F5F4F34E1FA01119276
:109C90003A95E9F7E1EFF0E101900D922A95E1F7AD
:109CA000FC01EE5BFF4F10820F94E84B7C010197A3
:109CB00009F053C080E591E00F946B026091BD0CF8
:109CC0007091BE0C625F7F4FCE0101960F94B73545
:109CD000CE0103960F9489416091BD0C7091BE0C2A
:109CE0006A5E7F4FCE0101960F94B735CE01039681
:109CF0000F9497416091BD0C7091BE0C6E5E7F4FCA
:109D0000CE0101960F94B735CE0103960F94904182
:109D10000F949E416091BD0C7091BE0C625E7F4FAE
:109D2000CE0101960F94B7358B819C81AD81BE81A8
:109D30008093000F9093010FA093020FB093030F35
:109D40000F94CC077F7380910102909102026827E3
:109D50007927709302026093010288E199E20FB6BD
:109D6000F894A895809360000FBE90936000A8952A
:109D7000EF2809F4EAC26FEF7CE08DE091E10F94E7
:109D80007735CE0101960F94AB4E8B819C81AD81CE
:109D9000BE81CA5DDE4F88839983AA83BB83C65286
:109DA000D14051E1E52E55E0F52EFA82E982CE014F
:109DB00001960E94A06D8DE091E10F947834CE0160
:109DC0008C5D9E4F0E94AEF88091000F9091010F24
:109DD000A091020FB091030F8B839C83AD83BE8350
:109DE000C05EDE4F88839983AA83BB83C052D14073
:109DF000CE01825E9E4F0E9458F9FA82E9821B8250
:109E00001C821D821E8280E591E00F946B0244E06B
:109E100050E0BE016D5F7F4F81E090E00F94903E77
:109E20000F949E418B819C81AD81BE81C65EDE4FC9
:109E300088839983AA83BB83CA51D140CE01885EAF
:109E40009E4F0E94ADF9FA82E9821B821C821D821C
:109E50001E8280E591E00F946B0244E050E0BE0169
:109E60006D5F7F4F85E090E00F94903E0F949E4190
:109E70008B819C81AD81BE81CC5EDE4F88839983CE
:109E8000AA83BB83C451D140CE018E5E9E4F0E94F7
:109E900003F981E00E9497FA1092BF0CD7C162E9E2
:109EA0007DE08DE091E10F94773581E195E09A8333
:109EB0008983CA5DDE4F88819981AA81BB81C652A0
:109EC000D1408B839C83AD83BE83CE0101960E94DB
:109ED000A06D8091E9109091EA10892B09F420C2BD
:109EE0000E94A3F7882309F41BC282E70E948EF721
:109EF0008091E9109091EA10DC01ED91FC910088CD
:109F0000F189E02D64E170E01995BE016F5F7F4F2C
:109F10008091E9109091EA100E9444F789819A811A
:109F2000AB81BC81C05EDE4F88839983AA83BB83EB
:109F3000C052D1408091E9109091EA10DC01ED917E
:109F4000FC910488F589E02D1995C05EDE4F88816B
:109F5000C052D140882309F4E3C18F3FB1F4CF5DF3
:109F6000DE4F8881C152D1408F3F79F4CE5DDE4F04
:109F70008881C252D1408F3F41F4CD5DDE4F888150
:109F8000C352D1408F3F09F4CBC16CE87DE08DE036
:109F900091E10F94773581E195E09A838983C05EE2
:109FA000DE4F88819981AA81BB81C052D1408B83C9
:109FB0009C83AD83BE83CE0101960E94A06D8091EB
:109FC000E9109091EA10892B09F483C10E94A3F74C
:109FD000882309F47EC182E70E948EF78091E91000
:109FE0009091EA10DC01ED91FC910088F189E02D5F
:109FF00068E170E01995BE016F5F7F4F8091E910B5
:10A000009091EA100E9444F789819A81AB81BC81CA
:10A01000C65EDE4F88839983AA83BB83CA51D14031
:10A020008091E9109091EA10DC01ED91FC91048897
:10A03000F589E02D1995C65EDE4F8881CA51D14061
:10A04000882309F446C18F3FB1F4C55EDE4F888195
:10A05000CB51D1408F3F79F4C45EDE4F8881CC5123
:10A06000D1408F3F41F4C35EDE4F8881CD51D14056
:10A070008F3F09F42EC167E87DE08DE091E10F94F8
:10A08000773581E195E09A838983C65EDE4F8881CA
:10A090009981AA81BB81CA51D1408B839C83AD83B6
:10A0A000BE83CE0101960E94A06D8091E91090912F
:10A0B000EA10892B09F4CDC00E94A3F7882309F484
:10A0C000C8C082E70E948EF78091E9109091EA1053
:10A0D000DC01ED91FC910088F189E02D6CE170E0EC
:10A0E0001995BE016F5F7F4F8091E9109091EA1042
:10A0F0000E9444F789819A81AB81BC81CC5EDE4F9E
:10A1000088839983AA83BB83C451D1408091E9108D
:10A110009091EA10DC01ED91FC910488F589E02D25
:10A120001995CC5EDE4F8881C451D140882309F453
:10A1300090C08F3FB1F4CB5EDE4F8881C551D140D6
:10A140008F3F79F4CA5EDE4F8881C651D1408F3F80
:10A1500041F4C95EDE4F8881C751D1408F3F09F479
:10A1600078C060E87DE08DE091E10F94773561E1A2
:10A17000E62E65E0F62EFA82E982CC5EDE4F88811B
:10A180009981AA81BB81C451D1408B839C83AD83CB
:10A19000BE83CE0101960E94A06DFA82E982CC5E58
:10A1A000DE4F88819981AA81BB81C451D1408B83C4
:10A1B0009C83AD83BE83F801F182E082C65EDE4FF0
:10A1C00088819981AA81BB81CA51D14082839383BE
:10A1D000A483B583CE53DF4FF982E882C25CD040BE
:10A1E000C05EDE4F88819981AA81BB81C052D14077
:10A1F000CC53DF4F88839983AA83BB83C45CD04050
:10A20000CE5FDE4FF982E882C250D140CA5DDE4F98
:10A2100088819981AA81BB81C652D140CC5FDE4F33
:10A2200088839983AA83BB83C450D1409E012F5F4A
:10A230003F4FA801BE016E537F4FCE018E5F9E4FF0
:10A240000F942E038DE091E10F94783482E090E03A
:10A250008FC081E195E09A838983C65EDE4F488195
:10A2600059816A817B81CA51D1404B835C836D8364
:10A270007E83D8018D939C93C05EDE4F48815981C7
:10A280006A817B81C052D140F80142835383648349
:10A290007583CE53DF4F99838883C25CD040CA5DFB
:10A2A000DE4F88819981AA81BB81C652D140CC53AF
:10A2B000DF4F88839983AA83BB83C45CD040AE01FF
:10A2C0004F5F5F4FB801CE018E539F4F0F946D03C8
:10A2D000B9CF81E195E09A838983C05EDE4F4881E2
:10A2E00059816A817B81C052D1404B835C836D83ED
:10A2F0007E83D8018D939C93CA5DDE4F88819981BE
:10A30000AA81BB81C652D140F80182839383A48382
:10A31000B583BE016F5F7F4FC8010F94BF0392CF1B
:10A3200081E195E09A838983CA5DDE4F88819981B6
:10A33000AA81BB81C652D1408B839C83AD83BE83EF
:10A34000CE0101960F940A047DCF6EE37DE087E194
:10A3500091E10F9477356FE07DE087E191E10F9413
:10A3600077358091BF0C8F5F8093BF0C86EF9FEF96
:10A370009093401380933F1389E0E9E2F2E0D80123
:10A3800001900D928A95E1F787E1F8013996DF0196
:10A390001D928A95E9F785EF90E1009731F0A801C9
:10A3A000485F5F4F62E00F94D854CE018E539F4FA9
:10A3B0000F94AB4E0F941709683B7B4081059105C4
:10A3C00038F464E670E080E090E00F94E408F2CFA7
:10A3D000CC53DF4F88819981AA81BB81C45CD04076
:10A3E00080935F1090936010A0936110B0936210FF
:10A3F000C8010F94F302892BC9F0E0905B10F09034
:10A400005C10D701ED91FC91C088D18863E072E0C7
:10A41000CE0101960F94B73549EE54E1BE016F5F4E
:10A420007F4FC701F601199581113CC26EED7CE0AA
:10A4300087E191E10F94773587E191E10F947834CA
:10A440004FE6A42E40E1B42E7501D12CC12CD701CA
:10A450008D919C91892B49F1960143E050E060E099
:10A4600070E0CB010F943A14D701ED91FC918085F7
:10A470009185009711F00F942F62D701ED91FC9117
:10A4800086819781009711F00F942F62D701ED918B
:10A49000FC91848195810F942F62F70180819181D5
:10A4A0000F942F62D7011D921C92BFEFCB1ADB0ACB
:10A4B000E2E0EE0EF11CF8E0CF16D10441F686E0A2
:10A4C000E9E4F2E09E012F5F3F4F4901D90101907D
:10A4D0000D928A95E1F7FE0137968AE1DF011D9220
:10A4E0008A95E9F7AE014A5F5F4F8BE1FA0111925D
:10A4F0008A95E9F781EF90E1009719F066E00F94F3
:10A50000D85465E676E0C8010F94E16FD12CC12CD8
:10A51000D5018D919D915D01892B09F0CCC18AE017
:10A5200090E00F9493617C01009709F4C4C1FC0191
:10A53000178216821186108615821482D8010D901A
:10A540000020E9F7CD010197801B910B0F949361D7
:10A550005C01F70195838483892B11F40C949F5C33
:10A56000D4010D900020E9F7CD01019788199909D0
:10A570000F949361F70191878087009711F40C94F1
:10A580009C5CB4010F94007080E590E0D7011196B7
:10A590009C938E9313961C921E921297B801C5013C
:10A5A0000F940070F50101900020E9F73197AE1685
:10A5B000BF0620F4319781818E32C9F75F01B2E086
:10A5C000AB0EB11CF50101900020E9F7CF018A190B
:10A5D0009B090B960F9493614C01D70117969C939E
:10A5E0008E931697009741F0B5010F9400706CE6BA
:10A5F00076E0C4010F94E16FF601EE0FFF1FE15901
:10A60000FF4EF182E082960142E050E060E070E0AF
:10A61000CB010F943A14019709F456C168E776E02C
:10A6200087E191E10F94203587E191E10F9478342F
:10A630000FB6F894A89580916000886180936000BF
:10A64000109260000FBE80913F13909140130297CB
:10A650000CF401C18091BF0C81110C94625C0091DB
:10A66000BD0C1091BE0C0115110511F40C94625C27
:10A670000F9417094B015C017801FEE3EF0EF11C0A
:10A68000F70180819181A281B381A5019401281BEA
:10A69000390B4A0B5B0BCA01B901683E33E0730703
:10A6A00081059105B0F128EE33E040E050E00F94D1
:10A6B0000B6B861A970AA80AB90AD7018D929D9248
:10A6C000AD92BC921397F80186A597A5A0A9B1A950
:10A6D00069017A01CC0CDD1CEE1CFF1C8C159D055C
:10A6E000AE05BF0510F00C944A5C16A617A610AA7A
:10A6F00011AAF80182A993A9A4A9B5A98C159D0551
:10A70000AE05BF0510F00C94545C12AA13AA14AA4B
:10A7100015AAF80186A597A5A0A9B1A9892B8A2B0E
:10A720008B2B11F00C945E5CEE5BFF4F80818330CD
:10A7300011F00C945E5C84E08083C8010F94E84BB8
:10A7400001967C01F80182A993A9A4A9B5A9892B36
:10A750008A2B8B2BA1F4EE5BFF4F8081833011F0AD
:10A7600081110DC01082F8013E9684E1DF011D9237
:10A770008A95E9F7C8010F94E84B03967C01B2E093
:10A78000EB16F10429F0E4E0EE16F10409F046C0FE
:10A7900080E591E00F946B026091BD0C7091BE0C4E
:10A7A000625F7F4FCE0101960F94B735CE010396BD
:10A7B0000F9489416091BD0C7091BE0C6A5E7F4F11
:10A7C000CE0101960F94B735CE0103960F949741B1
:10A7D0006091BD0C7091BE0C6E5E7F4FCE010196F4
:10A7E0000F94B735CE0103960F9490410F949E417C
:10A7F0006091BD0C7091BE0C625E7F4FCE010196E0
:10A800000F94B7358B819C81AD81BE818093000F01
:10A810009093010FA093020FB093030F0F94C74EB4
:10A82000029711F40C94705CF3E0EF16F10411F44C
:10A830000C94855C14F00C94665C31E0E316F10432
:10A8400011F40C94825C64E270E142E0E416F104DD
:10A8500011F40C948A5C88E199E20FB6F894A895FB
:10A86000809360000FBE9093600020913F13309161
:10A870004013C901C15DDE4F0FB6F894DEBF0FBEB5
:10A88000CDBFDF91CF911F910F91FF90EF90DF909F
:10A89000CF90BF90AF909F908F907F906F905F9080
:10A8A0004F90089566EC7CE08DE091E10F94773550
:10A8B0008DE091E1C3CDBFEFCB1ADB0AE8E0CE1605
:10A8C000D10409F025CEAACE65EB7CE08DE091E1C4
:10A8D0000F947735B8018DE091E10F9420356EEA41
:10A8E0007CE08DE091E10F9477358DE091E19ECE93
:10A8F00082E090E09093401380933F1399CE809133
:10A9000046138111D2C10E94FB1E69E471E18EEBF6
:10A9100091E10F9477358EEB91E10F94783480912B
:10A92000E9109091EA10892B09F432C10E94A3F733
:10A93000882309F42DC182E70E948EF78091E910E7
:10A940009091EA10DC01ED91FC910088F189E02DF5
:10A9500060E570E019954FE050E0BE016F5F7F4FFA
:10A960008091E9109091EA100E94E8F78C018091A3
:10A97000E9109091EA10DC01ED91FC910488F589D1
:10A98000E02D19950115110509F402C1E1E0F0E08F
:10A99000EC0FFD1FE00FF11F1082BE016F5F7F4FB4
:10A9A0008EEB91E10F9420358EEB91E10F9478348A
:10A9B000CE01865D9E4F0F94AB4EC45DDE4F888105
:10A9C0009981AA81BB81CC52D1408093C8109093C9
:10A9D000C910A093CA10B093CB1069E976E088EB58
:10A9E00090E10F94A931BE016F5F7F4FCE01825E6F
:10A9F0009E4F0F9418326AE07EE0CE01885E9E4F33
:10AA00000F94E13169E976E0CE018E5F9E4F0F949D
:10AA10001832BE016E5F7E4FCE018E5E9E4F0F9448
:10AA20000F32BE01685E7E4FCE018E5E9E4F0F9448
:10AA30007531BE01625E7E4F0F9475318C0162EFFD
:10AA40007BE0CE018C5D9E4F0F941832F80184811B
:10AA50009581880F991F880F991F63E070E00F940C
:10AA60006E6BCE018C5D9E4F0F94B030F12CE12CBB
:10AA7000D80114968D919C91E816F90608F0B7C09C
:10AA8000B701C8010F940630E82F880FFF0BF5952A
:10AA9000E795F595E795EF73FF27EF53F24F649134
:10AAA000CE018C5D9E4F0F940431B701C8010F9405
:10AAB0000630B0E18B0250011124E0E3AE22BB244A
:10AAC0006701FFEFCF1ADF0AD80114968D919C9190
:10AAD000C816D90608F078C0B601C8010F94063030
:10AAE000E82F880FFF0BB4E0F595E795BA95E1F7ED
:10AAF000EF70FF27EA29FB29EF53F24F6491CE0153
:10AB00008C5D9E4F0F940431B601C8010F9406303E
:10AB1000B4E08B0250011124ECE3AE22BB246701A8
:10AB2000F2E0CF0ED11CD80114968D919C91C816DD
:10AB3000D90608F03EC0B601C8010F940630E82FD0
:10AB4000880FFF0BA6E0F595E795AA95E1F7E3706E
:10AB5000FF27EA29FB29EF53F24F6491CE018C5D68
:10AB60009E4F0F940431B601C8010F940630E82FB0
:10AB7000EF730E2E000CFF0BEF53F24F6491CE01DA
:10AB80008C5D9E4F0F940431B3E0EB0EF11C70CF3F
:10AB900065E57EE0CE0101960F94D5636DE17EE020
:10ABA00087E191E10F94773587E191E10F94783453
:10ABB000F4CEF501EF53F24F6491CE018C5D9E4FC0
:10ABC0000F9404316DE3DBCFF501EF53F24F649145
:10ABD000CE018C5D9E4F0F94043142E050E061EA5B
:10ABE00076E0CE018C5D9E4F0F94D830CDCF63E0E0
:10ABF0007EE0CE018F579F4F0F94E131BE016F571A
:10AC00007F4FCE018E539F4F0F940F32BE016C5D6C
:10AC10007E4FCE018E539F4F0F947531BC018EEB4A
:10AC200090E10F94C231CE018E539F4F0F94D931D2
:10AC3000CE018F579F4F0F94D931CE018C5D9E4F1F
:10AC40000F94D931CE018E5E9E4F0F94D931CE0133
:10AC50008E5F9E4F0F94D931CE01885E9E4F0F9428
:10AC6000D931CE01825E9E4F0F94D93189ED9EE09D
:10AC70009093C5108093C41087EF90E19093C71014
:10AC80008093C61084ED90E10F946C4D8EEF90E4AC
:10AC90009093D3108093D2106CE07EE08DE091E130
:10ACA0000F94773581E08093461383E090E022CEC5
:10ACB0008091CC0C80913B138111DBCD0E9402FA74
:10ACC00070FD2DC08091C40C81111EC00E944647AA
:10ACD000883C910519F484E090E00CCE8091CC0C76
:10ACE00062E271E1811112C0CE0101960F94AB4E68
:10ACF0008B819C81AD81BE81892B8A2B8B2B09F4A2
:10AD00003BC28FE090E0F6CD62E171E18DE091E130
:10AD10000F9477358DE091E10F947834DCCF8091FA
:10AD2000CC0C882349F084E090E09093401380930A
:10AD30003F1368ED70E1D5CD8FE090E0F6CFA89598
:10AD40008091CC0C8091C70C9091C80C009721F099
:10AD50000E9434F7823068F465EC70E18DE091E197
:10AD60000F9477358DE091E10F94783487E090E08F
:10AD7000C1CDC85EDE4F1882C851D140FE01EE5FE2
:10AD8000FE4F119211928EE0DF011D928A95E9F734
:10AD90000E9408F6882319F085E090E0ABCDE090A2
:10ADA000C70CF090C80CE114F10441F0C7010E94F7
:10ADB00034F7082F10E0023011055CF466E87FE0FC
:10ADC00087E191E10F94773587E191E10F94783431
:10ADD00098CF70E060E0C7010F94C655009709F462
:10ADE00089C09093DB0C8093DA0C69E77FE08DE0FB
:10ADF00091E10F9477356091DA0C7091DB0C8DE066
:10AE000091E10F9420358DE091E10F947834809199
:10AE1000DA0C9091DB0C0F94F302892B09F06DC0D2
:10AE200064EA76E087E191E10F94203587E191E1D2
:10AE30000F947834E090C70CF090C80C61E070E09B
:10AE4000C7010F94C6555C010230110509F46CC0AE
:10AE500062E0C7010E9462F6FC01C184D284033023
:10AE6000110509F46AC063E070E0C7010F94C6558C
:10AE70007C018091E9109091EA10892B09F462C05D
:10AE80000E94A3F7882309F45DC082E70E948EF731
:10AE90008091E9109091EA10DC01ED91FC9100881D
:10AEA000F189E02D60E470E019954FE050E0BE01BB
:10AEB0006E5F7E4F8091E9109091EA100E94E8F752
:10AEC0004C018091E9109091EA10DC01ED91FC9128
:10AED0000488F589E02D19958114910499F1E2E037
:10AEE000F1E0EC0FFD1FE80DF91D10828E010E5FE1
:10AEF0001E4F3EC080E792E074CF65E67FE08DE0B4
:10AF000091E10F9477356091DA0C7091DB0C8DE054
:10AF100091E10F9420356EE57FE08DE091E10F9493
:10AF200077358DE091E184CF7BE5C72E77E0D72E92
:10AF30009E01285E3E4F79019CCFAE01485E5E4F78
:10AF40007A0197CF053011058CF264E070E08091B2
:10AF5000C70C9091C80C0F94C6558C016EE37FE02E
:10AF60008DE091E10F9477358DE091E10F94783485
:10AF7000B092320FA092310FD092340FC092330FA3
:10AF80008AEB94E490932A0F8093290F40E150E0DC
:10AF900061E37FE0CE018E539F4F0F94036430E056
:10AFA00020E041E050E060E2CE018F579F4F0E94C9
:10AFB000916A40E250E063E975E3CE018F579F4FFD
:10AFC0000F94E56360E17FE08DE091E10F947735C8
:10AFD000B5018DE091E10F9420356EE07FE08DE0CA
:10AFE00091E10F947735B6018DE091E10E947BF6F7
:10AFF00067E07FE08DE091E10F947735B7018DE058
:10B0000091E10F94203562E07FE08DE091E10F94B3
:10B010007735F7018081811104C010E000E0F12C48
:10B02000E12CA090DA0CB090DB0C0E9408F68111A4
:10B03000C6C18091140F9091150FDC01ED91FC9128
:10B040000688F789E02D1995882309F498C081E0D6
:10B0500090E090931F0F80931E0F87E0E9E6F2E0E7
:10B06000DE01119601900D928A95E1F7FE0131966D
:10B0700085E090E02191A091160FB091170FA80FD5
:10B08000B91F2C9301968C309105A1F786E3E1144A
:10B09000F10429F086EB0115110509F086EFC09047
:10B0A000160FD090170FF601848780911B0F8587AC
:10B0B00080911A0F86878090180F9090190FB40115
:10B0C000C5010F94166441968816990608F08EC043
:10B0D0008091140F9091150FDC01ED91FC91048883
:10B0E000F589E02D19956FEB7EE087E191E10F94F2
:10B0F00077356091370F7091380F87E191E10E94A9
:10B100007BF667EA7EE087E191E10F94773587E18E
:10B1100091E10F9478348091C90C882379F0E09103
:10B12000C70CF091C80C828193819093C80C8093D6
:10B13000C70C892B09F0B4C10E94CA1B0F941709D0
:10B140006093C00C7093C10C8093C20C9093C30C9D
:10B150008091BC0C8F5F8093BC0C83330CF4ABC12B
:10B1600069E77EE087E191E10F94773587E191E12E
:10B170000F9478341092BC0C86EF9FEFBBCB60919C
:10B18000310F7091320F8091140F9091150FDC01E7
:10B19000ED91FC914091330F5091340F6115710581
:10B1A00071F00088F189E02D1995019709F44FCFCE
:10B1B0008EEF9FEF9093380F8093370F94CF0684D4
:10B1C000F785E02D21E135E03A83298340902D0F6A
:10B1D00050902E0F60902F0F7090300F4B825C823A
:10B1E0006D827E82BE016F5F7F4FDECF4FE050E009
:10B1F000B601C5010E9440F66C01A090180FB090F6
:10B20000190FB501CE018F579F4F0F9416648C0D07
:10B210009D1D0296A816B90608F45ACF6091160F24
:10B220007091170FA601CE018F579F4F0E9440F6D5
:10B230006C01A090180FB090190FB501CE018E537C
:10B240009F4F0F9416648C0D9D1D0296A816B9068B
:10B2500008F43ECF6091160F7091170FA601CE0132
:10B260008E539F4F0E9440F66C01E114F104B9F136
:10B27000A090180FB090190FB501C7010F94166474
:10B2800096012E5F3F4F820F931FA816B90608F450
:10B290001FCF6091160F7091170FA601C7010E9472
:10B2A00040F66C0101151105D1F0E090180FF090F7
:10B2B000190FB701C8010F94166496012E5F3F4F16
:10B2C000820F931FE816F90608F402CF6091160F5B
:10B2D0007091170FA601C8010E9440F66C01A601EB
:10B2E000455051096091160F7091170F80E10F942E
:10B2F00023090F9417096093200F7093210F8093F7
:10B30000220F9093230F6093240F7093250F809347
:10B31000260F9093270F8091140F9091150FDC0149
:10B32000ED91FC910084F185E02D1995892B21F593
:10B330000F9417090091240F1091250F2091260FCB
:10B340003091270F6B017C01C01AD10AE20AF30A7F
:10B3500020911C0F30911D0FA8EEB3E00F945F6B8E
:10B36000C616D706E806F906B0F28CEF9FEF909369
:10B37000380F8093370FACCECE018E5E9E4F0F9468
:10B38000CA0D643071058105910509F0A1CEE091E7
:10B39000160FF091170F838190E08111E8CF0F9481
:10B3A00017096093240F7093250F8093260F9093B5
:10B3B000270F1092280F1092380F1092370F10920B
:10B3C000BC0C64EF7EE08DE091E10F9477356091E5
:10B3D000DA0C7091DB0C8DE091E10F9420358DE05B
:10B3E00091E10F94783481E08093C40C30E020E048
:10B3F00043E050E061E4CE0101960E94916A6EEB59
:10B4000076E0CE0101960F94E16FCE0101960F9484
:10B410001E0A30E020E042E050E061E4CE010196F7
:10B420000E94916A62EC76E0CE0101960F94E16F82
:10B43000BE016F5F7F4F8EEB91E10F947C34CE01A4
:10B4400001960F941E0A30E020E041E050E061E4F4
:10B45000CE0101960E94916A62EC76E0CE010196DF
:10B460000F94E16FBE016F5F7F4F8EEB91E10F9400
:10B470007C34CE0101960F941E0A85E090E09093F3
:10B48000401380933F130F9417096093C00C70937F
:10B49000C10C8093C20C9093C30C61ED7EE021CA75
:10B4A0006EE57EE08DE091E10F9477358DE091E1DE
:10B4B0000F94783443CE8CE090E01CCA0F941709A7
:10B4C0000091C00C1091C10C2091C20C3091C30CA2
:10B4D000601B710B820B930B60347F4181059105DA
:10B4E00008F4A6C830E020E043E050E061E4CE017B
:10B4F0008F579F4F0E94916A6EEB76E0CE018F5777
:10B500009F4F0F94E16F0091180F1091190FB80120
:10B51000CE018F579F4F0F9416640996081719078D
:10B5200090F10E9408F6882371F180911E0F90918E
:10B530001F0F019609F4BCC090931F0F80931E0F3C
:10B54000E091160FF091170F80911F0F8583E09106
:10B55000160FF091170F80911E0F86836091160FC2
:10B560007091170F47E050E0CE018F579F4F0E9418
:10B5700040F6AC01455051096091160F7091170FBC
:10B5800082EA0F942309FE01EE53FF4F11921192AC
:10B590008EE3DF011D928A95E9F71A821982FE0176
:10B5A00033968EE7DF011D928A95E9F730E020E0BF
:10B5B00041E050E060E4CE018E539F4F0E94916ABB
:10B5C0004FE350E063E975E3CE018E539F4F0F9434
:10B5D000E5634FE750E06DE875E3CE0101960F9407
:10B5E000036441E0BE016F5F7F4FCE018E539F4FDA
:10B5F0000F94E50930E020E041E050E060E4CE0146
:10B600008E539F4F0E94916A4FE350E06FEE7FE0B0
:10B61000CE018E539F4F0F94E5634FE750E065EEE8
:10B620007FE0CE0101960F9403644FE750E062ED96
:10B630007FE0CE0101960F94E56341E0BE016F5FAC
:10B640007F4FCE018E539F4F0F94E50930E020E0ED
:10B6500041E050E060E4CE018E539F4F0E94916A1A
:10B660004FE350E06AEA75E3CE018E539F4F0F948B
:10B67000E5634FE750E062EC7FE0CE0101960F9466
:10B68000036441E0BE016F5F7F4FCE018E539F4F39
:10B690000F94E50986E090E09093401380933F1368
:10B6A00068EA70E18DE091E10F9477350C941853BE
:10B6B00081E090E041CF8091CC0C0E9408F681118E
:10B6C0000C94185308CB0F9417096093C00C709317
:10B6D000C10C8093C20C9093C30C85EF9FEF9093A5
:10B6E000401380933F138091CC0C0C9418530F940B
:10B6F00017090091C00C1091C10C2091C20C30911F
:10B70000C30C601B710B820B930B6838734181056E
:10B71000910510F40C9418531092401310923F139B
:10B720000C9418530E9408F681110F94B4100F94D2
:10B7300017096093C00C7093C10C8093C20C909356
:10B74000C30C8DE090E0D6C80F9417090091C00C8F
:10B750001091C10C2091C20C3091C30C601B710B75
:10B76000820B930B603177428105910508F0B3CAD3
:10B770000C9418530F9417096093C00C7093C10C6C
:10B780008093C20C9093C30C8EE090E0B3C80F94EA
:10B7900017090091C00C1091C10C2091C20C30917E
:10B7A000C30C601B710B820B930B603C744D81408A
:10B7B000910508F0E1CC0C9418530E94824B00973D
:10B7C00041F18130910509F486CA019611F00C947B
:10B7D00018530F9417090091C00C1091C10C2091BF
:10B7E000C20C3091C30C601B710B820B930B603346
:10B7F00075478105910510F40C94185365E870E1C4
:10B8000087E191E10F947735F0E0E0E019950C9431
:10B81000185383E190E09093401380933F130F946B
:10B8200017096093C00C7093C10C8093C20C909365
:10B83000C30C0C9418530E9408F681110F94B41095
:10B840000E94CA1B0F9417096093C00C7093C10C1F
:10B850008093C20C9093C30C8FEE9FEF4BC88091E6
:10B86000CC0C80913B1381110C94395482E190E00F
:10B870009093401380933F130E944647883C910564
:10B8800009F429CA8091CC0C882309F42DCA6EE5ED
:10B8900070E13CCA821B930BA40BB50B86A797A73C
:10B8A000A0ABB1AB0C947953821B930BA40BB50BDB
:10B8B00082AB93ABA4ABB5AB0C948953F12CE12CC8
:10B8C0000C94A253F12CE12C0C940E5454E0E51688
:10B8D000F104F1F085E0E816F10411F00C942B541A
:10B8E00065E570E187E191E10F94773587E191E1BA
:10B8F0000F94783486EF9FEF9093401380933F131B
:10B900000C942B5461E470E1EDCF61E170E1EACF7A
:10B9100065EF7FE08DE091E10F947735CE010196E0
:10B920000F94AB4ECE0101960E94A06D8DE091E187
:10B930000F9478340C942B54C5010F942F62D701C7
:10B9400018968D919C91009711F00F942F62C7016A
:10B950000F942F620C940E53A8950F94B03B82E085
:10B9600090E00E9493200E94B44C039734F00F940F
:10B970001B0F0F948C230F942D170C94FBED90E06C
:10B9800080E00895DC01ED91FC910284F385E02DC7
:10B990001994DF92EF92FF920F931F93CF93DF934F
:10B9A000EC010C891D890115110559F01D8A1C8AAD
:10B9B000C801DF91CF911F910F91FF90EF90DF9021
:10B9C0000895EC85FD858E859F85DF01A80FB91F41
:10B9D0002C91243209F055C011962C912B3709F087
:10B9E00050C00296E80FF91FF12CE12CDF01D19035
:10B9F000DD2009F446C08DE7D816E9F08FEFE81A8C
:10BA0000F80AF4CF198A188A2C853D85211531054D
:10BA100079F08E859F85280F391FF9012081222317
:10BA200021F001969F878E873EC01D861C86C0CF61
:10BA30000FEF1FEFBDCFE114F10419F11C928E85B9
:10BA40009F8502966C857D85680F791FE881F98155
:10BA50000684F785E02DCE011995998B888B1B8A7A
:10BA60001A8AEC85FD858E859F85E80FF91FEE0DFE
:10BA7000FF1DD2828E859F850396E80EF91EFF86F4
:10BA8000EE86288939892115310509F4BDCF8A89C7
:10BA90009B89280F391FF9012081222309F4B2CF95
:10BAA00001969B8B8A8B022F220F110B81CFDC0119
:10BAB0001C96ED91FC911D971E968D919C91E80F1F
:10BAC000F91F8081082E000C990B0895DC01159652
:10BAD0008D919C91009739F0DC01ED91FC910680ED
:10BAE000F781E02D1994089583E090E00895DC013A
:10BAF0001296ED91FC9113973097B9F016968D91AF
:10BB00009C918430910541F08530910541F0039777
:10BB100049F482E090E0089581E090E0089581E1A9
:10BB200090E00895828590E0089590E080E0089587
:10BB300085E090E008951F93CF93DF930097A1F0E5
:10BB4000FC011085212F2F70223071F4EC016185EA
:10BB50007285838594850F94C86969877A878B87F6
:10BB60009C87107F13601887DF91CF911F910895F4
:10BB70008EE090E008950D942F620D942F620D9445
:10BB80002F620D942F62EF92FF920F931F93CF932A
:10BB9000DF938C0161E071E28EEB91E10F947735D8
:10BBA0008EEB91E10F947834D8011496ED91FC91CD
:10BBB000309749F1C681D781209729F1E881F98131
:10BBC0003097E9F080818823D1F064EC76E0CE01F3
:10BBD0000E94EAF57C01009791F0FC018185928535
:10BBE000A385B4850097A105B10549F00F942F6294
:10BBF000D70119961D921D921D921C921C970A80C6
:10BC0000DB81C02DD9CFD801ED91FC910484F5855D
:10BC1000E02D60E0C801199581E090E0DF91CF91BF
:10BC20001F910F91FF90EF9008950D942F620D9446
:10BC30002F62EF92FF920F931F93CF93DF93EC014C
:10BC40008B018091DC0C9091DD0C0097A9F0FC0138
:10BC500020852F70263081F40E94EAF5FC01908542
:10BC60009F70943049F481859285DF91CF911F9127
:10BC70000F91FF90EF900895EE88FF88C70101971C
:10BC80000D97D0F468EC76E0C8010F94F76F892B1C
:10BC900099F48FE2888F85E08E9DB0018F9D700DA5
:10BCA00011246F507A4D46E050E0CE0149960F9432
:10BCB0000364CE014896D9CF90E080E0D6CF3F9282
:10BCC0004F925F926F927F928F929F92AF92BF92AC
:10BCD000CF92DF92EF92FF920F931F93CF93DF9358
:10BCE00000D000D0CDB7DEB77C01362E8091D90CC4
:10BCF000882309F40AC1D70114969C9180911D02F2
:10BD0000891708F402C180913B0D90913C0DBAE077
:10BD10006B1312C28A51934FFC011082D7011896FF
:10BD20008D919C91892B09F4ECC08091E20C90914B
:10BD3000E30CA091E40CB091E50C892B8A2B8B2BA2
:10BD400009F0CBC00F9417092B013C01F7010085C6
:10BD50001185D80119966D917C916115710599F441
:10BD6000F80185809680A780B0848091FA0E90912A
:10BD7000FB0EA091FC0EB091FD0E88169906AA0646
:10BD8000BB0609F484C0D8011B964D915C911C97A9
:10BD90004115510509F47BC0F701248153968C911C
:10BDA000539790E0322F377002C0959587953A955A
:10BDB000E2F780FF6CC0C22ED12CC601887F937041
:10BDC000892B39F451968D919C91887F9370C82A64
:10BDD000D92AD8018D919C91DC01ED91FC916115DE
:10BDE000710509F4C1C00688F789E02D19950197FE
:10BDF00009F04DC06CE3F801808191810F94933478
:10BE0000B601D8018D919C910E94EFFAF801228130
:10BE10008081918163EA75E2222311F061EA75E283
:10BE20000F947735D8011D966D917C911E978D9159
:10BE30009C910F94203560E2F801808191810F94EC
:10BE40009334D8011F966D917C9150978D919C9160
:10BE50000F942035F80122818081918166E975E295
:10BE6000222311F060E975E20F94773566EE7CE0ED
:10BE7000D8018D919C910F942035F801808191819A
:10BE8000DC01ED91FC91008CF18DE02D19950F9462
:10BE90001709AB01BC014419550966097709F70177
:10BEA00085819681453651056105710508F472C09A
:10BEB000009721F060EE75E20F949B354FEF5FEF36
:10BEC000BA0180E00F9452566093E20C7093E30C39
:10BED0008093E40C9093E50C14C00F941709009123
:10BEE000E20C1091E30C2091E40C3091E50C601B06
:10BEF000710B820B930B603375478105910508F038
:10BF000021CF10923C0D10923B0DD70115968D91CB
:10BF10009C911697009771F014963C9120911E0207
:10BF2000231740F0DC01ED91FC910190F081E02DB0
:10BF3000632D199581E090E026960FB6F894DEBF48
:10BF40000FBECDBFDF91CF911F910F91FF90EF906A
:10BF5000DF90CF90BF90AF909F908F907F906F9029
:10BF60005F904F903F9008950488F589E02D21E17E
:10BF700035E03A832983D80115968D909D90AD9038
:10BF8000BC9018978B829C82AD82BE82BE016F5F8F
:10BF90007F4F2CCF4091E20C5091E30C6091E40C68
:10BFA0007091E50C452B462B472B09F4AACF00973F
:10BFB00021F061ED75E20F949B351092E20C109226
:10BFC000E30C1092E40C1092E50CD70118960D9139
:10BFD0001C91F801618572856115710591F44580A8
:10BFE0005680678070848091FA0E9091FB0EA0912C
:10BFF000FC0EB091FD0E481659066A067B0609F440
:10C0000080CFD8011B964D915C911C97411551052D
:10C0100009F477CFF701248153968C91539790E0E0
:10C02000322F377002C0959587953A95E2F780FFD9
:10C0300068CFC22ED12CC601887F9370892B39F42A
:10C0400051968D919C91887F9370C82AD92AD801E6
:10C050008D919C91DC01ED91FC916115710509F4C4
:10C0600055C00688F789E02D1995019709F049CF49
:10C070006CE3F801808191810F949334B601D8016B
:10C080008D919C910E94EFFAF8012281808191812B
:10C090006CEB75E2222311F06AEB75E20F947735B1
:10C0A000D8011D966D917C911E978D919C910F9456
:10C0B000203560E2F801808191810F949334D8019A
:10C0C0001F966D917C9150978D919C910F94203586
:10C0D000F8012281808191816FEA75E2222311F0BB
:10C0E00069EA75E20F94773562EC75E2D8018D91BB
:10C0F0009C910F947735F80180819181DC01ED915D
:10C10000FC91008CF18DE02D1995FBCE0488F5890A
:10C11000E02D21E135E03A832983D80115964D9031
:10C120005D906D907C9018974B825C826D827E82D0
:10C13000BE016F5F7F4F98CF843591050CF0E5CE3F
:10C14000BDE06B1709F4E1CE9C012F5F3F4F3093A8
:10C150003C0D20933B0D8A51934FFC016083D5CE5B
:10C16000FC01828193810E949BBC21E030E08230FF
:10C1700011F430E020E0C9010895CF93DF93EC0182
:10C1800060E075E28EEB91E10F94773564EF74E235
:10C190008EEB91E10F9477356C817D818EEB91E18F
:10C1A0000E947BF66EEE74E28EEB91E10F94773590
:10C1B0008EEB91E10F94783460E08C810F949C06B3
:10C1C000E881F9810484F585E02D60E0CE011995C0
:10C1D00081E090E0DF91CF910895CF93DF93EC0160
:10C1E00067EC74E28EEB91E10F9477356C817D8181
:10C1F0008EEB91E10E947BF665EC74E28EEB91E1AF
:10C200000F947735EA81FB810280F381E02D608114
:10C2100071818EEB91E10F9420356FEB74E28EEB20
:10C2200091E10F9477358EEB91E10F947834E881AA
:10C23000F981008CF18DE02DCE01199581309105A9
:10C2400029F0029759F060E08C811AC063E070E039
:10C25000CE010E94A2EF60E00F949C0660E08C810A
:10C260000F949C0661E070E0CE010E94A2EF60E0B6
:10C270000F949C0662E070E0CE010E94A2EF60E0A5
:10C280000F949C06E881F9810484F585E02D60E037
:10C29000CE01199581E090E0DF91CF910895AF92A2
:10C2A000BF92CF92DF92EF92FF920F931F93CF93A3
:10C2B000DF93CDB7DEB768970FB6F894DEBF0FBE39
:10C2C000CDBFFC01098B1A8B2B8B3C8B4D8B5E8B6E
:10C2D0006F8B788F82819381009709F49DC02481B0
:10C2E0003581232B09F498C0CC2009F495C06F0147
:10C2F00070E060E00E945CB5192FD601ED91FC91D1
:10C30000008CF18DE02DC60119955C0182309105FC
:10C3100009F476C0039709F445C095E0F1E0AF1643
:10C32000B10409F091E019861A861B861C861D86C9
:10C330001E861F86188A8A85807F892B8A87EE242D
:10C34000EA94FE2C09891A892B893C894D895E89DA
:10C350006F89788DCE0109960E944530F1E0AF16C5
:10C36000B10409F44FC082E0A816B10409F045C039
:10C370006F8570E0D60114968C910F94D80661E019
:10C3800070E0C6010E94A2EF6E8570E00F94D8069F
:10C3900062E070E0C6010E94A2EF6D8570E00F942C
:10C3A000D8062BC0612F661F6627661FCE014196F7
:10C3B0000E9414285C01BC01D60114968C910F9444
:10C3C000D80663ED74E28EEB91E10F947735F601B8
:10C3D000648175818EEB91E10E947BF661ED74E2E0
:10C3E0008EEB91E10F947735B5018EEB91E10E94D0
:10C3F0007BF68EEB91E10F94783481E090E00EC0F3
:10C4000094E091CF63E070E0C6010E94A2EF6889DA
:10C4100070E00F94D806ACCF90E080E068960FB63D
:10C42000F894DEBF0FBECDBFDF91CF911F910F916A
:10C43000FF90EF90DF90CF90BF90AF900895CF9294
:10C44000DF92FF920F931F93CF93DF9300D000D022
:10C450001F921F92CDB7DEB76C01F02E1A83022F08
:10C4600010E0FF2029F00115110511F401E010E0A2
:10C4700040E050E061E070E0F601828193810E942B
:10C480002FB601301105A9F10230110541F0012B41
:10C49000B1F56DEB70E28EEB91E10F9477358A8107
:10C4A0008F70B9F1F60102811381C8010E94D0B4E6
:10C4B000672B682B692B89F401E010E0C8012896EE
:10C4C0000FB6F894DEBF0FBECDBFDF91CF911F91A5
:10C4D0000F91FF90DF90CF9008954FEF5FEFBA017B
:10C4E00080E00F945256AB01BC01C8010E948FB48A
:10C4F000E3CFF1E0FF1681F082E0F81669F061EB1E
:10C5000070E28EEB91E10F9477358EEB91E10F9411
:10C51000783410E000E0D2CFF601C280D380C601AB
:10C520000E94D0B4672B682B692B31F24FEF5FEF7D
:10C53000BA0180E00F945256AB01BC01C6010E94C3
:10C540008FB4BCCFCF92DF92EF92FF920F931F93E5
:10C55000CF93DC011296ED91FC9160E0848195818E
:10C560000E9462F68C01009729F0FC0180858F7093
:10C570008530D1F060E174E287E191E10F94773585
:10C5800087E191E10F947834C12CD12C90E8E92E09
:10C590009FEBF92EC701B601CF911F910F91FF902C
:10C5A000EF90DF90CF900895C8010E9434F781305A
:10C5B00040F18630A8F1893020F565E0C8010E947D
:10C5C00062F6FC0190859F709330F9F4C184D284A7
:10C5D000E384F484C1E060E0C8010E9462F6FC01DB
:10C5E00090859F70933009F5618572858385948568
:10C5F00020E030E0A9010F94C16987FF1FC0C1117D
:10C60000C9CFC12CD12C7601C5CF923049F46185B8
:10C610007285838594850F94C8696B017C01DACF9C
:10C62000C0E0C12CD12C7601D6CF923039F461858F
:10C630007285838594850F94C869DACFC111AACF1A
:10C64000C12CD12C8FE7E82E83E4F82EA3CFCF9313
:10C65000DF93EC016EED73E28EEB91E10F94773591
:10C66000EA81FB810280F381E02D608171818EEB94
:10C6700091E10F947C34EC81FD81309721F0808131
:10C6800091810F942F628C819D810F942F6270E0B5
:10C6900060E08A819B810E944CB41D821C8281E0F3
:10C6A00090E0DF91CF910895CF93DF93EC016CEC94
:10C6B00076E08EEB91E10F947C3440E050E0BA01DB
:10C6C0008A819B810E948FB4E881F9810484F58579
:10C6D000E02D60E0CE0119956D858C810F946E067A
:10C6E0006D858D810F946E0681E090E0DF91CF9192
:10C6F0000895CF93DF93EC016BED76E08EEB91E143
:10C700000F942035EA81FB810280F381E02D608166
:10C7100071818EEB91E10F947C348C819D81009727
:10C7200011F00F942F6270E060E08A819B810E947B
:10C730004CB41D821C8281E090E0DF91CF9108957E
:10C74000CF93DF93DC011496ED91FC91309741F18A
:10C75000C681D781209721F1E881F9813097E1F0F6
:10C7600080818823C9F020E030E0A9016BED77E0FB
:10C77000CE010F949155603171054CF46E30710506
:10C780001CF46130710541F481E090E00BC063510D
:10C79000710964307105C0F30A80DB81C02DDACFE6
:10C7A00090E080E0DF91CF9108951F93CF93DF93C6
:10C7B000142F0F940155EC01892BF9F08885982FDF
:10C7C0009F70923039F0933071F0911116C0807FD4
:10C7D00082608887412F50E070E060E049875A8787
:10C7E0006B877C870AC0612F70E090E080E00F9437
:10C7F000C66969877A878B879C87CE01DF91CF9145
:10C800001F910895CF92DF92EF92FF92CF93DF9323
:10C8100069017A010F940155EC01892BC9F08885D3
:10C82000982F9F70923039F0933051F0911110C0D1
:10C83000807F82608887C986DA86EB86FC8608C09E
:10C84000C701B6010F94C86969877A878B879C876F
:10C85000CE01DF91CF91FF90EF90DF90CF900895C0
:10C86000CF92DF92EF92FF92CF93DF9369017A012B
:10C870000F940155EC01892BC9F08885982F9F7082
:10C88000923039F0933071F0911110C0807F826046
:10C890008887C701B6010F94936C69877A878B8765
:10C8A0009C8704C0C986DA86EB86FC86CE01DF91C0
:10C8B000CF91FF90EF90DF90CF9008950F931F934B
:10C8C000CF93DF938A010F940155EC01892BF9F086
:10C8D0008885982F9F70923039F0933071F09111C4
:10C8E00016C0807F82608887012E000C220B330BDC
:10C8F00009871A872B873C870AC0B801110F880B5C
:10C90000990B0F94C86969877A878B879C87CE01BA
:10C91000DF91CF911F910F910895CF92DF92EF9207
:10C92000FF920F931F93CF93DF93009701F1DC01E8
:10C930001896EC91EF70E630D1F469017A018B0121
:10C94000EC010E94EAF50097A1F4A7019601B80155
:10C95000CE010F944702B801CE01DF91CF911F9114
:10C960000F91FF90EF90DF90CF900C94EAF590E05C
:10C9700080E0DF91CF911F910F91FF90EF90DF90BA
:10C98000CF900895CF92DF92EF92FF920F931F9373
:10C99000CF93DF93009701F1DC011896EC91EF70D3
:10C9A000E630D1F469017A018B01EC010E94EAF5CD
:10C9B0000097A1F4A7019601B801CE010F942302BC
:10C9C000B801CE01DF91CF911F910F91FF90EF90B1
:10C9D000DF90CF900C94EAF590E080E0DF91CF916A
:10C9E0001F910F91FF90EF90DF90CF9008952F92BD
:10C9F0003F924F925F926F927F928F929F92AF92EF
:10CA0000BF92EF92FF920F931F93CF93DF93CDB717
:10CA1000DEB72C970FB6F894DEBF0FBECDBF6130E6
:10CA2000710509F463C18C01FC01E280F38040E0F0
:10CA300050E061E070E0C7010E9458B6672B682B98
:10CA4000692B09F453C140E050E062E070E0C70197
:10CA50000E9458B6672B682B692B89F480910002DD
:10CA6000882309F443C140E050E062E070E0C70170
:10CA70000E942FB680910002815080930002F8013D
:10CA8000E280F380C7010E94D0B44B015C0119829F
:10CA90001A821B821C821D821E821F8218868A8136
:10CAA000807F8A8340E050E2B701CE0101960E9468
:10CAB000512760E0CE0101960E9414287C01F80104
:10CAC000828193810E949BBC823011F0853011F4E9
:10CAD000F12CE12CF80186819AEC980F903108F046
:10CAE000B7C121853285A90170E060E049875A8786
:10CAF0006B877C8743845484712C612C0F94AF071F
:10CB00009C01990F440B550B241935094609570907
:10CB1000AFEFB0E00F944C6B29853A854B855C856F
:10CB200024193509460957090F942D6B390137FD32
:10CB3000B9C15FEF6516710411F00CF0B6C1811434
:10CB40009104A104B10409F08BC1E618F70856EF6F
:10CB5000E5165FEFF5060CF0F6C0F80165858581F6
:10CB60000F946E06F801A280B380C5010E94D0B474
:10CB7000672B682B692B59F44FEF5FEFBA0180E008
:10CB80000F945256AB01BC01C5010E948FB4F8014D
:10CB9000B48065858EEF8B0D8C3028F084ED8B0D85
:10CBA000833008F070C0AA27BB27AE19BF096623DF
:10CBB00009F45CC09D01A1E0BFEF0F94A56B29E1D2
:10CBC00030E040E050E00F942D6BBA01A9014150D4
:10CBD0005F4F6F4F7F4F942F852F692F782F6F3FB7
:10CBE000710519F014F06FEF70E06634710514F4FC
:10CBF00066E470E08B2D78C062EA70E28EEB91E122
:10CC00000F9477358EEB91E10F9478346AEE76E0ED
:10CC10008EEB91E10F947C34F801658584810F944B
:10CC20006E06F801658585810F946E0640E050E040
:10CC3000BA01F801828193810E948FB440E050E0F4
:10CC400061E070E0F801828193810E9406B640E0C5
:10CC500050E062E070E0F801828193810E9406B6A4
:10CC6000809100028F5F8093000240C02FEF30E080
:10CC70000F94AD6B29E130E040E050E00F942D6B54
:10CC8000922F832FAACF858191E069279EEF980F7D
:10CC90009C3020F08C52833008F0D6C08B2D0F943E
:10CCA0006E06AA27BB27AE19BF09F8018585882320
:10CCB000B1F12FEF30E00F94AD6B29E130E040E0AF
:10CCC00050E00F942D6B922F832F692F782F6F3F99
:10CCD000710519F014F06FEF70E06634710514F40B
:10CCE00066E470E0F80185810F94D80690E080E05A
:10CCF0002C960FB6F894DEBF0FBECDBFDF91CF915B
:10CD00001F910F91FF90EF90BF90AF909F908F90E9
:10CD10007F906F905F904F903F902F9008959D016E
:10CD2000A1E0BFEF0F94A56B29E130E040E050E0B7
:10CD30000F942D6BBA01A90141505F4F6F4F7F4F88
:10CD4000942F852FC2CFFBE0EF16F1040CF45ECFD9
:10CD5000F801658584810F946E06F801A280B38086
:10CD6000C5010E94D0B4672B682B692B59F44FEF93
:10CD70005FEFBA0180E00F945256AB01BC01C501D0
:10CD80000E948FB4F801B58065858EEF8B0D8C30D5
:10CD900020F084ED8B0D8330B0F4662351F09701C1
:10CDA000A1E0BFEF0F94A56B23E330E040E050E03B
:10CDB0000ACF2FEF30E0D7010F94AD6B23E330E0C3
:10CDC00040E050E05BCF848191E069279EEF980FAF
:10CDD0009C3018F08C528330B8F58B2D0F946E0672
:10CDE000F80185858823E1F02FEF30E0D7010F941B
:10CDF000AD6B29E130E040E050E00F942D6B922FB5
:10CE0000832F692F782F77FF02C070E060E06F3FBB
:10CE1000710519F014F06FEF70E0F801848164CFB0
:10CE20009701A1E0BFEF0F94A56B29E130E040E04E
:10CE300050E00F942D6BBA01A90141505F4F6F4F25
:10CE40007F4F942F852FDDCF8B2D0F946E064ECF05
:10CE500066246A94762C81149104A104B104F1F043
:10CE6000F80127803084032C000C440855080F94E7
:10CE70001709211431044104510409F4BDCE681985
:10CE800079098A099B09621573058405950508F0DF
:10CE9000B3CEFFEF6F167F0609F057CE4FE7E41AC7
:10CEA000F10855CE712C612C4ACE66246A94712CFF
:10CEB00046CE5F926F927F928F929F92AF92BF9277
:10CEC000CF92DF92EF92FF920F931F93CF93DF9356
:10CED000CDB7DEB760970FB6F894DEBF0FBECDBFFB
:10CEE000E986FA860B871C872D873E874F87588BEC
:10CEF0006115710511F0011103C090E080E0D7C009
:10CF00004B018C01DB01AD90BC9019821A821B820F
:10CF10001C821D821E821F8218868A81807F8A83DE
:10CF200068EF76E0C4010E94EAF56C016FEE75E0EF
:10CF3000C4010E94EAF57C016DEF76E0C4010E9415
:10CF4000EAF54C01C114D10471F1F60180858F70AE
:10CF5000843049F5818592850E943020782EF9E051
:10CF60008F17D1F1F8173CF081E07816F4F4C12C5A
:10CF7000D12C76016AC0AAE08A13F9CFB701CE019D
:10CF800009960E946F2C29833A834B835C836D83BF
:10CF90007E838F8398873F7009F4AFCFCE010196CF
:10CFA0000E94172F16C077247394B701CE010996FB
:10CFB0000E946F2C29833A834B835C836D837E832D
:10CFC0008F8398873F7009F498CFCE0101960E9415
:10CFD000BB296B017C0139C0B701CE0109960E94C3
:10CFE0006F2C29833A834B835C836D837E838F838D
:10CFF00098873F7009F481CF31503B3008F0B7CFAC
:10D00000E32FF0E08827E85FF7498F4F0D94966B88
:10D010001C681C68B767136813687A686D686D6868
:10D020006D68136813682D813E814F815885AAE091
:10D03000B0E00F944C6BCDCFCD80BAE0CB9E6001B9
:10D0400011240D2C000CEE08FF0880911E0289307F
:10D0500020F480911D028930E8F060E770E28EEBE9
:10D0600091E10F947735B5018EEB91E10F94203566
:10D0700069E670E28EEB91E10F9477352AE030E0BB
:10D08000B701A6018EEB91E10F949A348EEB91E1FA
:10D090000F947834D8011296ED91FC9162E084816E
:10D0A00095810E9462F6009791F581E090E060968C
:10D0B0000FB6F894DEBF0FBECDBFDF91CF911F91A9
:10D0C0000F91FF90EF90DF90CF90BF90AF909F9027
:10D0D0008F907F906F905F90089520E030E040E265
:10D0E00051E46D817E818F8198850F94276A0F941A
:10D0F000936C6FCF6D817E818F8198852AE030E0BF
:10D1000040E050E00F942D6B69017A019ECFFC0145
:10D1100020852F70263049F6B5010E94EAF58C0172
:10D12000009719F2DC0118968C9118978F709BEF7D
:10D13000980F923008F0B9CF502E612E853029F427
:10D1400016965C90169717966C9069E077E0852D9F
:10D15000962D0E94EAF55C01852D962D0F94CF0443
:10D16000A114B104F9F081149104E1F0F4012085D7
:10D170002F702130B9F421852223A1F0009749F1C5
:10D18000DC0119964D915D916D917C911C974C1528
:10D190005D056E057F0531F418968C91807F6CE0FB
:10D1A00077E071F1D80118968C91189780681896DD
:10D1B0008C93A114B10469F1F501C186D286E3868E
:10D1C000F486729490EF792280858F70782A708629
:10D1D0006CCFF50181859285A385B4858C159D055D
:10D1E000AE05BF05F9F6208522952F70872D8F702B
:10D1F000082E000C990B28171906A1F66DE277E0AE
:10D200008EEB91E10F9420358EEB91E10F94783401
:10D210004CCF60E670E28EEB91E10F947735D80148
:10D220006D917C918EEB91E10F9420358EEB91E125
:10D230000F947834A701960169E077E0852D962D4B
:10D240000F94230269E077E0852D962D0E94EAF580
:10D25000FC01892B09F429CF729480EF7822908504
:10D260009F70792AB4CF2F923F924F925F927F9214
:10D270008F929F92AF92BF92CF92DF92EF92FF92E6
:10D280000F931F93CF93DF9300D000D01F921F9274
:10D29000CDB7DEB709831A832B833C834D835E832E
:10D2A0006F837887DC011496ED91FC910FEF1FEFEF
:10D2B0003097F9F057014C01C288D388E114F1048A
:10D2C00089F1F7018081882369F1C114D10489F1C2
:10D2D000B701C6010E94EAF5E980FA800B811C8142
:10D2E0002D813E814F815885BC01C4010E94596740
:10D2F0008C01C80128960FB6F894DEBF0FBECDBFD3
:10D30000DF91CF911F910F91FF90EF90DF90CF9021
:10D31000BF90AF909F908F907F905F904F903F9085
:10D320002F900895C114D10421F0D6011696CD9006
:10D33000DC907B80F12C0FEF1FEF272C312C512C30
:10D34000412CC114D10449F165EC76E0C6010E947C
:10D35000EAF50097E9F0FC0120852F702230C1F436
:10D3600081859285A385B48582159305A405B505AD
:10D3700079F4E980FA800B811C812D813E814F81F7
:10D380005885B601C4010E9459678C01FF24F394AB
:10D39000D6011296CD90DC90D4CFF110AACF6BE8D5
:10D3A00070E287E191E10F947735B50187E191E172
:10D3B0000F9420356FE770E287E191E10F947735A4
:10D3C000672D70E087E191E10E947BF687E191E1B2
:10D3D0000F9478348ECF1F93CF93DF9300D000D07B
:10D3E000CDB7DEB76130710509F46BC05CF4672B13
:10D3F00009F45DC06FE07EE18EEB91E10F9477352B
:10D4000080E04BC06230710571F06330710591F7B7
:10D4100090933E0F80933D0F55275093400F4093BC
:10D420003F0F84E009C090933E0F80933D0F5093CF
:10D43000400F40933F0F83E00F94710A182F4FEF76
:10D440005FEFBA0180E00F9452566093DE0C709348
:10D45000DF0C8093E00C9093E10C1123D9F06AEF7C
:10D460007DE187E191E10F947735812F90E0B0E085
:10D47000A0E089839A83AB83BC8380E190E09E83A4
:10D480008D83BE016F5F7F4F87E191E10E94AFBE48
:10D490000F94783481E01111B3CF26960FB6F8942B
:10D4A000DEBF0FBECDBFDF91CF911F910895909346
:10D4B0003E0F80933D0F5093400F40933F0F81E00C
:10D4C000BBCF90933E0F80933D0F5093400F4093FE
:10D4D0003F0F82E0B1CFCF93DF93EC01EC81FD8170
:10D4E00040815181052E000C660B770B22818CE365
:10D4F0009EE00F94833670E060E08A819B810E94F9
:10D500005CB5E9E3FFE082838CE39EE09183808356
:10D510001092491010924B1010924A10DF91CF9147
:10D5200008958F929F92AF92BF92CF92DF92EF9227
:10D53000FF920F931F93CF93DF937C014A01590110
:10D54000C091DC0CD091DD0C062F660F110B2097DB
:10D5500009F45CC088858F70863009F055C06EE490
:10D5600077E0CE010E94EAF56C0182E08816910412
:10D5700049F063E577E0E3E08E16910429F0D0E00E
:10D58000C0E006C067E577E0CE010E94EAF5EC0155
:10D59000C114D104D9F1F60180858F708430B1F5C2
:10D5A00061857285A801C7010F942570A8016CE5FB
:10D5B00077E0C7010F940770209779F188858F7005
:10D5C000843059F569857A85A801C7010F940770E1
:10D5D000A8016CE577E0C7010F940770A114B104AE
:10D5E00029F0A801B501C7010F940770C701DF91A9
:10D5F000CF911F910F91FF90EF90DF90CF90BF9050
:10D60000AF909F908F900895D0E0C0E0A80164E4AF
:10D6100076E2C7010F940364C9CFF2E08F1691043C
:10D6200081F083E08816910429F06091DA0C709102
:10D63000DB0CCACFA8016EE376E2C7010F94E56365
:10D64000C7CFA8016BE376E2F8CFFF920F931F9349
:10D65000CF93DF93CDB7DEB7C455D1090FB6F89499
:10D66000DEBF0FBECDBF8C01F62EDC0116966C918D
:10D67000FF2011F081E06827F80184810F946E0685
:10D68000F80187819085A185B285883E9340A105E8
:10D69000B10508F49BC060E475E28EEB91E10F9454
:10D6A00077356BE375E28EEB91E10F947735D80116
:10D6B00014966D917C918EEB91E10E947BF666E36E
:10D6C00075E28EEB91E10F9477356F2D70E08EEB64
:10D6D00091E10E947BF68EEB91E10F947834FE018C
:10D6E000E55BFF4F8FE290E08193919388E0DF014B
:10D6F0001D928A95E9F76FE275E2CE01855B9F4F37
:10D700000F94C163F801828193810E949BBCFF202A
:10D7100009F469C067E275E2853151F060E275E2B3
:10D72000863131F064E175E28F3011F46CE175E21D
:10D73000CE018F5B9F4F0F94D56380913F139091E3
:10D740004013059709F442C0D8011296ED91FC915F
:10D750000280F381E02D0081118101151105B1F1E5
:10D7600040E450E0B801CE0101960F9425706FE2BD
:10D7700070E0CE0101960F94EC6F892B41F4980173
:10D7800043E050E060E4CE0101960E94916A4FE3CD
:10D7900050E0BE01655B7F4FCE0101960F9407708C
:10D7A0000E9408F6882391F080913F1390914013D6
:10D7B000069761F480913A13811108C041E0BE01DF
:10D7C0006F5B7F4FCE0101960F94E509CC5ADF4F76
:10D7D0000FB6F894DEBF0FBECDBFDF91CF911F9182
:10D7E0000F91FF90089560E175E2823009F4A0CFB7
:10D7F0006BE075E29DCFAF92BF92CF92EF92FF9216
:10D800000F931F93CF93DF9300D000D01F921F92EE
:10D81000CDB7DEB75C0109831A832B833C834D832C
:10D820005E836F83788765E875E28EEB91E10F94F4
:10D830007735CE0101960E94F425E114F10439F008
:10D840006EE775E2C7010F94CC63009749F1F501CB
:10D85000028113810115110509F18981811163C0CC
:10D860008B81813009F467C068F1823049F1082F5B
:10D8700010E06BE575E28EEB91E10F9477356BE488
:10D8800075E28EEB91E10F947735B8018EEB91E163
:10D890000E947BF68EEB91E10F94783490E080E06B
:10D8A00028960FB6F894DEBF0FBECDBFDF91CF91A3
:10D8B0001F910F91FF90EF90CF90BF90AF90089580
:10D8C000CC20D9F060E0CE0101960E941428892B6B
:10D8D00009F44EC0C8010E94D0B4672B682B692B95
:10D8E000F9F44FEF5FEFBA0180E00F945256AB01AD
:10D8F000BC01C8010E948FB413C0C8010E949BBC28
:10D900008E3019F050F4813059F460E0CE01019668
:10D910000E941428892B21F0DDCF83518430A8F395
:10D9200081E090E0BDCF8031F0F48E3098F6813008
:10D9300089F28230E9F063E775E28EEB91E10F94B2
:10D94000773566E675E28EEB91E10F947735698164
:10D950008EEB91E10E9474F68EEB91E10F94783496
:10D9600001E010E086CF8351843008F4B3CFE3CFD9
:10D9700040E050E0BA01C8010E948FB460E0C501E8
:10D980000E94256BCDCF4F925F926F927F928F92C4
:10D990009F92AF92BF92CF92DF92FF920F931F930D
:10D9A000CF93DF9300D000D01F921F92CDB7DEB788
:10D9B0006130710509F482C0FC01628173816115D7
:10D9C000710509F47BC08C0119821A821B821C82AA
:10D9D0001D821E821F8218868A81807F8A8340E092
:10D9E00050E2CE0101960E94512760E0CE010196DF
:10D9F0000E9414286C01F801828193810E94D0B4A6
:10DA00002B013C01F8012781308541855285D601E3
:10DA10000F94576B2FEF30E040E050E00F940B6B0A
:10DA200049015A010F941709FF24F39481149104BA
:10DA3000A104B10461F06419750986099709FF24EE
:10DA4000F394681579058A059B0508F4F12C4114B7
:10DA500051046104710491F1F80187809084A184DC
:10DA6000B2840F941709F80181149104A104B10440
:10DA700051F06419750986099709681579058A05B1
:10DA80009B0508F449C0A280B3804FEF5FEFBA0155
:10DA900080E00F945256AB01BC01C5010E948FB4C7
:10DAA000CD2861F0F80184810F943B56F8019681EE
:10DAB000891304C061E0C8010E94256B90E080E0FA
:10DAC00028960FB6F894DEBF0FBECDBFDF91CF9181
:10DAD0001F910F91FF90DF90CF90BF90AF909F90DC
:10DAE0008F907F906F905F904F900895FF20D9F0B6
:10DAF00060E0C8010E94256BF801828193810E9439
:10DB0000D7D6892BD9F640E050E0BA01F8018281DE
:10DB100093810E948FB4D2CF84810F943B56F80139
:10DB200096818913E3CFCD2849F2F80184810F94BF
:10DB30003B56F80196818913C1CFF110BFCFBACF00
:10DB4000AF92BF92CF92DF92EF92FF921F93CF934B
:10DB5000DF9300D000D0CDB7DEB76C017C0110E0C0
:10DB60008AE0A82EB12C133061F1F701828190E098
:10DB7000B0E0A0E089839A83AB83BC83BE82AD8290
:10DB8000BE016F5F7F4F8DE091E10E94AFBE69E300
:10DB900076E20F9477351F5FFFEFEF1AFF0A14301C
:10DBA00011F726960FB6F894DEBF0FBECDBFDF91FA
:10DBB000CF911F91FF90EF90DF90CF90BF90AF90EB
:10DBC0000895F601858190E0B0E0A0E089839A8312
:10DBD000AB83BC83BE82AD82BE016F5F7F4F8DE0A1
:10DBE00091E10E94AFBE67E376E2D3CFFC01DC0196
:10DBF0008D918111FDCF30E020E050E040E08AE0DF
:10DC00009191992301F1443051055CF59E3271F4F4
:10DC10002F3F310509F02CF5DB01A40FB51F12963B
:10DC20002C934F5F5F4F30E020E0EACF829FD0011E
:10DC3000839FB00D1124292F990F330B20533109E5
:10DC40002A0F3B1FDDCF2F3F310509F054F444303C
:10DC500051053CF4640F751FFB01228381E090E0C5
:10DC6000089590E080E00895CF93DF931F921F9274
:10DC7000CDB7DEB78091571490915814009711F4E6
:10DC800083E694E1BE016F5F7F4F681B790B072E1F
:10DC9000000C880B990B0F900F90DF91CF91089596
:10DCA0004F925F926F927F929F92AF92BF92CF926C
:10DCB000DF92EF92FF920F931F93CF93DF93CDB735
:10DCC000DEB768970FB6F894DEBF0FBECDBFFC017C
:10DCD000198A1A8A1B8A1C8A1D8A1E8A1F8A188E14
:10DCE0008A89807F8A8BA081B181109709F47AC0DC
:10DCF0008C91882309F476C000811181D8019C9110
:10DD0000992309F443C09D3209F4DAC090539A3044
:10DD100028F00F5F1F4F11830083EECFC801912CB5
:10DD2000DC016D01C81AD90A2D91022E000C330BAB
:10DD3000205331092A303105A0F37F016EE270E0F3
:10DD4000C8010F94EC6FFC01009709F448C0DC0196
:10DD50005D01AE1ABF0A11968C911197082E000C26
:10DD6000990BC09711960A9798F38181282F082E56
:10DD7000000C330B205331092A30310518F480335D
:10DD80000CF057C020E030E0A90108C0912CD12C44
:10DD9000C12CD3CF29E030E040E050E0AAE0B0E071
:10DDA0000F944C6B2B013C012281822F022E000C20
:10DDB000990BC0978A30910570F420330CF441C060
:10DDC0002A330CF042C0092E000CAA0BBB0B480EE4
:10DDD000591E6A1E7B1EA114B10409F088C0CD280B
:10DDE00009F073C088E0FE017196DE01199601907A
:10DDF0000D928A95E1F729853A854B855C856D857D
:10DE00007E858F85988968960FB6F894DEBF0FBE21
:10DE1000CDBFDF91CF911F910F91FF90EF90DF90D9
:10DE2000CF90BF90AF909F907F906F905F904F90FA
:10DE300008958A330CF0AECF032E000C440B550B23
:10DE4000ADCF80E090E0DC01C2CF89E090E0A0E0BF
:10DE5000B0E0BDCFB8E0CB16D1040CF04DC0C80186
:10DE60000F947E639B01AC01A4E6B0E00F944C6B71
:10DE7000992041F07094609450944094411C511C3E
:10DE8000611C711C2A89207F26602A8B460E571E32
:10DE9000681E791E4D8A5E8A6F8A788E6CE270E009
:10DEA000F701808191810F94EC6F009721F4D701E5
:10DEB0001D921C9297CF0196F7019183808392CF98
:10DEC000C8010196992493942BCFC8010F947E63C7
:10DED000AB01BC01CE0141960E94282729833A83D9
:10DEE0004B835C836D837E838F839887D7CFF3E0EA
:10DEF000AF16B1040CF4AECFC8010F945C632A894D
:10DF0000207F27602A8B6D8B7E8B8F8B988FC6CF5F
:10DF1000CF92DF92EF92FF920F931F93CF93DF93F5
:10DF2000EC01A881B981109781F18C91882369F166
:10DF300008811981F8019081992351F09D3241F0B7
:10DF400090539A3028F00F5F1F4F19830883F0CF4A
:10DF5000C8010F947E636B017C016CE270E0C80124
:10DF60000F94EC6F009769F419821882C701B6010B
:10DF7000DF91CF911F910F91FF90EF90DF90CF90A5
:10DF80000895019699838883F1CFC12CD12C760115
:10DF9000EDCF0097B1F1FC01DB01AC01405F5F4FB9
:10DFA00080E090812FE9290F263098F497559295BB
:10DFB000907F9C9321813FE9320F3630B0F4275592
:10DFC000922B9D933296E417F50759F791E0892734
:10DFD00008952FEB290F263010F49753E8CF905374
:10DFE0009A3028F381E090E0E2CF3FEB320F3630F9
:10DFF00010F42753E5CF20532A3010F381E020E0BE
:10E00000DFCF80E008950097D1F0DC011696ED9106
:10E01000FC913097A1F080858F70843021F4818548
:10E020009285009771F40680F781E02D309739F0E2
:10E0300080858F70843019F481859285089590E0F1
:10E0400080E00895089508950895089508950F9320
:10E050001F93CF93DF93EC011D860A811B8170E033
:10E0600060E0C8010E945CB587FD44C08C838C8150
:10E070008150853410F080E28C8361E070E0C8014B
:10E080000E945CB587FD3BC08D838D8181508534B6
:10E0900010F081E28D8362E070E0C8010E945CB5FF
:10E0A000863490F58E8363E070E0C8010E945CB511
:10E0B0009C01215031092115344040F59A87898708
:10E0C00064E070E0C8010E945CB5813024E09207F2
:10E0D00000F59C878B8765E070E0C8010E945CB505
:10E0E00018161906CCF498878F83DF91CF911F9172
:10E0F0000F91089581958C8381E08D87B8CF8195AC
:10E100008D8381E08D87C1CF1E82CDCF1A8619867F
:10E11000D7CF80E094E0DDCF80E197E2E4CFCF93EA
:10E12000DF93EC0163EE74E28EEB91E10F947735AF
:10E130006EED74E28EEB91E10F9477356C817D8109
:10E140008EEB91E10E947BF668ED74E28EEB91E13B
:10E150000F9477358EEB91E10F94783461E08C81E8
:10E160000F949C066E818C810F946E068A819B8130
:10E17000009729F040E050E0BA010E948FB4E88196
:10E18000F9810484F585E02D62E0CE0119958A813C
:10E190009B81009799F00E94D7D61816190674F43F
:10E1A0000A80DB81C02D4FEF5FEFBA0180E00F9452
:10E1B0005256AB01BC01CE010E948FB481E090E0C9
:10E1C000DF91CF910895CF93DF93EC0165EB74E27B
:10E1D0008EEB91E10F9477356C817D818EEB91E12F
:10E1E0000E947BF663EB74E28EEB91E10F9477353E
:10E1F000EA81FB810280F381E02D608171818EEBE9
:10E2000091E10F9420356DEA74E28EEB91E10F9469
:10E2100077358EEB91E10F9478348A819B81892B3D
:10E2200009F451C08C819D81892B09F04CC0E88193
:10E23000F981008CF18DE02DCE0119958130910589
:10E2400029F0029759F061E08C811AC063E070E018
:10E25000CE010E94A2EF61E00F949C0661E08C81E8
:10E260000F949C0661E070E0CE010E94A2EF61E095
:10E270000F949C0662E070E0CE010E94A2EF61E084
:10E280000F949C068091A100887F8093A1008091CB
:10E290009100887F809391008091A100826080939B
:10E2A000A10080919100826080939100E881F981C2
:10E2B0000484F585E02D62E0CE01199581E090E0BF
:10E2C000DF91CF91089590E080E0FACF2F923F92B6
:10E2D0004F925F926F927F928F929F92AF92BF9276
:10E2E000CF92DF92EF92FF920F931F93CF93DF9322
:10E2F000CDB7DEB76A970FB6F894DEBF0FBECDBFBD
:10E300009C878B87DC011496ED91FC91309709F482
:10E310008FC2268037802114310409F450C2D10104
:10E32000ED91FC91309709F445C28081882309F46E
:10E3300041C22FEF3FEFA90163E979E0C1010E94DB
:10E34000C26422E030E040E050E06BED77E0C101D4
:10E350000E94C2642FEF3FEFA90163E577E0C1019E
:10E360000E94C26464EC76E0C1010E94EAF59A83DF
:10E370008983009709F41EC2FC0180858F70853067
:10E3800009F018C2CF010E9434F7833008F412C29A
:10E3900020E030E040EA51E463E578E0C1010E940A
:10E3A0008D645C010E949B5D20E030E040EC5FE703
:10E3B0006DE775E0C1010E948D646C010E949B5D58
:10E3C00020E030E040E050EC6EE577E0C1010E94D3
:10E3D0008D647C010E949B5D00E010E020E83FE33B
:10E3E00050E040E061E677E089819A810F945455CE
:10E3F0002B013C0120E030E0A9010F94C169912C70
:10E40000812C87FF07C077FA709477F8709488247E
:10E410008394912C00E010E0980141E050E064E624
:10E4200077E089819A810F9454556B837C838D8327
:10E430009E8300E010E0980142E050E067E677E05C
:10E4400089819A810F9454556F83788789879A8739
:10E4500000E010E020EA30E443E050E06AE677E0D4
:10E4600089819A810F945455698B7A8B8B8B9C8B05
:10E4700000E010E020EF32E444E050E06DE677E0A9
:10E48000C1010F9454556D877E878F87988B00E06C
:10E4900010E0980145E050E067E777E0C1010F9494
:10E4A00054556D8B7E8B8F8B988F88E490E00F9402
:10E4B00093619A8F898FF9E0EF0EF11CDC015F9672
:10E4C000FC92EE925E97B9E0CB0ED11CFC01D58E8A
:10E4D000C48EF9E0AF0EB11CDC019196BC92AE92F5
:10E4E0009097FC01EA5BFF4F1082389710821182EF
:10E4F00012821382349680E090E0AFE7B3E4808329
:10E500009183A283B38384E690E0A0E0B0E0E98D3C
:10E51000FA8D82AF93AFA4AFB5AFB401CF010F9422
:10E52000E53620E030E0A901C301B2010F94C169D2
:10E5300087FD9FC020E030E0A9016B817C818D8147
:10E540009E810F94C16987FD94C020E030E0A9014D
:10E550006F81788589859A850F94C16987FD89C007
:10E5600081E090E0A98DBA8D5B969C938E935A972B
:10E57000FD01E95BFF4FB1E0B083E98DFA8D408288
:10E580005182628273828B819C81AD81BE81848342
:10E590009583A683B7838F819885A985BA8580875F
:10E5A0009187A287B38762AD73AD84AD95AD0F94AB
:10E5B000C66920E030E04AE754E40F94216C6B0117
:10E5C0007C01A98DBA8D1C964D925D926D927C92C4
:10E5D0001F97AC019B016B817C818D819E810F9483
:10E5E000276A4B015C01E98DFA8D808A918AA28AA3
:10E5F000B38AA70196016F81788589859A850F94E2
:10E60000216C6B017C01A98DBA8D5496CD92DD925F
:10E61000ED92FC92579758968D919C91019749F5F0
:10E62000A301920160E070E0CB010F94B46BE98D1F
:10E63000FA8D6487758786879787A501940160E0C6
:10E6400070E0CB010F94B46BA98DBA8D50966D9389
:10E650007D938D939C935397A701960160E070E0A2
:10E66000CB010F94B46BE98DFA8D648B758B868B1F
:10E67000978B20E030E04AE754E46D857E858F85F6
:10E6800098890F94276A0F949A6C6B017C010F9400
:10E690001709A98DBA8DDA968D909D90AD90BC909A
:10E6A000DD97681979098A099B09FD0166A377A39B
:10E6B00080A791A79E96CD92DD92ED92FC92D19784
:10E6C0008D899E89AF89B88D82A393A3A4A3B5A396
:10E6D00012A613A614A615A6CD28CE28CF2859F029
:10E6E000048CF58DE02D80E090E0A0ECBFE7808306
:10E6F0009183A283B383E98DFA8DC2A0D3A0E4A055
:10E70000F5A0A7019601C701B6010F94296D8111EB
:10E7100009C0A98DBA8D5E96ED91FC91C082D1821F
:10E72000E282F382E98DFA8DCF01FF0FAA0BBB0BBA
:10E73000E981FA8181879287A387B48720E030E05E
:10E740004AE754E469897A898B899C890F94276AFE
:10E750000F94936C898D9A8D0F94723964EF70E2E7
:10E760008EEB91E10F947735B301A2018EEB91E12D
:10E770000E94F5FA62E877E08EEB91E10F94203584
:10E780004B815C816D817E818EEB91E10E94F5FA77
:10E7900066E877E08EEB91E10F9420354F81588544
:10E7A00069857A858EEB91E10E94F5FA8EEB91E115
:10E7B0000F947834D10112962D903C90ACCD69EE37
:10E7C00070E28EEB91E10F9477358EEB91E10F942F
:10E7D000783440E050E0BA01EB85FC85828193817A
:10E7E0000E948FB4AB85BC85ED91FC911197048498
:10E7F000F585E02D62E0CD01199581E090E06A9603
:10E800000FB6F894DEBF0FBECDBFDF91CF911F9141
:10E810000F91FF90EF90DF90CF90BF90AF909F90BF
:10E820008F907F906F905F904F903F902F900895C2
:10E8300065ED70E28EEB91E10F9477358EEB91E10F
:10E840000F94783490E080E0DACFCF93DF93EC013F
:10E850000E9427706AE877E08EEB91E10F947C3498
:10E8600061E08C810F949C0661E08D810F949C0681
:10E870006D858C810F946E066D858D810F946E066B
:10E8800060E08E810F949C0640E050E0BA018A81DE
:10E890009B810E948FB440E050E061E070E08A818B
:10E8A0009B810E9406B640E050E062E070E08A8101
:10E8B0009B810E9406B6E881F9810484F585E02DEC
:10E8C00062E0CE01199582E08093000281E090E041
:10E8D000DF91CF9108952F923F924F925F926F9266
:10E8E0007F928F929F92AF92BF92CF92DF92EF92E0
:10E8F000FF920F931F93CF93DF93CDB7DEB7CB5724
:10E90000D1090FB6F894DEBF0FBECDBFE296EFAED1
:10E91000E297E396FFAEE397E4960FAFE497E596B0
:10E920001FAFE597E6962FAFE697E7963FAFE797DD
:10E93000E8964FAFE897E9965FAFE9970097B9F18E
:10E9400024012B2CEC96AFAEEC97EB96DFAEEB9759
:10E95000EA96CFAEEA97362E8C0180911E0289305E
:10E9600020F480911D028930C0F0C8010E943EFE53
:10E970007C01892B91F066E977E08EEB91E10F94B1
:10E980002035B7018EEB91E10F9420358EEB91E1AC
:10E990000F947834C7010F942F62F80180858F702F
:10E9A000843009F45FC128F4882309F464C180E04D
:10E9B0002FC0853009F446C08630C9F769E375E099
:10E9C000C8010E94EAF53C01009709F476C0912C39
:10E9D000812CB12CA12CD12CC12CE296EFACE2976A
:10E9E000E396FFACE397E4960FADE497E5961FAD91
:10E9F000E597E6962FADE697E7963FADE797E89661
:10EA00004FADE897E9965FADE997632D0E946B746F
:10EA1000C558DF4F0FB6F894DEBF0FBECDBFDF91F4
:10EA2000CF911F910F91FF90EF90DF90CF90BF900B
:10EA3000AF909F908F907F906F905F904F903F909E
:10EA40002F90089580913B138F5F80933B136680D6
:10EA500077806114710459F14201EC96AFACEC97E8
:10EA6000B22CEA96CFACEA97EB96DFACEB97E29646
:10EA7000EFACE297E396FFACE397E4960FADE49733
:10EA8000E5961FADE597E6962FADE697E7963FAD85
:10EA9000E797E8964FADE897E9965FADE997632D64
:10EAA000C3010E946B74F30162807380D2CF8091A6
:10EAB0003B13815080933B137ACF6CE977E0C80118
:10EAC0000E94EAF52C0161EA77E0C8010E94EAF5AC
:10EAD0007C0166EA77E0C8010E94EAF5332039F04C
:10EAE000F1E03F1609F49FC0D12CC12C0CC06AEA9A
:10EAF00077E0C8010E94EAF53C016AED77E0C801C1
:10EB00000E94EAF56C016114710409F43801C11422
:10EB1000D10409F468014114510431F4EA964FAC70
:10EB2000EA97EB965FACEB97E114F10421F4EC96D5
:10EB3000EFACEC97F22C6114710409F4A5C0F30159
:10EB400080858F70843009F09FC061847284C11405
:10EB5000D10409F49CC0F60180858F70843009F0DF
:10EB600096C0C184D28410E000E04114510409F43D
:10EB7000F3C06114710409F4B1C061E976E28EEB6F
:10EB800091E10F947735F201618572858EEB91E109
:10EB90000F9420356CE876E28EEB91E10F94773597
:10EBA000B3018EEB91E10F9420358EEB91E10F9440
:10EBB0007834CE018F589F4F0E94F425E114F10460
:10EBC00009F0D3C0F20180858F70843009F083C1D1
:10EBD000409141135091421361857285CE01019697
:10EBE0000E94C7BDCE0101960E9469B38823B1F08F
:10EBF0000E94346E6B01683C71050CF083C06BE4BD
:10EC000076E287E191E10F947735B60187E191E1F2
:10EC10000E947BF687E191E10F947834CE01019652
:10EC20000E9464BE58C16FEA77E0C8010E94EAF50D
:10EC30003C0164EB77E0C8010E94EAF56C016114C5
:10EC4000710409F04AC16AEA77E0C8010E94EAF556
:10EC50003C01C114D10409F450CF892B09F05BCFDA
:10EC6000380159CFD12CC12C712C612CF12CE12C05
:10EC7000512C412C48CFD12CC12C712C612CF12C62
:10EC8000E12C512C412C47CF712C612C60CF00E03E
:10EC900020E030E340E150E0BE016F597F4FCE01EC
:10ECA0008F589F4F0E94CF236C01E4960FADE497DD
:10ECB00010E00115110509F058CFE2968FADE297EB
:10ECC000811109C0E3968FADE3978F7009F44DCFA2
:10ECD00002E010E04ACF01E010E047CF62E876E2C0
:10ECE0008EEB91E10F947735F201618572858EEBA1
:10ECF00091E10F9420356DE776E28EEB91E10F9470
:10ED0000773557CF6114710431F0B301CE0101960C
:10ED10000E947DFE83CFA12CC12CF12CE12CE29628
:10ED20000FADE297E3961FADE397E4962FADE4971E
:10ED3000E5963FADE597E6964FADE697E7965FAD72
:10ED4000E797E8966FADE897E9967FADE997CE0132
:10ED500001960E94C2C262CFE114F10409F4BBC063
:10ED6000C114D10409F4B7C004C0C114D10409F41A
:10ED700029CFF70180858F70843009F0A8C0818584
:10ED8000928525961FAE1EAE259748EE53E060E0B3
:10ED900070E029964CAF5DAF6EAF7FAF29972BED3A
:10EDA00032E023963FAF2EAF23972F969FAF8EAFC3
:10EDB0002F9761961FAE1EAE619763961FAE1EAE73
:10EDC000639765961FAE1EAE659767961FAE1EAE23
:10EDD000679769961FAF0EAF69976A961FAE6A97DD
:10EDE00040E450E0BE016F5F7F4FCE018F5B9F4FCD
:10EDF0000E94E8F721E030E02C0F3D1F820F931FA7
:10EE0000FC01108265E776E28EEB91E10F94773595
:10EE1000F701618572858EEB91E10F94203569EBE6
:10EE200077E08EEB91E10F942035BE016F5F7F4F4D
:10EE30008EEB91E10F94203560E776E28EEB91E165
:10EE40000F947735B6018EEB91E10F9420358EEB60
:10EE500091E10F9478340E9408F68823C1F18091E3
:10EE60003A13811134C06FE270E0CE0101960F9425
:10EE7000EC6F892B51F4F7012185328543E050E096
:10EE800060E4CE0101960E94916A69E676E28EEB1B
:10EE900091E10F947735BE016F5F7F4F8EEB91E16B
:10EEA0000F94203564E676E28EEB91E10F9477358E
:10EEB000B6018EEB91E10F9420358EEB91E10F942A
:10EEC000783441E0B601CE0101960F94E509411472
:10EED000510409F077CE81E09BCD892B09F01BCE40
:10EEE0000CCE8F929F92AF92BF92CF92DF92EF9211
:10EEF000FF920F931F93CF93DF9300D000D01F9208
:10EF00001F92CDB7DEB7DC011296ED91FC913097E0
:10EF100009F468C024813581232B09F463C08C0176
:10EF2000662309F472C00E94A262E62EB72E6C011D
:10EF3000D8011296ED91FC910280F381E02D608161
:10EF4000718187E191E10F94203566E374E287E1F6
:10EF500091E10F94773587E191E10F94783420E0C7
:10EF600030E0A9016E2D7B2DC6010F94C96C87FD81
:10EF700039C06AE274E287E191E10F9477354E2D52
:10EF80005B2DB60187E191E10E94F5FA87E191E1FD
:10EF90000F947834D8011296ED91FC9161E0848150
:10EFA00095810E9462F619821A821B821C822A8134
:10EFB000207F2760F22E2E2D4E2D5B2DB6014D8326
:10EFC0005E836F837887912C812CB12CA12CD12C5E
:10EFD000C12CE9800B811C813E814F8158856FEFE8
:10EFE0000E946B7428960FB6F894DEBF0FBECDBF9B
:10EFF000DF91CF911F910F91FF90EF90DF90CF9015
:10F00000BF90AF909F908F9008950280F381E02D84
:10F01000608171818DE091E10F94203563E474E2A9
:10F020008DE091E10F9477358DE091E128960FB650
:10F03000F894DEBF0FBECDBFDF91CF911F910F912E
:10F04000FF90EF90DF90CF90BF90AF909F908F9008
:10F050000D9478344F925F926F927F928F929F922D
:10F06000AF92BF92CF92DF92EF92FF920F931F93D6
:10F07000CF93DF93CDB7DEB7E8970FB6F894DEBF36
:10F080000FBECDBF09AB1AAB2BAB3CAB4DAB5EABF0
:10F090006FAB78AFDC011496ED91FC91309719F4C9
:10F0A00090E080E0C9C020813181232BC9F33C016D
:10F0B000DC01ED91FC910284F385E02D1995029716
:10F0C00079F78BA9E82EF12C19A9112321F0E1146D
:10F0D000F10409F431C1823009F4D7C090F48130D1
:10F0E000A9F066E574E28EEB91E10F947735B701F4
:10F0F0008EEB91E10E947BF68EEB91E10F947834D8
:10F10000CFCF833009F44AC0893059F7D301129622
:10F11000ED91FC9161E0848195810E9462F62C0161
:10F1200019A61AA61BA61CA61DA61EA61FA618AACF
:10F130008AA5807F8AA719A761E0CE0189960E94DF
:10F14000E42629A33AA34BA35CA36DA37EA38FA3BC
:10F1500098A71150193108F013C2E12FF0E0882769
:10F16000EB54F7488F4F0D94966BE279A079C07AF3
:10F17000C07AC07AC07AC07AC07AC07A117A717ABD
:10F18000C07AC07AE279E279C07AC07AC07AE2794C
:10F19000E279E279E279C07AC07AAD7A8AA98F7091
:10F1A00009F47ECFCE01C1960E947529D301149631
:10F1B000ED91FC91668377838087918767EA74E29B
:10F1C0008EEB91E10F947735D3011296ED91FC917E
:10F1D0000280F381E02D608171818EEB91E10F94CB
:10F1E000203569E974E28EEB91E10F947735D30114
:10F1F0001496ED91FC9146815781608571858EEB67
:10F2000091E10E94F5FA8EEB91E10F947834F301CD
:10F21000E480F5800F941709D70152966D937D9382
:10F220008D939C935597D3011496ED91FC9186890B
:10F23000811119C081E090E0E8960FB6F894DEBF26
:10F240000FBECDBFDF91CF911F910F91FF90EF9037
:10F25000DF90CF90BF90AF909F908F907F906F90F6
:10F260005F904F900895168A60E0C3010E94717705
:10F27000D3011496ED91FC9180E090E0A0E0B0EC19
:10F2800086879787A08BB18BD5CF8AA98F7009F419
:10F2900007CFCE01C1960E947529D3011496ED9136
:10F2A000FC91628773878487958763E974E28EEBAC
:10F2B00091E10F947735D3011296ED91FC91028084
:10F2C000F381E02D608171818EEB91E10F94203507
:10F2D00068E874E28EEB91E10F947735D3011496D0
:10F2E000ED91FC9142855385648575858EEB91E1A6
:10F2F0000E94F5FA8EEB91E10F947834D3011296C7
:10F30000ED91FC9162E0848195810E9462F6009704
:10F3100009F490CF912C812CB12CA12CD12CC12C93
:10F32000E9A8FAA80BA91CA92DA93EA94FA958AD77
:10F330006FEF0E946B747ECFEE24E394F12CE6CE47
:10F3400080913F13909140130597F1F019821A8232
:10F350001B821C821D821E821F8218868A81807FEA
:10F360008A836BE0CE0101960E940627912C812CA6
:10F37000B12CA12CD12CC12C79018A019B01AC01AB
:10F380006FEFC2010E946B74912C812CB12CA12CC7
:10F39000D12CC12CE9A4FAA40BA51CA52DA53EA532
:10F3A0004FA558A96FEFC2010E946B7430E020E0B6
:10F3B00040E050E460E070E0F301828193810E94BC
:10F3C000E8B938CF19821A821B821C821D821E82E4
:10F3D0001F8218868A81807F8A8340E051E060E046
:10F3E00070E0D30112968D919C910E9458B6672BC4
:10F3F000682B692BA1F06BE0CE0101960E940627D5
:10F40000912C812CB12CA12CD12CC12C79018A01F9
:10F410009B01AC016FEFC2010E946B74BBCF6AE02D
:10F42000EBCF80913F1390914013059791F061E0ED
:10F43000D30112968D919C910E947CBC30E020E01B
:10F4400040E050E160E070E0F301828193810E942E
:10F45000E8B940E050E061E070E0D30112968D9190
:10F460009C910E942FB6912C812CB12CA12CD12CD7
:10F47000C12CE9A4FAA40BA51CA52DA53EA54FA55A
:10F4800058A96FEFC2010E946B74D301ED91FC91FA
:10F490000288F389E02DC3011995892B09F4E8CE80
:10F4A00019821A821B821C821D821E821F8218866C
:10F4B0008A81807F8A8361E0CE0101960E940627BF
:10F4C00029873A874B875C876D877E878F87988BE4
:10F4D00079018A019B01AC016FEFC2010E946B743C
:10F4E000C7CE912C812CB12CA12CD12CC12CE9A4FC
:10F4F000FAA40BA51CA52DA53EA54FA558A96FEFF5
:10F50000C2010E946B74D301ED91FC910288F389D2
:10F51000E02DC3011995892B09F08CCE19861A8626
:10F520001B861C861D861E861F86188A8A85807FFC
:10F530008A8762E0CE0109960E94062729833A83D2
:10F540004B835C836D837E838F83988779018A01E7
:10F550009B01AC016FEFC201ECCED3011496ED918B
:10F56000FC91808191810F9424376DE774E28EEBDA
:10F5700091E10F9477358EEB91E10F9478345ACE68
:10F580006BE674E28EEB91E10F94773569A98EEB0F
:10F5900091E10E9474F68EEB91E10F947834A1CD45
:10F5A0002F923F924F925F926F927F928F929F9293
:10F5B000AF92BF92CF92DF92EF92FF920F931F9381
:10F5C000CF93DF93CDB7DEB768970FB6F894DEBF61
:10F5D0000FBECDBF1C01DC0114968D919C91159737
:10F5E000892B99F41296ED91FC91FA83E98389E1D4
:10F5F00090E00F949361BC0189819A810E944CB480
:10F60000D10115969C938E931497F1010480F58196
:10F61000E02DFE83ED83EF2B69F46BEC73E287E161
:10F6200091E10F94773587E191E10F94783490E080
:10F6300080E07FC4AD81BE811D921C92F1010280E9
:10F64000F381E02DF88FEF8B309791F084819581D5
:10F650009A838983009761F0DC0118968C91189742
:10F660008F70853029F4CD010E9434F7811186C056
:10F6700061E973E287E191E10F94773561E070E031
:10F68000F10184819581892B11F470E060E087E1BC
:10F6900091E10E947BF66FE873E287E191E10F94BC
:10F6A000773561E070E0D10112968D919C91892BA4
:10F6B00011F470E060E087E191E10E947BF66DE873
:10F6C00073E287E191E10F947735D1011296ED91C4
:10F6D000FC9161E070E084819581892B11F470E0E8
:10F6E00060E087E191E10E947BF66BE873E287E1DD
:10F6F00091E10F947735D1011296ED91FC91048040
:10F70000F581E02D80858F7061E070E0853011F427
:10F7100070E060E087E191E10E947BF669E873E2C6
:10F7200087E191E10F947735D1011296ED91FC912B
:10F73000848195810E9434F761E070E0823010F09E
:10F7400070E060E087E191E10E947BF687E191E162
:10F750000F94783465EA73E287E191E10F9477358D
:10F7600087E191E10F947834D101ED91FC9104840B
:10F77000F585E02D61E0C101199559CF60E08981DF
:10F780009A810E9462F69E8B8D8B009729F0FC0176
:10F7900080858F70853039F06FE673E287E191E103
:10F7A0000F947735D3CF8D899E890E9434F781508D
:10F7B000883008F099C1E82FF0E08827ED51F4482F
:10F7C0008F4F0D94966B467D1A7DED7C6D7C557C3C
:10F7D000557C407CEB7B67E08D899E890E9462F6B8
:10F7E000FC0190859F70933009F03FC041845284A2
:10F7F0006384748411E066E08D899E890E9462F6BC
:10F80000FC0190859F70933009F042C081859285FC
:10F81000A385B48589839A83AB83BC8311E064E0BC
:10F820008D899E890E9462F6FC0180858F708330ED
:10F8300009F04CC061857285838594850F949A6C1C
:10F840004B0163E08D899E890E9462F6FC018085F0
:10F850008F70833009F05CC081859285A385B48563
:10F86000898B9A8BAB8BBC8B60C0923049F46185DD
:10F870007285838594850F94C8692B013C01BACFAA
:10F88000412C512C1FE7612E13E4712E10E0B3CFF1
:10F890009230B9F461857285838594850F94C86927
:10F8A00069837A838B839C83B9CF412C512CBFE72A
:10F8B0006B2EB3E47B2E19821A821B821C8210E00D
:10F8C000AECF19821A821B821C82A9CF8230C1F46A
:10F8D00081849284A384B484B4CFF0EC8F2EF7E2B9
:10F8E0009F2EF9E0AF2EB12C412C512CAFE76A2EA0
:10F8F000A3E47A2E19821A821B821C8210E0A1CF07
:10F90000E0EC8E2EE7E29E2EE9E0AE2EB12C99CFF0
:10F91000823009F07DC061857285838594850F945E
:10F92000C869698B7A8B8B8B9C8B62E08D899E89F1
:10F930000E9462F6FC0180858F70833009F06DC0F3
:10F9400081859285A385B48589879A87AB87BC8793
:10F9500061E08D899E890E9462F6FC0180858F702E
:10F96000833009F086C081859285A385B4858D8713
:10F970009E87AF87B88B60E08D899E890E9462F672
:10F98000FC0190859F70933009F0A3C0C184D2849C
:10F99000E384F48420E030E0A901C701B6010F94AC
:10F9A000C16987FFCCC0F7FAF094F7F8F094A1E0B2
:10F9B000B0E0BE8BAD8BAF89B88D1696ED91FC9102
:10F9C00080858F70823009F4BDC0833009F4CAC2CB
:10F9D00080E090E0A0EAB1E4C9C260EC862E67E264
:10F9E000962E69E0A62EB12C80E090E0A0EAB0E46B
:10F9F000898B9A8BAB8BBC8B412C512C7FE7672E6C
:10FA000073E4772E19821A821B821C8210E08DCF3C
:10FA100080E090E0A0EAB0E423CF823029F5618550
:10FA20007285838594850F94C86969877A878B87E7
:10FA30009C878ECF40EC842E47E2942E49E0A42E82
:10FA4000B12C80E090E0A0EAB0E4898B9A8BAB8B7C
:10FA5000BC8B412C512C5FE7652E53E4752E198227
:10FA60001A821B821C8210E019861A861B861C864D
:10FA70006FCF823049F561857285838594850F94B7
:10FA8000C8696D877E878F87988B75CF20EC822E13
:10FA900027E2922E29E0A22EB12C80E090E0A0EA8D
:10FAA000B0E4898B9A8BAB8BBC8B412C512C3FE7FC
:10FAB000632E33E4732E19821A821B821C8210E09B
:10FAC00019861A861B861C861D861E861F86188A26
:10FAD00052CF923089F561857285838594850F9424
:10FAE000C8696B017C0156CF80EC882E87E2982E86
:10FAF00089E0A82EB12C80E090E0A0EAB0E4898BE8
:10FB00009A8BAB8BBC8B412C512C9FE7692E93E4D5
:10FB1000792E19821A821B821C8210E01E8A1D8A8D
:10FB200019861A861B861C861D861E861F86188AC5
:10FB3000C12CD12C76013FCF1E8A1D8AF9CF1E8A97
:10FB40001D8A39CF61857285838594850F94C86934
:10FB5000ED81FE816287738784879587AD81BE8141
:10FB600016961D921D921D921C921997FD011282EC
:10FB70001382148215820F941709AD81BE815296AB
:10FB80006D937D938D939C935597D1011496ED9130
:10FB9000FC9101E0068B908E878A61E0C1010E9492
:10FBA0007177F101A480B580D5018D919C9166E5B6
:10FBB00073E2892B09F0F2CD88E490E00F94936111
:10FBC000988F8F8BC5010296EF89F88D978F868F5E
:10FBD0000496958F848FFAE0AF0EB11CAF89B88D73
:10FBE0009196BC92AE929097FD01EA5BFF4F108216
:10FBF00038971082118212821382349680E090E04E
:10FC0000AFE7B3E480839183A283B38384E690E07B
:10FC1000A0E0B0E0EF89F88D82AF93AFA4AFB5AFAD
:10FC20006D897E89CF010F94E53620E030E0A9018F
:10FC3000C701B6010F94C16987FDA1C020E030E083
:10FC4000A9016D857E858F8598890F94C16987FD8F
:10FC500096C020E030E0A90169857A858B859C8576
:10FC60000F94C16987FD8BC081E090E0AF89B88DAA
:10FC70005B969C938E935A97FD01E95BFF4F00833F
:10FC8000FD01C082D182E282F3828D859E85AF859F
:10FC9000B88984839583A683B78389859A85AB8544
:10FCA000BC8580879187A287B38762AD73AD84AD31
:10FCB00095AD0F94C66920E030E04AE754E40F9414
:10FCC000216C4B015C01AF89B88D1C96CD92DD9201
:10FCD000ED92FC921F97AC019B016D857E858F850F
:10FCE00098890F94276A6D837E838F839887EF8925
:10FCF000F88D608B718B828B938BA5019401698544
:10FD00007A858B859C850F94216C4B015C01AF89B2
:10FD1000B88D54968D929D92AD92BC9257975896FD
:10FD20008D919C91019759F5A701960160E070E0D3
:10FD3000CB010F94B46BEF89F88D64877587868744
:10FD400097872D813E814F81588560E070E0CB011F
:10FD50000F94B46BAF89B88D50966D937D938D934E
:10FD60009C935397A501940160E070E0CB010F9440
:10FD7000B46BEF89F88D648B758B868B978B0F94A2
:10FD80001709AF89B88DDA96CD90DD90ED90FC9093
:10FD9000DD976C197D098E099F09FD0166A377A384
:10FDA00080A791A79E961D921D921D921C92D1979D
:10FDB00080E090E0A0ECBFE782A393A3A4A3B5A347
:10FDC00012A613A614A615A6D1011496ED91FC91C6
:10FDD0008F89988D91838083009709F4BBCC7C0137
:10FDE00096E4E90EF11CD7018C91811104C08F8932
:10FDF000988D0F94243781E0F7018083D101149608
:10FE0000ED91FC91808191819E838D83112309F472
:10FE100052C0A301920169817A818B819C810F94E8
:10FE2000C96C87FF48C0ED81FE81FE9689819A8169
:10FE3000AB81BC8180839183A283B383ED81FE81FA
:10FE4000EE5BFF4F4082518262827382ED81FE81C0
:10FE5000EA5BFF4F8081882371F1AD81BE815E96A0
:10FE6000ED90FC90F70180809180A280B380A50185
:10FE70009401C301B2010F94C16987FF7EC0D7010D
:10FE80004D925D926D927C921397AD81BE81D29618
:10FE9000CD90DD90ED90FC90D597A7019601C30120
:10FEA000B2010F94C16987FF7DC0ED81FE8142AA36
:10FEB00053AA64AA75AA20E030E04AE754E46989AD
:10FEC0007A898B899C890F94276A0F94936C8D8112
:10FED0009E810F94723967EB73E28DE091E10F948C
:10FEE0007735D1011296ED91FC910280F381E02DDE
:10FEF000608171818DE091E10F9420358DE091E179
:10FF00000F947834D1011496ED91FC9180E090E04B
:10FF1000A0E0B0EC86879787A08BB18BD101ED91E3
:10FF2000FC910484F585E02D62E0C101199581E022
:10FF300090E068960FB6F894DEBF0FBECDBFDF919C
:10FF4000CF911F910F91FF90EF90DF90CF90BF90D6
:10FF5000AF909F908F907F906F905F904F903F9069
:10FF60002F90089581859285A385B485ED81FE81CA
:10FF700082879387A487B587F1CDA5019401698114
:10FF80007A818B819C810F94C96C18160CF07DCFFF
:10FF900089819A81AB81BC81F70180839183A2839F
:10FFA000B38373CFA701960169817A818B819C818C
:10FFB0000F94C96C18160CF07ECF89819A81AB81A1
:10FFC000BC81ED81FE8182AB93ABA4ABB5AB73CFAB
:10FFD0004F925F926F927F928F929F92AF92BF9259
:10FFE000CF92DF92EF92FF920F931F93CF93DF9305
:10FFF000CDB7DEB760970FB6F894DEBF0FBECDBFAA
:020000021000EC
:100000006130710509F4DDC1DC011496ED91FC91BC
:100010003097C9F481E090E060960FB6F894DEBFA7
:100020000FBECDBFDF91CF911F910F91FF90EF9049
:10003000DF90CF90BF90AF909F908F907F906F9008
:100040005F904F90089520813181232B19F33C015B
:10005000DC01ED91FC910284F385E02D1995029766
:10006000C9F6F301E280F380E114F10499F2C701CB
:100070000E949BBC823071F240E051E060E070E091
:10008000C7010E9458B6672B682B692B19F6D3015C
:100090001496ED91FC9180819181FC01EA5BFF4F08
:1000A0002081222309F455C10F947E37882309F457
:1000B00050C1D3011496ED91FC9186898823A1F05B
:1000C000C3010E94A2626B017C0120E030E0A90123
:1000D0000F94C96C87FD08C0D3011496ED91FC9173
:1000E000C282D382E482F5826AE074E28EEB91E10F
:1000F0000F947735D3011296ED91FC910280F38134
:10010000E02D608171818EEB91E10F94203564E0E8
:1001100074E28EEB91E10F947735D3011496ED9153
:10012000FC9142855385648575858EEB91E10E9433
:10013000F5FA6FEF73E28EEB91E10F947735D3010F
:100140001496ED91FC9146815781608571858EEB07
:1001500091E10E94F5FA6CEB77E08EEB91E10F9460
:100160002035D3011496ED91FC9142815381648135
:1001700075818EEB91E10E94F5FA6BEF73E28EEBE5
:1001800091E10F947735D3011496ED91FC91019094
:10019000F081E02D40815181628173818EEB91E18C
:1001A0000E94F5FA67EF73E28EEB91E10F947735D9
:1001B000D3011496ED91FC910190F081E02D4481E2
:1001C0005581668177818EEB91E10E94F5FA63EFAC
:1001D00073E28EEB91E10F947735D3011496ED9194
:1001E000FC910190F081E02D4085518562857385F9
:1001F0008EEB91E10E94F5FAD3011496ED91FC91FA
:100200008689882331F06CEE73E28EEB91E10F94D6
:1002100077358EEB91E10F947834F301E480F5802B
:10022000D70156968C918111F5CE0281138161E040
:10023000F801848195810E9462F62C0120E030E073
:10024000A901D7011E966D917D918D919C91519739
:100250000F94C16981110CC020E030E0A901F701C1
:1002600062817381848195810F94C96C18165CF04A
:1002700040E050E061E070E0C8010E9458B6672B92
:10028000682B692B31F119861A861B861C861D8600
:100290001E861F86188A8A85807F8A8761E0CE0144
:1002A00009960E94062729833A834B835C836D83DA
:1002B0007E838F839887912C812CB12CA12CD12CFB
:1002C000C12C79018A019B01AC016FEFC2010E9430
:1002D0006B7440E050E061E070E0D30112968D91C4
:1002E0009C910E9406B6D3011496ED91FC91328147
:1002F00063815481458119861A861B861C868A85EE
:10030000807F8760F82E8A87232F832F962FA52F33
:10031000B42F8D879E87AF87B88B912C812CB12C01
:10032000A12CD12CC12CE9840B851C853E854F85E1
:1003300058896FEFC2010E946B74D3011496ED913E
:10034000FC9182819381A481B58186879787A08B58
:10035000B18BD3011496ED91FC91868981115ACE0F
:100360008789908D009709F455CE28EE33E0829F5F
:100370002001839F500C929F500C11240F94170959
:10038000D3011496ED91FC914114510499F062014E
:10039000F12CE12C0289138924893589AB01BC0138
:1003A000401B510B620B730B4C155D056E057F05F1
:1003B00008F430CE81E0868B61E0C3010E94717742
:1003C00029CE90E080E028CE2F923F924F925F920C
:1003D0006F927F928F929F92AF92BF92CF92DF9255
:1003E000EF92FF920F931F93CF93DF93CDB7DEB7BA
:1003F000EF970FB6F894DEBF0FBECDBF09AB1AABB7
:100400002BAB3CAB4DAB5EAB6FAB78AFFC01068169
:1004100017810115110509F4DDC11C012FE030E041
:1004200040E050E062EC77E0C8010F9491552B0159
:10043000D9A8DD2009F495C020E030E0A9016AECDC
:1004400077E0C8010F9491557B0120E030E0A901CD
:1004500063ED77E0C8010F949155CB01892B79F0BA
:10046000F2E0DF1661F0CE01C1960E94062729A7AF
:100470003AA74BA75CA76DA77EA78FA798AB89A9C2
:100480008E151F0431F4C20184709927892B09F05D
:1004900068C06FED77E08EEB91E10F942035CE01CF
:1004A000C1960E94F4258EEB91E10F947834198661
:1004B0001A861B861C868A85807F8A8789A98987F8
:1004C00089859A85AB85BC85898B9A8BAB8BBC8BD8
:1004D0001D8A1E8A1F8A188E61E0CE0141960E94F5
:1004E000E426298F4B8F5C8F6D8F7E8F8F8F98A323
:1004F000307F3A8F88E0FE017996DE0111960190F7
:100500000D928A95E1F788E0FE013196DE01919621
:1005100001900D928A95E1F7912C812CB12CA12CA0
:10052000D12CC12CE9A0FAA00BA11CA12DA13EA1A8
:100530004FA158A56FEFF101868197810E946B74DE
:1005400049A96AEC77E0F101868197810E94D56321
:100550004FEF5FEF65EF77E0F101868197810E94B1
:100560005E648AA98F70D9F481E090E0EF960FB6AF
:10057000F894DEBF0FBECDBFDF91CF911F910F91D9
:10058000FF90EF90DF90CF90BF90AF909F908F90B3
:100590007F906F905F904F903F902F900895F10162
:1005A000068117812FEF3FEFA90165EF77E0C801C2
:1005B0000F9491556B017FAF6EAF20E030E0A90141
:1005C0006EEF77E0C8010F9428554B015C012FEFC7
:1005D0003FEFA90167E078E0C8010F9491556AAF39
:1005E0007BAF8CAF9DAF8AAD9BAD8230910519F08A
:1005F000019609F068C021E029AF8EAD9FAD1816B5
:1006000019060CF019AE8BA9823009F479C0873035
:1006100009F0CAC0E1E04E225524452869F0CE0118
:10062000C1960E94BB290D2C000CEE08FF08C616CF
:10063000D706E806F90619F16CE078E08EEB91E157
:100640000F942035CE01C1960E94F4258EEB91E1E6
:100650000F94783460E0CE01C1960E940627912C59
:10066000812CB12CA12CD12CC12C79018A019B01A8
:10067000AC016FEFF101868197810E946B74CE010E
:10068000C1960E94BB299B01AC0165EF77E0F101A7
:10069000868197810E940264CE01C1960E94BB2987
:1006A000611571058105910589F4F9ADFF2309F400
:1006B0005BCF4AAD5BAD62E278E0F1018681978164
:1006C0000E945E6451CF91E099AF9DCF1616170638
:1006D000180619060CF048CFF9ADF11145CFF1011C
:1006E000068117812FE030E040E050E062E278E0E0
:1006F000C8010F949155AB016AEC77E0C801E0CFD7
:10070000F2E04F2255244528B1F0CE01C1960E9457
:1007100075296B017C01C501B4010F94936C072E00
:10072000000C880B990B0F94C869A70196010F94D0
:10073000C169882359F16AE278E08EEB91E10F9468
:100740002035CE01C1960E94F4258EEB91E10F94E5
:10075000783460E0CE01C1960E940627298B3A8B3F
:100760004B8B5C8B6D8B7E8B8F8B988F912C812C20
:10077000B12CA12CD12CC12C79018A019B01AC0197
:100780006FEFF101868197810E946B74CE01C19653
:100790000E9475299B01AC016EEF77E0F101868123
:1007A00097810E943064E0CE60E0CE01C1960E9445
:1007B0000627912C812CB12CA12CD12CC12C790194
:1007C0008A019B01AC016FEFF101868197810E9444
:1007D0006B74CACE90E080E0C9CEEF92FF920F9387
:1007E0001F93CF93DF9300D000D01F921F92CDB7FD
:1007F000DEB709831A832B833C834D835E836F832B
:100800007887DC011696ED91FC91309709F445C08C
:1008100020852F70263031F441855285638574859B
:1008200060FD3BC07C0160E478E08EEB91E10F94C9
:1008300020358EEB91E10F947834F7010681178112
:1008400025E130E040E050E063E578E0C8010F9436
:100850009155AB016FE478E0C8010E945E640981A4
:100860001A812B813C814D815E816F817885C70122
:100870000E94E481D7011696ED91FC91309769F0C2
:1008800080858F70863049F481859285A385B485F3
:10089000A16081879287A387B48728960FB6F894C2
:1008A000DEBF0FBECDBFDF91CF911F910F91FF90A3
:1008B000EF9008956F927F928F929F92AF92BF9226
:1008C000CF92DF92EF92FF920F931F93CF93DF931C
:1008D000CDB7DEB760970FB6F894DEBF0FBECDBFC1
:1008E000E986FA860B871C872D873E874F87588BB2
:1008F000009731F1FC0120852F70263009F50E9408
:10090000EAF53C01892BE1F090E080E0CC2029F071
:100910006FEE75E0C3010E94EAF5BC01CE010996B5
:100920000E94FF29912C812CB12CA12CD12CC12CFF
:1009300079018A019B01AC016FEFC3010E946B74C6
:1009400060960FB6F894DEBF0FBECDBFDF91CF919A
:100950001F910F91FF90EF90DF90CF90BF90AF90DD
:100960009F908F907F906F9008952F923F924F921B
:100970005F926F927F928F92AF92BF92CF92DF92EF
:10098000EF92FF920F931F93CF93DF93CDB7DEB714
:10099000AA970FB6F894DEBF0FBECDBF8C013B0106
:1009A000342E20E030E0A90167E578E0C3010F9420
:1009B000915521E0672B682B692B09F420E0231562
:1009C00009F4B2C06DE578E0C3010E94EAF52C019C
:1009D0006FE071E28EEB91E10F947735632D70E05B
:1009E0008EEB91E10E947BF68EEB91E10F947834CF
:1009F00067E578E0C3010F9401555C01009711F1A0
:100A0000FC018085982F9F70923039F0933079F0F7
:100A1000911118C0807F82608087832D90E0B0E0C4
:100A2000A0E0F50181879287A387B4870BC0632D6F
:100A300070E090E080E00F94C669F50161877287ED
:100A400083879487332009F487C080913F13909166
:100A50004013059799F1F80122803380F301A080BB
:100A6000B18019821A821B821C821D821E821F8203
:100A700018868A81807F8A836EE0CE0101960E946B
:100A8000062729873A874B875C876D877E878F8704
:100A9000988B67E0CE0109960E94E426022F242F4E
:100AA00088248394C12CE0E1DE2EE12CF12C132F5D
:100AB000352FAB01BC01C1010E947CB619821A829C
:100AC0001B821C821D821E821F8218868A81807F63
:100AD0008A836EE0CE0101960E940627298B3A8B0D
:100AE0004B8B5C8B6D8B7E8B8F8B988F67E0CE01F1
:100AF00041960E94E42629873A874B875C876D8759
:100B00007E878F87988BC12C79018A019B01AC016C
:100B100063E979E0C2010E945A8450E040E063E951
:100B200079E0C3010E945E64AA960FB6F894DEBF16
:100B30000FBECDBFDF91CF911F910F91FF90EF902E
:100B4000DF90CF90BF90AF908F907F906F905F902D
:100B50004F903F902F90089563E979E0C3010E9480
:100B6000EAF51C01009701F3FC0180858F7082304B
:100B7000D9F680913F1390914013059709F442C034
:100B80006185728583859485F8010280F381E02D6B
:100B9000FAA7E9A7F301A080B18019821A821B820B
:100BA0001C821D821E821F8218862A81207F2A8332
:100BB000CE0101960E94E02729873A874B875C8700
:100BC0006D877E878F87988B67E0CE0109960E949C
:100BD000E426022F242F098F3A8F4B8F5C8F6D8F65
:100BE0007E8F8F8F98A388248394C12C40E2D42ECB
:100BF000E12CF12C132F352FAB01BC0189A59AA54F
:100C00000E947CB619861A861B861C861D861E8647
:100C10001F86188A8A85807F8A87F101618572859F
:100C2000CE0109960E94E027298B3A8B4B8B5C8B77
:100C30006D8B7E8B8F8B988F67E0CE0141960E94E3
:100C4000E42629833A834B835C836D837E838F8381
:100C50009887CC24C39479018A019B01AC0163E994
:100C600079E0C2010E945A845FCF2F923F924F9247
:100C70005F926F927F928F929F92AF92BF92CF922C
:100C8000DF92EF92FF920F931F93CF93DF93CDB735
:100C9000DEB7C550D1400FB6F894DEBF0FBECDBF52
:100CA000C752DF4F0883C95DD040C652DF4F18835B
:100CB000CA5DD040C552DF4F2883CB5DD040C452BF
:100CC000DF4F3883CC5DD040C352DF4F4883CD5DCA
:100CD000D040C252DF4F5883CE5DD040C152DF4F6B
:100CE0006883CF5DD040C052DF4F7883C05ED04074
:100CF000DC0114962D913C911597232B09F468C6BD
:100D000016962D913C91232B09F462C6202F2A5070
:100D1000223008F45DC6CB5FDE4FC882C550D1409B
:100D2000C650DF4FF982E882CA5FD040CF51DF4F13
:100D300099838883C15ED040C552DF4F8881CB5DE7
:100D4000D040E82FF0E0CB51DF4FF983E883C55E58
:100D5000D04061E678E08EEB91E10F942035C650EB
:100D6000DF4F68817981CA5FD0408EEB91E10F94AB
:100D7000203560EA75E08EEB91E10F942035CE01CD
:100D800087529F4F0E94F425C752DF4F1881C95DDB
:100D9000D040112381F0CB51DF4F28813981C55ECE
:100DA000D040232B41F441E050E0CB51DF4F598339
:100DB0004883C55ED04020E030E0A9016DE678E0D0
:100DC000CF51DF4FA881B981C15ED04016968D9179
:100DD0009C910F949155CE5FDE4F6883C250D140F5
:100DE000CA50DF4F6883C65FD040C950DF4F788359
:100DF000C75FD040C552DF4F8881CB5DD040873080
:100E000009F066C0113109F452C1123109F4ADC1C3
:100E1000103109F008C26FEF70E0CE0187529F4F8A
:100E20000E94E027CF52DF4F2883C15DD040CE52D1
:100E3000DF4F3883C25DD040CD52DF4F4883C35D62
:100E4000D040CC52DF4F5883C45DD040CB52DF4FEF
:100E50006883C55DD040CA52DF4F7883C65DD040FD
:100E6000C952DF4F8883C75DD040C852DF4F988397
:100E7000C85DD04060E0CE0187529F4F0E94062798
:100E8000C753DF4F2883C95CD040C653DF4F388338
:100E9000CA5CD040C553DF4F4883CB5CD040C453BD
:100EA000DF4F5883CC5CD040C353DF4F6883CD5CA9
:100EB000D040C253DF4F7883CE5CD040C153DF4F68
:100EC0008883CF5CD040C053DF4F9883C05DD04053
:100ED000C650DF4FE881F981CA5FD040EF2BA1F403
:100EE000CB51DF4F28813981C55ED0402330310599
:100EF00009F462C20CF0D2C12130310509F409C5F0
:100F00002230310509F414C3CF51DF4FA881B981D4
:100F1000C15ED0401496ED91FC91309711F40C9481
:100F2000859326803780C050DF4F19821882C050C9
:100F3000D140CC50DF4F19821882C45FD040C251DB
:100F4000DF4F19821882CE5ED040C551DF4F198223
:100F50001882CB5ED040CE50DF4F19821882C25F1C
:100F6000D0402114310411F40C949D9363E979E08D
:100F7000C1010E94EAF5C751DF4F99838883C95E9A
:100F8000D0406BED77E0C1010E94EAF5CD51DF4F13
:100F900099838883C35ED0406DE578E0C1010E94EB
:100FA000EAF5C850DF4F99838883C85FD04064EC6E
:100FB00076E0C1010E94EAF55C01C751DF4FE8818C
:100FC000F981C95ED040309711F40C94C992CD518B
:100FD000DF4F28813981C35ED0402115310511F4DE
:100FE0000C94C99280858F70823011F00C94C99254
:100FF000D90118968C918F70823011F00C94C9929F
:101000002CE330E040E050E06AE077E0C1010F946B
:101010009155C450DF4F688379838A839B83CC5F6B
:10102000D04020E030E0A90167E578E0C1010F94ED
:1010300091556B017C01B1E0C351DF4FB883CD5EA8
:10104000D040C114D104E104F10429F4C351DF4FAD
:101050001882CD5ED040C650DF4FE881F981CA5F6B
:10106000D040309711F40C944D92BF01D1018D9175
:101070009C910F94F76F892B11F00C944D92CB51EA
:10108000DF4FE881F981C55ED040E230F10511F40F
:101090000C9435910CF06FC4412C512C32013197D6
:1010A00009F439C6412C512C32010C94959060E81A
:1010B00070E0CE0187529F4F0E94E027CF53DF4F51
:1010C0002883C15CD040CE53DF4F3883C25CD04010
:1010D000CD53DF4F4883C35CD040CC53DF4F5883A0
:1010E000C45CD040CB53DF4F6883C55CD040CA534B
:1010F000DF4F7883C65CD040C953DF4F8883C75C1D
:10110000D040C853DF4F9883C85CD04060E0CE0128
:1011100087529F4F0E940627C754DF4F2883C95B21
:10112000D040C654DF4F3883CA5BD040C554DF4F30
:101130004883CB5BD040C454DF4F5883CC5BD04056
:10114000C354DF4F6883CD5BD040C254DF4F7883F8
:10115000CE5BD040C154DF4F8883CF5BD040C054BA
:10116000DF4F9883C05CD040B3CE60E470E0CE0126
:1011700087529F4F0E94E027CF54DF4F2883C15BE7
:10118000D040CE54DF4F3883C25BD040CD54DF4FC8
:101190004883C35BD040CC54DF4F5883C45BD040FE
:1011A000CB54DF4F6883C55BD040CA54DF4F788390
:1011B000C65BD040C954DF4F8883C75BD040C8545A
:1011C000DF4F9883C85BD04060E0CE0187529F4FCD
:1011D0000E940627C755DF4F2883C95AD040C655FD
:1011E000DF4F3883CA5AD040C555DF4F4883CB5AAA
:1011F000D040C455DF4F5883CC5AD040C355DF4F41
:101200006883CD5AD040C255DF4F7883CE5AD04044
:10121000C155DF4F8883CF5AD040C055DF4F9883E8
:10122000C05BD04055CEC652DF4F8881CA5DD040EA
:101230008F7009F44DCECE0187529F4F0E94BB297B
:10124000CE0187529F4F0E94E027CF55DF4F288362
:10125000C15AD040CE55DF4F3883C25AD040CD5509
:10126000DF4F4883C35AD040CC55DF4F5883C45A10
:10127000D040CB55DF4F6883C55AD040CA55DF4FA9
:101280007883C65AD040C955DF4F8883C75AD040AB
:10129000C855DF4F9883C85AD0401ACECB51DF4F84
:1012A00048815981C55ED0404730510509F4D3C00B
:1012B0004830510509F028CEC752DF4F8881C95DFB
:1012C000D040882309F47FC069E272E28EEB91E19D
:1012D0000F9477356FE172E28EEB91E10F947735E1
:1012E000C752DF4F6881C95DD0408EEB91E10E940B
:1012F00074F68EEB91E10F947834CF51DF4FE88193
:10130000F981C15ED040068117810115110509F4EC
:1013100041C0C752DF4FF880C95DD0406F2C712C9F
:1013200020E030E0A9016AEC77E0C8010F94915504
:101330004B0120E030E0A90167E078E0C8010F949C
:1013400091551B012FEF3FEFA90165EF77E0C80131
:101350000F949155232809F016C26FEE78E08EEBBA
:1013600091E10F942035B3018EEB91E10E947BF661
:101370008EEB91E10F947834A3016AEC77E0CF51C2
:10138000DF4FA881B981C15ED04016968D919C91A6
:101390000E945E64C752DF4F4881C95DD04067E05C
:1013A00078E0CF51DF4FE881F981C15ED04086817E
:1013B00097810E94D56307C0C652DF4F8881CA5DFE
:1013C000D0408F7029F466246A94762C0C94A793ED
:1013D00068E772E28EEB91E10F9477356AE672E28C
:1013E0008EEB91E10F947735CE0187529F4F0E948B
:1013F0007529AB01BC018EEB91E10E94F5FA8EEBF1
:1014000091E10F947834CF51DF4FA881B981C15E4B
:10141000D04012960D911C914FEF5FEFBA0180E022
:101420000F945256AB01BC01C8010E948FB4CE018B
:1014300087529F4F0E9475299B01AC016DE775E0B3
:10144000CF51DF4FE881F981C15ED040868197811D
:101450000E943064B8CFC652DF4F8881CA5DD04049
:101460008F7009F4B0CF63E672E28EEB91E10F94D6
:1014700077356AE572E28EEB91E10F947735CE0114
:1014800087529F4F0E94BB29AB01BC012AE030E08C
:101490008EEB91E10F949A348EEB91E10F947834B6
:1014A000CE0187529F4F0E94BB296B01CF51DF4F66
:1014B000A881B981C15ED04016968D919C9100970C
:1014C00011F120E030E0A90163E979E00F94915532
:1014D000C616D706C1F067E778E08EEB91E10F946E
:1014E00020358EEB91E10F9478344FEF5FEF65EF8D
:1014F00077E0CF51DF4FE881F981C15ED04086812E
:1015000097810E945E64CE0187529F4F0E94BB2943
:101510009B01AC0163E979E0CF51DF4FA881B9812C
:10152000C15ED04016968D919C910E9402644BCF73
:10153000C652DF4F8881CA5DD0408F7009F443CF17
:1015400063E572E28EEB91E10F9477356AE472E223
:101550008EEB91E10F947735CE0187529F4F0E9419
:101560007529AB01BC018EEB91E10E94F5FA8EEB7F
:1015700091E10F947834CE0187529F4F0E947529D4
:10158000CF51DF4FE881F981C15ED04006811781DC
:101590000115110571F10F94936C1B012FEF3FEFB3
:1015A000A9016EEF77E0C8010F9491556B01CB0153
:1015B0006F3F760709F06CC06CE978E08EEB91E143
:1015C0000F942035B1018EEB91E10E947BF68EEBFA
:1015D00091E10F947834A1016EEF77E0CF51DF4FA6
:1015E000A881B981C15ED04016968D919C910E94D0
:1015F0005E64CE0187529F4F0E9475299B01AC010A
:1016000063E578E0CF51DF4FE881F981C15ED040DA
:10161000868197810E943064CE0187529F4F0E943D
:1016200075296B017C0120E030E040EF51E40F941C
:10163000C169882351F020E030E048E851E4C70157
:10164000B6010F94C1698111BECECF51DF4FA88181
:10165000B981C15ED0401696ED91FC91309769F04A
:1016600080858F70863049F481859285A385B48505
:10167000A16081879287A387B48760E372E28EEBD3
:1016800091E10F9477358EEB91E10F9478349BCEF6
:10169000892B09F4AECF2616370609F4AACF6DEBD5
:1016A00078E08EEB91E10F942035B6018EEB91E15D
:1016B0000E947BF661EE78E08EEB91E10F9420358D
:1016C000B1018EEB91E10E947BF68EEB91E10F94DC
:1016D000783466EE78E0CF51DF4FE881F981C15E62
:1016E000D040868197810E94EAF53C01892B09F45C
:1016F00072CF198A1A8A1B8A1C8A1D8A1E8A1F8A1F
:10170000188E8A89807F8A8BA101032C000C660BBE
:10171000770BCE0141960E94282729873A874B876D
:101720005C876D877E878F87988B62E0CE010996F4
:101730000E94E42629833A834B835C836D837E83F6
:101740008F8398876FEE75E0C3010E94EAF5BC01B4
:10175000CE0101960E94FF29298F3A8F4B8F5C8F13
:101760006D8F7E8F8F8F98A3912C812CB12CA12C03
:10177000D12CC12C79018A019B01AC016FEFC3010F
:101780000E946B7428CF8114910409F403CE68146D
:10179000790409F4FFCDB2E06B16710419F4672BDC
:1017A00009F499C061E179E08EEB91E10F94203565
:1017B000B4018EEB91E10E947BF661EE78E08EEB56
:1017C00091E10F942035B3018EEB91E10E947BF6FD
:1017D0008EEB91E10F947834CF51DF4FE881F9819E
:1017E000C15ED04084819581F2E0FF1286C0892BD2
:1017F00041F0CF51DF4F88819981C15ED0400E9476
:10180000D29F66EE78E0CF51DF4FA881B981C15EEB
:10181000D04016968D919C910E94EAF52C01892B5F
:1018200009F459C019A61AA61BA61CA61DA61EA619
:101830001FA618AA8AA5807F8AA76F2DCE01899638
:101840000E94062729A33AA34BA35CA36DA37EA302
:101850008FA398A761E0CE0181960E94E426298F8C
:101860004B8F5C8F6D8F7E8F8F8F98A3307F3A8FD9
:1018700088E0FE017996DE01199601900D928A9515
:10188000E1F788E0FE013996DE01519601900D9254
:101890008A95E1F788E0FE017196DE0111960190CC
:1018A0000D928A95E1F76FEE75E0C2010E94EAF5AC
:1018B000BC01CE0101960E94FF29912C812CB12CF4
:1018C000A12CD12CC12C79018A019B01AC016FEFB5
:1018D000C2010E946B74A3016AEC77E0CF51DF4F25
:1018E000E881F981C15ED040868197810E945E6463
:1018F0004FEF5FEF65EF77E042CD892B09F481CFA1
:10190000CF51DF4F88819981C15ED0400E94479FAF
:1019100078CFC752DF4F8881C95DD0408031C0F495
:101920008E30D0F48130C1F0823009F04CCDCF51EF
:10193000DF4FA881B981C15ED04014968D919C91F2
:101940001597892B09F43FCDCD010E94D29F3BCD45
:101950008351843008F037CDCF51DF4FE881F981D2
:10196000C15ED04084819581892B09F42CCDCF01B3
:101970000E94479F28CDCB51DF4F28813981C55E1A
:10198000D0402330310509F40AC62730310509F06B
:1019900089CBD10118968C9118978F708630E9F415
:1019A00019968D919D910D90BC91A02D88279670D0
:1019B000AA27BB27892B8A2B8B2B79F06DE072E24B
:1019C0008EEB91E10F9477358EEB91E10F947834A3
:1019D0009EEF692E77247A94BAC6C652DF4F88816B
:1019E000CA5DD0408F7009F404C1CE0187529F4F69
:1019F0000E94BB299B01AC01CB5FDE4FB881C55073
:101A0000D140B11131C066E379E0C1010E940264A6
:101A10006DE379E08EEB91E10F942035CE01875292
:101A20009F4F0E94BB29AB01BC012AE030E08EEB46
:101A300091E10F949A348EEB91E10F947834A114D4
:101A4000B10491F0F50181859285A385B485009755
:101A5000A105B10549F08A5B9F4FDC018C91882379
:101A600019F06BEE71E2ACCFCE0187529F4F0E940E
:101A7000BB29CD51DF4FE881F981C35ED04001859C
:101A8000128523853485672B682B692B09F46FC079
:101A9000023011052105310509F04FC0CA50DF4F52
:101AA00028813981C65FD040232B09F446C0CE5F20
:101AB000DE4F6881C250D140CE0187529F4F0E94B5
:101AC0000627C756DF4F2883C959D040C656DF4F77
:101AD0003883CA59D040C556DF4F4883CB59D040D0
:101AE000C456DF4F5883CC59D040C356DF4F68836C
:101AF000CD59D040C256DF4F7883CE59D040C15621
:101B0000DF4F8883CF59D040C056DF4F9883C05AEB
:101B1000D0406FE579E08EEB91E10F942035CA500B
:101B2000DF4F68817981C65FD0408EEB91E10E94E2
:101B30007BF68EEB91E10F947834CE0187529F4F64
:101B40000E94BB29C751DF4FA881B981C95ED0402F
:101B500019966D937D938D939C931C97CD28CE28D9
:101B6000CF2809F40DC1412C512C3201B9C00230EB
:101B700011052105310509F3CA50DF4F488159810C
:101B8000C65FD040452BC9F262E0CE0187529F4F1D
:101B90000E940627CF56DF4F2883C159D040CE562A
:101BA000DF4F3883C259D040CD56DF4F4883C359E9
:101BB000D040CC56DF4F5883C459D040CB56DF4F6E
:101BC0006883C559D040CA56DF4F7883C659D04084
:101BD000C956DF4F8883C759D040C856DF4F988316
:101BE000C859D0406DE779E08EEB91E10F94203534
:101BF000A0CFC752DF4F8881C95DD0408E3009F039
:101C0000A9C041E0B101CF51DF4F88819981C15E08
